:1000000090490120AD5400007F270700995400005B
:10001000995400009954000099540000995400002C
:10002000000000000000000000000000E554000097
:10003000995400000000000031570000995400005E
:10004000F1570000F1570000F1570000F157000090
:10005000F1570000F1570000F1570000F157000080
:10006000F1570000F1570000F1570000F157000070
:10007000F1570000F1570000F1570000F157000060
:10026000F1570000F1570000D9630200F157000078
:10027000F1570000F1570000F1570000F15700005E
:10028000F1570000F1570000F1570000F15700004E
:10029000F1570000F1570000F1570000F15700003E
:1002A000F1570000F1570000F1570000F15700002E
:1004C80081F0004102E000BF83F0004330B54FEAFD
:1004D80041044FEA430594EA050F08BF90EA020F6A
:1004E8001FBF54EA000C55EA020C7FEA645C7FEAFD
:1004F800655C00F0E2804FEA5454D4EB5555B8BF20
:100508006D420CDD2C4480EA020281EA030382EA90
:10051800000083EA010180EA020281EA0303362D22
:1005280088BF30BD11F0004F4FEA01314FF4801CF5
:100538004CEA113102D0404261EB410113F0004F07
:100548004FEA03334CEA133302D0524263EB4303BE
:1005580094EA050F00F0A780A4F10104D5F1200E5C
:100568000DDB02FA0EFC22FA05F2801841F10001B7
:1005780003FA0EF2801843FA05F359410EE0A5F18B
:1005880020050EF1200E012A03FA0EFC28BF4CF0BC
:10059800020C43FA05F3C01851EBE37101F0004572
:1005A80007D54FF0000EDCF1000C7EEB00006EEB7F
:1005B8000101B1F5801F1BD3B1F5001F0CD3490809
:1005C8005FEA30004FEA3C0C04F101044FEA445260
:1005D80012F5800F80F09A80BCF1004F08BF5FEAE7
:1005E800500C50F1000041EB045141EA050130BDC7
:1005F8005FEA4C0C404141EB0101013C28BFB1F5D9
:10060800801FE9D291F0000F04BF01460020B1FA23
:1006180081F308BF2033A3F10B03B3F120020CDAF6
:100628000C3208DD02F1140CC2F10C0201FA0CF0D4
:1006380021FA02F10CE002F11402D8BFC2F1200C39
:1006480001FA02F120FA0CFCDCBF41EA0C019040EF
:10065800E41AA2BF01EB0451294330BD6FEA040438
:100668001F3C1CDA0C340EDC04F11404C4F1200223
:1006780020FA04F001FA02F340EA030021FA04F335
:1006880045EA030130BDC4F10C04C4F1200220FA8C
:1006980002F001FA04F340EA0300294630BD21FACA
:1006A80004F0294630BD94F0000F83F4801306BF90
:1006B80081F480110134013D4EE77FEA645C18BF84
:1006C8007FEA655C29D094EA050F08BF90EA020F1B
:1006D80005D054EA000C04BF1946104630BD91EA13
:1006E800030F1EBF0021002030BD5FEA545C05D116
:1006F8004000494128BF41F0004130BD14F5800455
:100708003CBF01F5801130BD01F0004545F0FE41C8
:1007180041F470014FF0000030BD7FEA645C1ABFFD
:10072800194610467FEA655C1CBF0B46024650EA34
:10073800013406BF52EA033591EA030F41F4002160
:1007480030BD00BF90F0000F04BF0021704730B5E6
:100758004FF4806404F132044FF000054FF00001BB
:1007680050E700BF90F0000F04BF0021704730B57C
:100778004FF4806404F1320410F0004548BF404251
:100788004FF000013EE700BF42004FEAE2014FEAA6
:1007980031014FEA02701FBF12F07F4393F07F4F81
:1007A80081F06051704732F07F4208BF704793F084
:1007B8007F4F04BF41F40021704730B54FF4607497
:1007C80001F0004521F000411CE700BF50EA01029A
:1007D80008BF704730B54FF000050AE050EA010243
:1007E80008BF704730B511F0004502D5404261EBB3
:1007F80041014FF4806404F132045FEA915C3FF4F4
:10080800D8AE4FF003025FEADC0C18BF03325FEA90
:10081800DC0C18BF033202EBDC02C2F1200300FA41
:1008280003FC20FA02F001FA03FE40EA0E0021FA66
:1008380002F11444BDE600BF70B54FF0FF0C4CF454
:10084800E06C1CEA11541DBF1CEA135594EA0C0F06
:1008580095EA0C0F00F0DEF82C4481EA030621EA41
:100868004C5123EA4C5350EA013518BF52EA03357C
:1008780041F4801143F4801338D0A0FB02CE4FF02E
:100888000005E1FB02E506F00042E0FB03E54FF05E
:100898000006E1FB03569CF0000F18BF4EF0010E56
:1008A800A4F1FF04B6F5007F64F5407404D25FEA52
:1008B8004E0E6D4146EB060642EAC62141EA555105
:1008C8004FEAC52040EA5E504FEACE2EB4F1FD0C47
:1008D80088BFBCF5E06F1ED8BEF1004F08BF5FEAC5
:1008E800500E50F1000041EB045170BD06F0004677
:1008F80046EA010140EA020081EA0301B4EB5C0424
:10090800C2BFD4EB0C0541EA045170BD41F480111B
:100918004FF0000E013C00F3AB8014F1360FDEBF40
:10092800002001F0004170BDC4F10004203C35DA1C
:100938000C341BDC04F11404C4F1200500FA05F39F
:1009480020FA04F001FA05F240EA020001F0004240
:1009580021F0004110EBD37021FA04F642EB0601B6
:100968005EEA430E08BF20EAD37070BDC4F10C04E0
:10097800C4F1200500FA04F320FA05F001FA04F2A4
:1009880040EA020001F0004110EBD37041F1000190
:100998005EEA430E08BF20EAD37070BDC4F120059B
:1009A80000FA05F24EEA020E20FA04F301FA05F203
:1009B80043EA020321FA04F001F0004121FA04F2AB
:1009C80020EA020000EBD3705EEA430E08BF20EA7B
:1009D800D37070BD94F0000F0FD101F000464000B5
:1009E80041EB010111F4801F08BF013CF7D041EA37
:1009F800060195F0000F18BF704703F0004652003B
:100A080043EB030313F4801F08BF013DF7D043EA0B
:100A18000603704794EA0C0F0CEA135518BF95EAC1
:100A28000C0F0CD050EA410618BF52EA4306D1D148
:100A380081EA030101F000414FF0000070BD50EA67
:100A4800410606BF1046194652EA430619D094EAF1
:100A58000C0F02D150EA013613D195EA0C0F05D1DB
:100A680052EA03361CBF104619460AD181EA03012F
:100A780001F0004141F0FE4141F470014FF00000E7
:100A880070BD41F0FE4141F4780170BD70B54FF082
:100A9800FF0C4CF4E06C1CEA11541DBF1CEA135502
:100AA80094EA0C0F95EA0C0F00F0A7F8A4EB0504E4
:100AB80081EA030E52EA03354FEA013100F08880DB
:100AC8004FEA03334FF0805545EA131343EA1263A4
:100AD8004FEA022245EA111545EA10654FEA002659
:100AE8000EF000419D4208BF964244F1FD0404F512
:100AF800407402D25B084FEA3202B61A65EB03056E
:100B08005B084FEA32024FF480104FF4002CB6EB2A
:100B1800020E75EB030E22BFB61A754640EA0C00AA
:100B28005B084FEA3202B6EB020E75EB030E22BFEA
:100B3800B61A754640EA5C005B084FEA3202B6EB2B
:100B4800020E75EB030E22BFB61A754640EA9C00EA
:100B58005B084FEA3202B6EB020E75EB030E22BFBA
:100B6800B61A754640EADC0055EA060E18D04FEA78
:100B7800051545EA16754FEA06164FEAC30343EA18
:100B880052734FEAC2025FEA1C1CC0D111F4801FE5
:100B98000BD141EA00014FF000004FF0004CB6E7DE
:100BA80011F4801F04BF01430020B4F1FD0C88BF7D
:100BB800BCF5E06F3FF6AFAEB5EB030C04BFB6EB88
:100BC800020C5FEA500C50F1000041EB045170BD7B
:100BD8000EF0004E4EEA113114EB5C04C2BFD4EBA8
:100BE8000C0541EA045170BD41F480114FF0000E2C
:100BF800013C90E645EA060E8DE60CEA135594EAA8
:100C08000C0F08BF95EA0C0F3FF43BAF94EA0C0FAA
:100C18000AD150EA01347FF434AF95EA0C0F7FF41F
:100C280025AF104619462CE795EA0C0F06D152EA73
:100C380003353FF4FDAE1046194622E750EA410657
:100C480018BF52EA43067FF4C5AE50EA41047FF468
:100C58000DAF52EA43057FF4EBAE12E74FF0FF3CCD
:100C680006E000BF4FF0010C02E000BF4FF0010C9E
:100C78004DF804CD4FEA410C7FEA6C5C4FEA430C17
:100C880018BF7FEA6C5C1BD001B050EA410C0CBF66
:100C980052EA430C91EA030F02BF90EA020F0020C8
:100CA800704710F1000F91EA030F58BF994208BF2F
:100CB80090422CBFD8176FEAE37040F001007047EC
:100CC8004FEA410C7FEA6C5C02D150EA013C07D143
:100CD8004FEA430C7FEA6C5CD6D152EA033CD3D08E
:100CE8005DF8040B704700BF8446104662468C4688
:100CF8001946634600E000BF01B5FFF7B7FF0028BB
:100D080048BF10F1000F01BD4DF808EDFFF7F4FFE3
:100D18000CBF012000205DF808FB00BF4DF808ED6E
:100D2800FFF7EAFF34BF012000205DF808FB00BF91
:100D38004DF808EDFFF7E0FF94BF012000205DF8B3
:100D480008FB00BF4DF808EDFFF7CEFF94BF012068
:100D580000205DF808FB00BF4DF808EDFFF7C4FF61
:100D680034BF012000205DF808FB00BF4FEA4102B4
:100D780012F5001215D211D56FF47873B3EB6252E5
:100D880012D94FEAC12343F0004343EA505311F00C
:100D9800004F23FA02F018BF404270474FF000009E
:100DA800704750EA013005D111F0004008BF6FF0DC
:100DB800004070474FF00000704700BF4FEA410203
:100DC800B2F1E04324BFB3F5001CDCF1FE5C0DD9A1
:100DD80001F0004C4FEAC0024CEA5070B2F1004FEB
:100DE80040EB830008BF20F00100704711F0804FEE
:100DF80021D113F13872BCBF01F00040704741F4B3
:100E080080114FEA5252C2F11802C2F1200C10FAB6
:100E18000CF320FA02F018BF40F001004FEAC1239A
:100E28004FEAD32303FA0CFC40EA0C0023FA02F33E
:100E38004FEA4303CCE77FEA625307D150EA013314
:100E48001EBF4FF0FE4040F44000704701F00040E4
:100E580040F0FE4040F40000704700BF80F00040C2
:100E680002E000BF81F0004142001FBF5FEA41037A
:100E780092EA030F7FEA226C7FEA236C6AD04FEA7A
:100E88001262D2EB1363C1BFD218414048404140BF
:100E9800B8BF5B42192B88BF704710F0004F40F471
:100EA800000020F07F4018BF404211F0004F41F48D
:100EB800000121F07F4118BF494292EA030F3FD059
:100EC800A2F1010241FA03FC10EB0C00C3F120036C
:100ED80001FA03F100F0004302D5494260EB4000FB
:100EE800B0F5000F13D3B0F1807F06D340084FEA66
:100EF800310102F10102FE2A51D2B1F1004F40EB5B
:100F0800C25008BF20F0010040EA030070474900C2
:100F180040EB0000013A28BFB0F5000FEDD2B0FA5F
:100F280080FCACF1080CB2EB0C0200FA0CF0AABF82
:100F380000EBC25052421843BCBFD0401843704720
:100F480092F0000F81F4000106BF80F40000013226
:100F5800013BB5E74FEA41037FEA226C18BF7FEAFD
:100F6800236C21D092EA030F04D092F0000F08BF3F
:100F78000846704790EA010F1CBF0020704712F026
:100F88007F4F04D1400028BF40F00040704712F165
:100F980000723CBF00F50000704700F0004343F0CA
:100FA800FE4040F4000070477FEA226216BF084600
:100FB8007FEA23630146420206BF5FEA412390EAC3
:100FC800010F40F4800070474FF0000304E000BFB9
:100FD80010F0004348BF40425FEA000C08BF70476A
:100FE80043F0964301464FF000001CE050EA01022E
:100FF80008BF70474FF000030AE000BF50EA010243
:1010080008BF704711F0004302D5404261EB41012F
:101018005FEA010C02BF84460146002043F0B64354
:1010280008BFA3F18053A3F50003BCFA8CF2083A79
:10103800A3EBC25310DB01FA02FC634400FA02FC82
:10104800C2F12002BCF1004F20FA02F243EB020089
:1010580008BF20F00100704702F1200201FA02FCEB
:10106800C2F1200250EA4C0021FA02F243EB0200DE
:1010780008BF20EADC7070477BB972B90029BEBF8F
:1010880000204FF0004106E008BF00281CBF6FF0A9
:1010980000414FF0FF3000F077B8ADF1080C6DE972
:1010A80004CE002909DB002B1ADB00F0A9F8DDF8D3
:1010B80004E0DDE9022304B07047404261EB4101DE
:1010C800002B1BDB00F09CF8DDF804E0DDE90223CF
:1010D80004B0404261EB4101524263EB4303704765
:1010E800524263EB430300F08BF8DDF804E0DDE9DE
:1010F800022304B0404261EB41017047524263EB66
:10110800430300F07DF8DDF804E0DDE9022304B0D4
:10111800524263EB4303704753B94AB9002908BFE9
:1011280000281CBF4FF0FF314FF0FF3000F02CB803
:10113800ADF1080C6DE904CE00F062F8DDF804E0CA
:10114800DDE9022304B07047D0B5FFF71DFB00228C
:101158000B4B06460F46FFF76FFB00F017F80446E7
:10116800FFF7F0FA0022074BFFF766FB02460B4633
:1011780030463946FFF7A8F900F008F82146D0BDF7
:101188000000F03D0000F041704700BF4A0011D256
:1011980012F5001211D20DD56FF47873B3EB6252C9
:1011A8000ED44FEAC12343F0004343EA505323FAD5
:1011B80002F070474FF00000704750EA013002D14A
:1011C8004FF0FF3070474FF00000704710F8012BC8
:1011D80011F8013B012A28BF9A42F7D0D01A70476C
:1011E800034611F8012B03F8012B002AF9D17047A7
:1011F800034613F8012B002AFBD1181A013870474F
:101208002DE9F0478C468E46089E15460446194639
:10121800002B40F0D080724547D9B2FA82F74FB11F
:10122800C7F120030EFA07FCBD40BC4020FA03F3C7
:1012380043EA0C0C4FEA154EA8B2230CBCFBFEF88F
:101248000EFB18CC08FB00F943EA0C43994528D952
:10125800EB1808F1FF3204D2994502D9A8F102022D
:101268002B44A3EB0903A4B2B3FBFEFC0EFB1C3317
:101278000CFB00F044EA0344A04214D92C190CF1E9
:10128800FF3304D2A04202D9ACF102032C44241A41
:1012980043EA02401EB1FC40002334607360BDE89D
:1012A800F0874246DDE76346F1E7002A79D0B2FAD3
:1012B80082F3002B3FD01946C1F1200302FA01F551
:1012C80000FA01F42EFA03F20EFA01FE20FA03F3F3
:1012D800AFB243EA0E034FEA154EB2FBFEFC0EFB1B
:1012E8001C201A0C0CFB07F842EA004290455AD918
:1012F800AA180CF1FF3004D2904502D9ACF10200D3
:101308002A44A2EB08029BB2B2FBFEFC0EFB1C2295
:101318000CFB07F743EA02439F4246D9EB180CF14E
:10132800FF3204D29F4202D9ACF102022B44DB1BEC
:1013380042EA004202E0AEEB020301224FEA154EF8
:10134800AFB2200CB3FBFEFC0EFB1C330CFB07F802
:1013580040EA034398452AD9EB180CF1FF3004D230
:10136800984502D9ACF102002B44A3EB0803A4B2C0
:10137800B3FBFEFC0EFB1C330CFB07F744EA0344EB
:10138800A74216D92C190CF1FF3304D2A74202D96F
:10139800ACF102032C44E41B43EA00400F4611461B
:1013A80078E71F2188E76046ABE76246BFE76046FB
:1013B800DBE76346EFE7734506D916B9002108460F
:1013C8006DE7C6E9000EF9E7B3FA83F787B9734505
:1013D80001D3824207D8841A6EEB030301209C468E
:1013E8001EB900215BE73846FAE7C6E9004CF8E782
:1013F800C7F1200CBB4000FA07F422FA0CF520FADA
:101408000CF1BA401D432EFA0CF30EFA07FE4FEA10
:10141800154941EA0E011FFA85FEB3FBF9F809FBED
:1014280018300B0C08FB0EFA43EA00439A4540D9E2
:10143800EB1808F1FF3004D29A4502D9A8F102004E
:101448002B44A3EB0A0389B2B3FBF9F809FB183361
:1014580008FB0EFE41EA03418E452CD9691808F1B4
:10146800FF3304D28E4502D9A8F10203294443EA86
:101478000040A1EB0E01A0FB02984145CE46434631
:1014880002D306D14C4504D20138B9EB020E68EB01
:101498000503002EA5D0B4EB0E0261EB030101FA9F
:1014A8000CFC22FA07F3F9404CEA0303C6E90031C1
:1014B80097E74046C5E74346D9E70000000000002B
:1014C8000022F0B5114640F6034085B008F0FAFE58
:1014D8000446002856D108F06DF9214641F2030070
:1014E80003AA08F0EFFE044600284BD1039A274DC3
:1014F800D16805F12C03D1F80100D1F8051003C318
:10150800104604F039FD214641F2010003AA08F013
:10151800D9FE0446002835D10398C3685A7885F85F
:1015280023205A88EA841A7985F82420B3F80720FA
:101538002A85B3F805306B8504F01EFD214641F27B
:10154800020003AA08F0BEFE0446D8B9039F05F1BD
:101558003406FA68531C413234461868596808330F
:1015680003C493422646F7D1384604F005FD95F8A2
:101578003030580610D40121054A064872F04EFD55
:101588006FF01204204605B0F0BD00BF80010020B6
:10159800DF510A00105D0900002142F2030003AA8E
:1015A80008F090FE04460028ECD1039AC04BD1689D
:1015B800D1F80100D1F8051003C3104604F0DCFC93
:1015C800214642F2020003AA08F07CFE04460028E5
:1015D800D8D1039EF468B4F801309AB292B1E27897
:1015E80082B1A5F8BC30E378032B06D00322022190
:1015F8000092B048B04A70F0BDFDE278AF4811469D
:1016080078F016F8304604F0B7FC002142F23A00B0
:1016180003AA08F057FE0446002840F020810398EA
:10162800C368B3F80130A5F8D83004F0A5FC95F8E4
:10163800306016F0200619D14FF0FF304FF0FF311F
:1016480008F06EFC0446002800F0768102210C3078
:1016580071F09EF90123214603704670324640F628
:101668006D4008F02FFE044600288BD195F85030C5
:101678001A0713D5002142F21C0003AA08F022FE23
:10168800044600287FF47EAF0398C368D3F801208E
:10169800D3F80530C5E9262304F06EFC95F89030A0
:1016A8009B0626D50DF10A0102A808F0B5FE0446EE
:1016B80000287FF467AF4FF0FF304FF0FF3108F09C
:1016C8002FFC0646002800F0378104210C3071F009
:1016D8005FF9BDF8083022460380BDF80A3031466C
:1016E800438042F2240008F0EDFD044600287FF410
:1016F80049AF95F890305F0610D5002142F22A00D4
:1017080003AA08F0DFFD044600287FF43BAF0398E6
:10171800C3685B7885F8DA3004F02EFC4FF0FF30B0
:101728004FF0FF3108F0FCFB0446002800F004816C
:1017380008210C3071F02CF995F890100246604899
:1017480011F0020F5F4B08BF034695F891008E0613
:1017580048BF43F0400310F0090F18BF43F400637B
:1017680001F0010143EA0110002172F07BFC2146DF
:10177800002242F2010008F0A5FD044600287FF48B
:1017880001AF95F83030B5F8BC10980673D4C9B9D4
:1017980041F2050003AA08F095FD044600287FF4ED
:1017A800F1AEB5F8BC30039C4BB9E368B3F801203F
:1017B800A5F8BC209A884148114677F039FF2046A1
:1017C80004F0DAFB4FF0FF304FF0FF3108F0A8FBD0
:1017D8000446002800F0B08008210C3071F0D8F8D9
:1017E80095F890300246D90747BF2FA1D1E90001EB
:1017F8004FF00051344872F035FC2146002240F683
:10180800014008F05FFD044600287FF4BBAE0146A6
:1018180003AA4FF6014008F055FD0446002834D0CD
:101828002A4A0221234872F0F9FBEB79002B74D184
:1018380072F0B1FE044600287FF4A4AE0CF030FC30
:10184800044600287FF49EAEEB79002B3FF49AAE55
:1018580008211F4872F0EBFB08F066FC92E6411D78
:101868007FF490AE02211B4A124872F0D7FB1F2367
:10187800A5F8D830DBE60029A4D10121164A0D4885
:1018880072F0CCFB6FF004047CE6039804F074FB60
:1018980021464FF6024003AA08F014FD0446F8B1A9
:1018A8000E4ABEE7AFF30080908800020080002057
:1018B80010020020105D090003520A0040020020B7
:1018C8000E1207002E12070010880002C9520A00E3
:1018D8000802002049520A00A6520A00ED520A00E6
:1018E8000398C368B3F80130A5F8753004F044FBD9
:1018F80095F875305A0798D521464FF6034003AA44
:1019080008F0E0FC08B11A4A8BE70398C3685B78D3
:1019180085F8743004F030FB87E72E78002E87D1E5
:1019280095F875309B061FD54FF0FF304FF0FF310B
:1019380008F0F6FA044610B96FF0680422E60621AA
:101948000C3071F025F8D5F8013021460360094BB9
:1019580032469B8883804FF6064008F0B3FC044665
:1019680000283FF465AF0DE66FF085040AE600BF76
:1019780016530A00810100204FF0FF329FED0A7BC9
:101988000D4B00211A6000200C4B002283ED007BD8
:101998009FED077B0A4BC3E900010A490A4B81ED19
:1019A800007B1A6016F0DCB8FFFFFFFFFF1F000086
:1019B8001F00000000000000A867002000030020AE
:1019C800D8340020F8020020A067002000000000A2
:1019D8002DE9F047044640F2712690F8623090F8FD
:1019E800382023F00103C3F3800060F386128CB023
:1019F80004F1460184F8623084F8382014F036FE89
:101A0800B4F84C300022A3FB0663A36D484D236550
:101A180003F5D673B34228BF33464649A4EB050500
:101A2800A1FB051594F83810C5F3471501F07901A5
:101A3800DFF81091C4E90222227032BF6360666049
:101A4800226584F8381005EB4502246149F82230F4
:101A580014F066FD63694FEA450A00F5D677002B56
:101A68004BD00DF12C089121AA4409EB8A034FF0C1
:101A780000094FF0020A0993CDF820800694B4F8C3
:101A88004C302D4A2D480792A3FB000201FB03218D
:101A98002B4BCDF80C9005936368CDF82CA00493DC
:101AA80021A3D3E90023FFF737FB104619464FF46B
:101AB8007A720023FFF730FB0535EDB20321CDE93B
:101AC80001603B462A464846CDF8009014F0AEFB2C
:101AD800414615F0DBFB60B994F8623043EA0A032B
:101AE80084F8623019F02EFBB8B100200CB0BDE8C4
:101AF800F0870C200CB0BDE8F0870DF12C08CDE97B
:101B08000A330320434661680AAA23F04DF90028E6
:101B1800A9D1DDE90A371F44A5E7504623F050FF55
:101B2800E3E700BFAFF3008000CA9A3B0000000063
:101B38000C6B00201F85EB51ED660100002AE7843D
:101B480091D30100006B002070B50D46044600F1EA
:101B58008F06334600223B3105F12B002AF076FC34
:101B680000229FED2D7BD4F89B30D4F89710C4F851
:101B7800BC30D4F8AC30D4F89300C4F8CD3094F825
:101B8800C830D4F88FC043F0010384F8C83094F803
:101B9800A730C4F8B810D4F8A81062F30003C4F84A
:101BA800B400C4F8C9102046294684ED307BC4F837
:101BB800B0C084F89F2084F8A02084F8A12084F87D
:101BC800A22084F8A32084F8A42084F8A52084F80F
:101BD800A62084F8A7301FF027F90646B8B1301DB3
:101BE80020F026FDF37931466B7320461FF032F959
:101BF800204620F031FA40F206636B8194F88E306B
:101C080023F0180343F0180384F88E3070BD00DE0B
:101C1800E5E700BFAFF3008000000000000000000F
:101C280070B504460D461FF0F7F810B90623AB72DD
:101C380070BD04F18F063346002205F13B0105F122
:101C48002B002AF003FC00229FED2B7BD4F89B305D
:101C5800D4F89710C4F8BC30D4F8AC30D4F893005A
:101C6800C4F8CD3094F8C830D4F88FC062F30003BC
:101C780084F8C83094F8A730C4F8B810D4F8A8107D
:101C880043F00103C4F8B400C4F8C910204629463B
:101C980084ED307BC4F8B0C084F89F2084F8A0207D
:101CA80084F8A12084F8A22084F8A32084F8A42032
:101CB80084F8A52084F8A62084F8A7301FF0B4F88B
:101CC8000646A8B1301D20F0A9FCF37931466B73A4
:101CD80020461FF0BFF8204621F092FE4FF4C16362
:101CE8006B8194F88E3043F0080384F88E3070BD11
:101CF80000DEE7E7AFF3008000000000000000000E
:101D08002DE9F04F03699146D3F8A460436891F830
:101D18002000D3F800B000F07F0440B20028B8BF1C
:101D2800A2464FF0010396F8C623A9BF04F158074D
:101D380004F1480704F1100A0BEB4717B8BF0BEB87
:101D4800471712F0100288463D6803FA0AF185B079
:101D580006F1F40334D0A4000028344417DBD4F887
:101D68003C2222F00042B9F1000F0DD042F40012DB
:101D7800C4F83C22184675F0E4FA0021404605B044
:101D8800BDE8F04F74F010BF42F00062F0E7D4F8FD
:101D98007C2122F00042B9F1000F0ED142F000621E
:101DA8000120C4F87C21C2F3835200FA02F2B6F88B
:101DB8009E030243A6F89E23DCE742F00262EFE7A7
:101DC8009FED377B18468DED007B0391029378F0E9
:101DD80033F8DDE90231D8B1B9F1000F02D045F48A
:101DE80000153D6001224FEA5A130AF01F0A02FA51
:101DF8000AF2D24306EB830303F58073D3E8EF0FAF
:101E08001040C3E8E10F0029F8D105B0BDE8F08F14
:101E180098F92020002A32DBEFF31180202282F388
:101E28001288BFF36F8F0122A240B6F8984392B28E
:101E38001443A6F89843B9F1000F04D0B6F89A43B2
:101E48002243A6F89A23DBF8042842F40072CBF860
:101E5800042880F31188BFF36F8F40F635440025BE
:101E680000221846CDE9004577F0E6FF002884D126
:101E780098F820200C490D4875F0FFF97DE7B9F175
:101E8800000F09D145F00065AA0303D5002DB8BF9E
:101E980045F080453D60E0E745F00265F4E700BFA6
:101EA800000000000000000030720A00305E0900E7
:101EB8002DE9F04F984685B000F15803C0E9163374
:101EC800129B0026838104239FED257B073222F095
:101ED800070A0374119B01EB0A090F4680ED087B82
:101EE8004946C0E9066686608373C6730446DDF812
:101EF80038B003F083F8109BC51D25F00705C4F81A
:101F08008850C4E9207A02930F9BA9EB0505CDE917
:101F180000B32A4643463946204603F069FB0F9B27
:101F2800C4E91B8B6367109B6665A367EFF3118297
:101F3800202383F31288BFF36F8F0B4B596A5C62BF
:101F4800E16782F31188BFF36F8F9B680BB1D3F8F9
:101F58008C302846C4F88C3005B0BDE8F08F00BF3F
:101F68000000000000000000A08000200000000029
:101F780030B5144617A3D3E9002385B0FFF77CF8E2
:101F8800054601A928464CF091FB9DF807309DF8BD
:101F980006201B0443EA42539DF808200C4943EAF3
:101FA800C2239DF8092025F0010543EA42139DF854
:101FB8000A20A5FB010143EA5203BDF80420A2F25E
:101FC800BC7243EA4263236005B030BDAFF30080C2
:101FD80000CA9A3B00CA9A3B0000000000000000BB
:101FE8002DE9F0412DED028B90F8A5300446B0EEB6
:101FF800408A86B01BB9F7EE007A37EEC08AD4F86B
:1020080084202F4B9A4213D118EE100AFEF7BCFB1E
:1020180029A3D3E90023FEF79FFE011E18BF012163
:1020280004F1840037F0BCFE84ED268A012005E027
:10203800B4F89C30B3F5807F05D1002006B0BDEC24
:10204800028BBDE8F08104F15008404651F082FA55
:102058000028F2D0DFED1B7A68EE277AFCEEE77AEB
:10206800CDED037A94F8806094F89C209DF80C30AC
:10207800276E206D6EB18DF8153002238DF814206F
:1020880000210122009305ABB847404683F006FEC5
:10209800CAE7012531468DF813208DF814302A46F9
:1020A8000DF113030095B847009532462946276E6F
:1020B800206D05ABE8E700BFAE47E17A14AEEF3F0D
:1020C800C4E3090000007F432DE9F04F044685B0C2
:1020D80008466160062190461D469DF838709DF8B7
:1020E8003CB03AF093FBA060067C16F0010602D0E3
:1020F8007D483BF03DFD9DF8403005FB08F084F835
:102108002A309DF844307D3084F828307E2390FBB7
:10211800F3F0C0010430C4E90485277360627EF0DF
:1021280033F90DF1080A0622C4E907066F4920466B
:10213800A66190F059FF022251462046ADF808806A
:1021480090F052FF022251462046ADF8085090F018
:102158004BFFF623032269462046ADF800308DF880
:10216800026090F041FF7B1EDBB2082B05D840F2DD
:102178005515DD4015F0010501D15D48B9E7052F7A
:1021880009D0072F06D0032F73D1012384F82930F3
:10219800002502E02E4684F82960002646F34F10F9
:1021A800C0EB0020FEF7DEFA0022524BFEF78EF954
:1021B8000022514BFEF76AFCFEF7D8FD5FFA80F863
:1021C800C6F38200C0EB0020FEF7CCFA00224B4B8E
:1021D800FEF77CF900224A4BFEF758FCFEF7C6FDD5
:1021E800C7B206F00300C0EB0020FEF7BBFA0022DE
:1021F800404BFEF76BF900223F4BFEF747FCFEF71A
:10220800B5FDC0B2002D5ED08DF808008DF80980AC
:102218008DF80A70032251462046013690F0E4FEFC
:10222800802EBBD1BBF1000F1AD0364D01A92A88E8
:10223800AB782046ADF8042003228B7090F0D4FED2
:102248000B222046304990F0CFFED5F80300EB79F9
:1022580002900522514620468AF8043090F0C4FEC8
:10226800204690F0AFFEA06990F0D0FE05B0BDE822
:10227800F08F092F84F829608AD10FF25C09D9E917
:102288000089354616A7D7E900672846FEF76AFA97
:1022980042464B46FEF71AF932463B46FEF7F6FB36
:1022A800FEF764FDC0B28DF808008DF809008DF8BE
:1022B8000A00032251462046FF3590F095FEB5F5F9
:1022C800FF4FE2D1AEE78DF808808DF809708DF8E0
:1022D8000A009FE7AFF300800000000000C04F40F5
:1022E8000000000000C05F40E9D60A00ECB90A000F
:1022F800F9CD0A000000F83F0000084000000C403B
:1023080000001C40F55F0900E0B90A000000000069
:1023180010EE103A33F0004210B52DED028B06D1C5
:102328000120BDEC028BBDE810406DF0B1BD002B63
:1023380005DABDEC028BBDE810406DF0B7BDB3F116
:10234800FF4F06DB30EE008AB0EE480ABDEC028B88
:1023580010BDB3F5000F6049BBBFDFED607A6FF0C9
:102368001802002260EE277AB8BF17EE903AF7EE0F
:10237800007ADC15C3F316037F3C1944144401F4B6
:10238800000282F07E5204EBD15403F10F011A438C
:1023980007EE102A524A0A4037EE678AB2BBB5EEFA
:1023A800408AF1EE10FA0FD1002C00F08C8007EE75
:1023B800904A9FED4C0A9FED4C7AF8EEE77A27EEAB
:1023C800808A07EE878ABFE741A1D1E90001FEF7BD
:1023D800F5FCB6EE007A07EE900A07EEC87A68EECA
:1023E800087A27EE277A14B938EE478AACE707EE61
:1023F800904ADFED3C6AF8EEE77A07EEE67A37EEC8
:10240800488A9FED397A17EE878A9DE7F0EE007AC1
:102418009FED365ADFED364A364A78EE277A1A4467
:10242800C3F5571388EE276A07EE904A03F522731F
:102438001343F8EEE76ADFED307A002B66EE065AB2
:1024480025EEA57A07EE275ADFED2C7A45EE077AB6
:102458009FED2B5A07EE875ADFED2A7A47EE274A77
:10246800DFED297A44EE877A67EE877A45EE257A9A
:102478001ADDB6EE007A28EE077A27EE087A77EEAC
:10248800877A67EE867A14B937EE677AACE79FEDFC
:10249800156A46EE867A37EE677A37EE488ADFEDB8
:1024A800127A16EEA78A4FE778EE677A67EE867A91
:1024B80014B938EE678A47E79FED0A7A46EEC77A7D
:1024C80037EEC88AEBE79FED118A3DE7AFF300804E
:1024D800555555555555D53F20FB4A000000004C31
:1024E800F0FF7F00D1F717378071313F25333A3E2F
:1024F800298E633E305CCFFF9788173E2549923E70
:10250800ABAA2A3F4FD01C3ECDCCCC3E00000000E9
:10251800F8B510EE904A10EE103A34F000472DED61
:10252800048BB0EE609A0DD183F480035B0013F541
:10253800000F40F2AA8230EE098AB0EE480ABDECDC
:10254800048BF8BD23F000411846B1F1FF4F02D8C3
:10255800B7F1FF4F08D9B3F17E5FECD184F4800462
:10256800640014F5000FE4E7002B25DAB7F1974F64
:1025780080F09482B7F17E5F39D3FA15C2F19602E2
:1025880047FA02F505FA02F2BA4229D105F0010527
:10259800C5F10205B7F17E5F2AD1002C80F27B825B
:1025A800B5EE400AF1EE10FA1CD1D80FBDEC048B41
:1025B800BDE8F8406DF06CBCB7F1FF4F10D1B1F138
:1025C8007E5F00F0628205D9002CDFEDD17A29FE0A
:1025D800278AB2E7002C80F25B82B1EE498AACE729
:1025E8000025D7E7B7EE007A87EE008AA5E7002531
:1025F800B4F1804F0A4640F05782B1F1BF4F0CD278
:10260800B1F1D05F02D920EE008A96E7B0EEC08A19
:1026180059BB012D00FE088A8FE723F04046B0EE33
:10262800C08AB6F17E5F17D1002CBCBFB7EE007A26
:1026380087EE088A002B80DAA1F17E51294305D163
:10264800BDEC048BBDE8F8406DF030BC012D7FF483
:1026580074AFB1EE488A70E739B9002CD9DA002B8B
:10266800A4D06B1E58425841A0E7DE0F013E55EA40
:102678000600E5D0B7F19A4F71D9A64B994208D810
:10268800002C0BDA0020BDEC048BBDE8F8406DF09F
:10269800F1BBA14B994208D9002CF3DC0020BDEC1A
:1026A800048BBDE8F8406DF0D7BBB7EE007ADFEDDC
:1026B8009B7ADFED9B9A38EE478A93A1D1E9000116
:1026C80068EE278AFEF77AFBB5EE007A07EE900AE5
:1026D800DFED946A68EE299A48EE477AB6EE007AFA
:1026E80007EEC87A68EE087A27EE277AF0EE687A5D
:1026F80047EE667A39EEA77A17EE103A6FF30B03B6
:1027080007EE103A77EE699A77EEE97A013DF7EE2F
:10271800006ABFEE008A6FF30B04354367EE890A3F
:1027280008FE268A06EE904A39EE666A67EE267A31
:1027380046EE070A30EEA77A17EE101A002921F0A4
:10274800004340F31381B3F1864F40F2CC80B5EEDD
:10275800C08AF1EE10FA4CBF0120002093E713F075
:10276800FF4F05BF9FED707A6FF01701002168EEEB
:10277800077A08BF17EE902AD315C2F316027F3BDB
:1027880042F07E500B4469498A4206DD68498A4214
:1027980040F3A7800133A0F500000021654A06EE4A
:1027A800100AF7EE006A02EB8102D2ED005A75EECC
:1027B800867A36EE657AC6EEA74A27EE245A15EED3
:1027C800102A6FF30B0206EE902A5B4A02EA6002B7
:1027D80042F0005202F5800202EB415207EE902AC5
:1027E80006EEE77A77EEE57ADFED545A36EE676A59
:1027F80065EE057A06EE667A9FED516A47EE865ACF
:102808009FED506A27EE247A66EEA64A05EEA76A7F
:10281800DFED4D5A46EE275A9FED4C6A05EEA76A42
:10282800DFED4B5A46EE275A36EE856A67EEA77AF1
:1028380026EE076A05EEA76AF0EE085A74EEA57A46
:1028480077EE867A17EE902A6FF30B0207EE902A3E
:1028580077EEE55A27EE277A66EEA76A75EEE45A10
:1028680036EE656A06EE057A9FED3A6A76EE877A65
:1028780017EE902A6FF30B0207EE902A364A77EE8E
:10288800E66A02EB810227EE866A37EE667ADFEDAA
:10289800336A67EEA67ADFED326A47EE267A92ED62
:1028A800007A77EE877A07EE103A2E4BF8EEC76A71
:1028B80003EB810336EE277AD3ED005A37EE257AFB
:1028C80037EE267A17EE103A6FF30B0307EE103A3D
:1028D80077EE666A76EEE56A76EEC66A77EEE67AAF
:1028E80014E701215AE755D1DFED1F6A37EE677A01
:1028F80070EEA66AF4EEC76AF1EE10FA3FF727AF5A
:1029080086234BE0AFF30080E13D55555555D53F43
:1029180000000000F3FF7F3F0700803F70A5EC3602
:1029280000AAB83F3BAAB83F0000804B71C41C0006
:10293800D6B35D00382B0A0000F0FFDF55326C3E3D
:1029480042F1533E05A38B3EABAAAA3EB76DDB3ED0
:102958009A99193F0040763F282B0A00C623F6B8FB
:102968004F38763F302B0A003CAA3833534A9342FB
:1029780007D9B5EEC08AF1EE10FA4CBF012000204D
:102988008DE607D137EE677AB4EEE07AF1EE10FA09
:10299800B6DBEEE7B3F17C5F72D9DB157E3B4FF413
:1029A8000000474A002940FA03F00844C0F3C7531F
:1029B800A3F17F0342FA03F2C3F1170302EA00020C
:1029C800C0F3160040F4000007EE102A40FA03F0A6
:1029D80077EEC77AB8BF404237EEA07ADFED396AA2
:1029E800DFED395AB7EE000A9FED386A17EE103A54
:1029F8006FF30B0307EE103A77EE677A67EE266AF5
:102A080070EEE70ADFED327A27EE277ADFED317ACA
:102A180000EEA77A76EE877A77EEE66A37EE667A80
:102A280067EEA76A07EE877A16EEA56ADFED2A5ADF
:102A380046EE265A9FED296A15EEA66ADFED285A5A
:102A480046EE265AB0EE676A05EEE66AF0EE006AD0
:102A580067EE865A36EE666AC5EE866A36EEC77A3D
:102A680077EE677A30EE670A10EE103A03EBC05340
:102A7800B3F5000F06DA6DF073F820EE088A5CE50E
:102A88000020A9E700EE103AF7E7B7EE008A54E510
:102A98009FED148A51E5B0EE408A4EE5B7F1FF4F3D
:102AA8003FF48DAD0A460225B4F17C5F7FF4B5ADE5
:102AB800002BFFF6B2ADB1EEC08A3EE5000016432A
:102AC800000080FF0072313F4CBB31330EEADD3528
:102AD8008CBEBF351872313F55B38A38610B363B0F
:102AE800ABAA2A3E0000000010EE103AB3F1FF4FE7
:102AF80010B52DED048BB0EE408A06DB30EE008A6F
:102B0800B0EE480ABDEC048B10BD774A934276DCE0
:102B180023F00042B2F17E5F13D3FFEE007AB4EEE9
:102B2800670AF1EE10FA06D10120BDEC048BBDE86E
:102B380010406DF0ADB9BDEC048BBDE810406DF0F0
:102B4800B5B9B2F1645F0FD2B2F14A5F24BF20EE8B
:102B5800007AF6EE007ABDEC048B28BF07EE670A10
:102B6800BDE810406CF0B6BF604A134493424ED89B
:102B7800F7EE007A38EE277A17EE103ADC157F3C2C
:102B8800002CD5BF77EE677A37EE488A78EE677AF9
:102B980077EEC87A87EE879AC3F31603544A9342AE
:102BA800CCBF43F07C5243F07E52F7EE007AC8BFA8
:102BB800C3F5000307EE102AC4BF01349B1037EE9B
:102BC800678AF6EE008A68EE288A68EE888A002B03
:102BD80044D1B5EE408AF1EE10FA1DD1002C7AD01E
:102BE80007EE904AB0EE498A9FED427AF8EEE77A0E
:102BF80007EE878A9FED407A07EE878A80E7B3F170
:102C0800B44FB5DBDC159FED3D9A7F3CC4E701234B
:102C180000249FED3A9AD4E731A1D1E90001FEF7EB
:102C2800CDF8B7EE007A07EE900A07EEC87A27EEDD
:102C3800287A14B938EE478A62E707EE904ADFED42
:102C48002D6AF8EEE77A07EEA69A37EE497A37EE5C
:102C5800488A9FED297A17EE878A51E7F0EE007AC5
:102C68009FED276A9FED277A78EE277AC8EE276AC4
:102C780066EEA67A07EE867A9FED236A07EE276A44
:102C88009FED227A06EE277A9FED216A07EE276AE2
:102C98009FED207A06EE277A9FED1F6A07EE276AD6
:102CA800B0EE687A06EE277A27EE267A24B978EE0F
:102CB800C78A38EE688A23E707EE904ADFED0D6A87
:102CC800F8EEE77A07EEA69A39EE079A78EEC98AFF
:102CD80038EEC88ABDE79FED098A11E7AFF3008097
:102CE800555555555555E53FD613D43EE0096A412B
:102CF800F6043500D1F717378071313F0000000026
:102D08009788173E4FD01C3E25333A3E298E633EA6
:102D18002549923ECDCCCC3EABAA2A3F2DE9F047BF
:102D28000546884600AF6DF002FDA9680646B1F574
:102D3800004F36BFA8F10403002303F00703B1F5E1
:102D4800004F34BF0420082002F0070407341C4455
:102D58000444E40804EBD2048C4228BF0C46012248
:102D6800314628466DF09DFC10EA020A16D1E94664
:102D780088B06A46504BCDE90538032342F8103F26
:102D88004FF4C25153464D4801F006FACD468AF336
:102D98001188BFF36F8F0423184602DF3146284697
:102DA8006DF095FC06EB00094946002228466DF0B7
:102DB80078FCA9EB00094E4518D0E94688B0694669
:102DC8003F4BCDE90538032341F8103F3B481346F4
:102DD8000A464FF4C25101F0DFF90023CD4683F3D0
:102DE8001188BFF36F8F0423184602DF3146284647
:102DF8006DF06DFC8442804623D028D2344431469D
:102E0800224628466DF025FD0122314628466DF000
:102E180064FC21466DF05BFC2618012231462846E9
:102E28006DF03FFCC30708D4314628466DF0C1FC5D
:102E38003246214628466DF033FD214628466DF07E
:102E48004DFD4FF001094846BD46BDE8F08706EB49
:102E5800000A0122514628466DF023FC10EA0209B7
:102E680027D1514628466DF032FC40448442EAD8C6
:102E7800514628466DF09DFC514628466DF027FCCA
:102E8800A4EB0808804509D2344451462846224616
:102E98006DF0DFFC214628466DF020FD5246314694
:102EA80028466DF0FDFC0122314628466DF015FCE0
:102EB800C7E74FF00009C6E78E350A00F05D090044
:102EC800B2350A002DE9F843884600AF00297DD0C5
:102ED8000568012228466DF02AFC0146044628466A
:102EE8006DF0DFFB10EA020616D1E94688B06A46A3
:102EF800384BCDE90538032342F8103F4FF4C2514F
:102F08003346354801F048F9CD4686F31188BFF3BA
:102F18006F8F0423184602DF214628466DF0D7FB41
:102F280026183146002228466DF0BBFB361AB442FB
:102F380018D06E4688B06946284BCDE9053803237A
:102F480041F8103F244813460A464FF4C25101F095
:102F580023F90023B54683F31188BFF36F8F042349
:102F6800184602DF0022214628466DF0B6FB2146AE
:102F78006DF0ADFB26180122314628466DF091FB15
:102F8800C20708D4314628466DF013FC3246214664
:102F980028466DF085FC0022214628466DF081FB0D
:102FA800261A0122314628466DF07BFBC30709D457
:102FB800314628466DF0FDFB2246314628466DF025
:102FC8006FFC3446214628466DF088FCBD46BDE8B6
:102FD800F88300BFDB350A00F05D0900B2350A004E
:102FE80008B502486EF017F8002008BD08360A0038
:102FF8000E4A0346904202D30D4A904211D30D4A1D
:1030080022B1934202D30C4A93420AD30B4A52B1DB
:103018000B48834234BF01200020934238BF002070
:103028007047012070471046704700BF9857090045
:10303800ACF10A00000000000000000000000000E1
:10304800000000002DE9F04F9BB000AF04468B460E
:10305800D7F890A0FA637B6349B9037846788078FB
:1030680000EB830020445E4522D8A0EB040B0AF055
:10307800010394F80280FB62E378B8F1000F0CBFFB
:103088004FF000090AF001093B6313B11AF0020F6F
:1030980017D1B9F1000F14D1FB6B1BB1594620466B
:1030A8007A6B98475D4628466C37BD46BDE8F08F79
:1030B800451C2846FEF79CF8013028440BF1010B0B
:1030C800D1E7CAF3C003FB612378BB629B00BB61F5
:1030D80063683B62BB6A04EB8301FB6B002B7DD109
:1030E8005D468844B9F1000F1DD08B469946A94E1C
:1030F8001BF8013B54F82300002808BF3046FEF7B0
:1031080077F8D7F8943001304BB1D7F898304B4561
:1031180082BFD7F8943023F8190009F10109C34593
:103128000544E5D1D8461AF0050F0CBF4FF0020B45
:103138004FF0010B00260AF00203FB633B6B9E4233
:10314800B1D298F8013008F1020854F823A050468B
:10315800FFF74EFFFA69034602B3B86318F8021C7A
:10316800386A6DF037FFBB6BC0B1EA468AB06A4671
:10317800894B05933B6ACDE906314FF40073ADF8EE
:103188002030864B42F8103F00234FF412518448F8
:1031980001F002F8D546023D0136CFE723B1FB6ABC
:1031A8002BB9A5EB0B05F7E7FB6B002BF4D079489F
:1031B800BAF1000F18BF5046FEF71AF8D7F8943046
:1031C80053B1D7F8983099453FBFD7F89420431C9E
:1031D80022F8193009F101090544DDE7B9F1000FBA
:1031E8006DD04346102B28BF10230026BB6397F8E9
:1031F800389007F14800BA6B796291F0F1FF796A6B
:1032080000227A620AF0020201EB08033A610AF02E
:1032180004027B61FA6002337A6A396B8A4267D3A7
:103228006378F96A1AF0020F7B624B4418BF0022D8
:10323800DBB208BF7208002940F0A9801AF0040F19
:1032480014BF314600216370A170E27020467A6B8A
:10325800B969FB6B9847051EFFF625AFBB6A314677
:1032680023707B6A7A6B63703B6B84F80280E3702F
:1032780007F15800FB6B9847061EC0F2C5803A6BF1
:10328800BB69386B03EB4203ABEB0301D7E90D23B2
:10329800C91A7B6903EB4000FB6B98470028C0F212
:1032A800B5804FF000082E44351807F1480AC84584
:1032B80078D300217A6B0846FB6B9847F3E6B8F1A0
:1032C800000F0CD01AF0040F0ED04346102B28BF65
:1032D8001023BB6397F8386007F158008BE7464620
:1032E800C146C7F838808BE74E46C7F8388087E76D
:1032F80013F8015C13F8021C54F82500BB60FFF7B3
:1033080077FE0246F869BB6838B1386AC7E9013206
:103318006DF060FED7E90132F0B912B3FA6A72B102
:10332800B9F10F0F18D809F1280107F1400009F188
:103338000102014401F8205C5FFA82F90CE0FA68A6
:1033480052B10F2E08D806F1280107F14000721C6F
:103358000E1806F8105CD6B27A6A023301327A6225
:103368005AE73A69002ADBD10F2EF5D806F1280072
:1033780007F1400C6044721C00F8101C07F168014A
:10338800023651FA82F2F6B202F8105CE4E7002144
:1033980059E700BF36360A003D360A00040000012E
:1033A800685D090018F80A3054F823B087F84730E8
:1033B800D7F8943033B3D7F89830984522D2D7F855
:1033C800943033F8186001217A6BFB6B07F14700E2
:1033D800984700281ADB0E4B0544BBF1000F08BFC5
:1033E8009B4626B95846FDF703FF461CB6B2314640
:1033F80058467A6BFB6B9847002807DB054408F1B1
:10340800010854E70026DEE735464CE605464AE65D
:1034180036360A00014B1860704700BF9803002039
:10342800044608B5EFF31183202383F31288BFF312
:103438006F8F2CF067FD204602F074FE02486DF095
:10344800EAFD6FF0B9F9FCE7F1360A002DE9F0471B
:10345800058B0446280717460CD501290CBF45F0F3
:10346800100545F02005258387F31188BFF36F8F7A
:10347800BDE8F087022905F0070540F09480204652
:103488006EF0DBF8052864D801A353F820F000BFDC
:1034980071340000AF3500005B3500001D350000B9
:1034A800373500004935000001F007035A1F012A8B
:1034B8001FD8002221F00701062BD4F8008089B21A
:1034C800C4E9002209D1434603E0628B01326283DA
:1034D8001B68002BF9D141F00201204621836EF0D0
:1034E800ACF84FF0000900286DD041F0200121838D
:1034F80069E0042B0AD121F0070189B22046218313
:103508006EF09BF810B141F0200121834FF00008C4
:10351800C14658E02369D3F80090238B23F00703B2
:1035280043F006034FF00008238346464BE0236927
:10353800D3F80490238B23F0070343F00403F1E747
:103548002369D3F80890238B23F0070343F005037E
:10355800E8E74FF00008C146E7E7012243F0080317
:10356800238387F31188BFF36F8F002A3BD1B8F10B
:10357800000F4AD1B9F1000F02D020462C49C847A4
:10358800EFF31187202383F31288BFF36F8F238B08
:1035980023F008039BB22383D9063FD523F01002FA
:1035A800228303F007056669218B002EBFF67CAFE6
:1035B80000239946D4F8008021F00701C4E90033BC
:1035C80041F001012183238B03F0070AAA4502D0A9
:1035D800A268002AC1D1B8F1000F02D1B9F1000FD9
:1035E800DAD00022BAE7A1680029C0D00D68002906
:1035F800BDD03346524620464F68B8471DB12B68A8
:1036080029461D46F3E72B46FAE74146334652461C
:103618002046D8F800806EF03CF8A8E79A067FF5B7
:1036280023AF23F02002228303F0070527E700BF1A
:10363800C716070037B504460821C06A6EF0DCFAE1
:1036480000234FF6FF72104DADF804306368ADF8F3
:1036580000208DF80620E26819182B401344181A28
:1036680060606846ADF802106EF01AFA69462046A6
:103678006EF0E1FA2046211D6EF0ECF963682B40EC
:10368800A36003B030BD00BF0000FFFF2DE9F74382
:103698000F4681460821C06A6EF0AEFA80463C6843
:1036A800124D241A3C6004EA0506B4421CD3A0B2A9
:1036B80010B903B0BDE8F08308236A46214648469E
:1036C8006EF08FF90028F4D16946A0B26EF080FA46
:1036D80038B1BDF80230BDF804202E4013441E4412
:1036E8003C60A4EB0804E0E70020E2E70000FFFFED
:1036F8002DE9F04704468AB000F11407384675F002
:10370800A3FEA06A83681B699847E06248B9A84984
:10371800A8486EF059FA6FF0150528460AB0BDE8BA
:10372800F087A06A83681B6998470368013B1F2BD1
:1037380001D9A149ECE7E368B3F5803F08D94FF414
:103748008032012100929B489C4A6EF013FDE2E70B
:10375800A06A216807AA74F0F7F908B19849D7E771
:10376800E5682DB1089BB5FBF3F203FB12550DB1CB
:103778009449CDE7238A012B01D89349C8E7E36A26
:10378800029593F805804FF0FF334FF0FF3238462B
:103798002EF00AFD0821E06A6EF02EFAA9460646C8
:1037A800238A1FFA85FA534544D8238A4B4500F0EB
:1037B8000F8153450BD10299082342462046891BA5
:1037C8006EF01DF918B9204602A96EF043F920469B
:1037D80002A9FFF75BFF0546002840F0FB8002992D
:1037E8004FEA11494FEA09496160C4F80890A36893
:1037F8008B420DD80823204603AA6EF0F2F8B8B918
:1038080003AB13F8012B904532D101300828F8D1C9
:10381800636820466FF30F0302A902936EF01AF94A
:1038280042462046E36802996EF0E9F800283CDA3F
:103838000546CFE0E1682B04891B13FA81F1424663
:103848000823204602916EF0DAF878B1204602A9E2
:103858006EF000F909F10109082342462046029951
:103868001FFA89F96EF0CBF800289ED0013597E74A
:10387800A08803A96EF0ACF9626810B9911B616069
:10388800B5E7BDF810A0BDF80E10E06AC4F80890BE
:1038980051446EF0B1F948448242A060EED1BAF1C9
:1038A800000FEBD06FF01C0594E05DD04FF6FF7968
:1038B800636806EB0308E3681FFA88F29B1B9A42C9
:1038C800CDF808801CD34FF000086168B8F1000FEC
:1038D80030D06FF30F012046029102A96EF0BAF8BA
:1038E800204602996EF0C3F80028A1D1E368A288A7
:1038F800A3EB46039A426DD120466EF0B9F997E7DB
:1039080008234146204605AA6EF06BF800288FD19F
:1039180005A91FFA88F06EF05BF930B1BDF81430D4
:103928004B4502D1BDF818300BB1B044C3E74FF096
:103938000108CAE720466EF09AF800287FF478AFAD
:103948006368224AE16813400B44A3EB46036360B3
:10395800134041462046A3606EF00EFAC4E7E26ABF
:10396800A36812681344A360D4E901318B4208D9D3
:10397800424620465B1A6EF042F80028FFF658AF20
:10398800EDD16168E36801EB46029A42AED10F4B74
:10399800A06801EA03029042A8D020466EF067F8BA
:1039A80000287FF445AF6268084B1A40A2609DE783
:1039B80039370A00985D09005B370A0078370A0032
:1039C800A1370A00B9370A00CD370A000000FFFF07
:1039D8006FF02C0538462EF059FC002D7FF49DAE73
:1039E8000123A37499E600BF2DE9F04F1E46837C9E
:1039F80004468946904695B04BB96A496A486EF0C4
:103A0800E3F86FF00C05284615B0BDE8F08FC26AE0
:103A1800082110466EF0F0F8B1B2019010466EF031
:103A2800EBF8E368019A0746A3EB82038342C0F0F0
:103A3800B6801EB1B8F1000F00F0B180D4F804A030
:103A4800CDF810A0204605AA04A96EF04BF905464A
:103A58000028D8D1BDF814304B4507D0DDF810A0A8
:103A680063685345EED1002E39D1CCE705A91FFA7A
:103A78008AF06EF0ADF80028F0D0BDF8183066B3C3
:103A8800B3422CD1B3464FEA1A43BDF816A01B0423
:103A98009A44E36ACDF800801B685B4203F0200378
:103AA8000293029B51465B4528BF5B4620460CAA01
:103AB80003936DF096FF00284DD1039B00981A469A
:103AC8000CA991F0BBFB50B9039B009ABBEB030B0D
:103AD8001A449A440092E4D195E7002B93D0002F22
:103AE8003CD1BA4604F1140B4FF0FF324FF0FF33CC
:103AF80058462EF059FB238A9D424DD0D4E9013215
:103B08000AEB02018B422ED39BB263B3FF23002141
:103B1800ADF81E200CA818228DF82230ADF81C90A4
:103B2800ADF8206091F082FB20460CA9CDE90E8605
:103B38006EF06CF8074648B907A86DF0B1FF20464B
:103B480007A96EF078F8074600B9374658462EF0B0
:103B58009DFB3D4657E7C2DC054654E7019B1F44E1
:103B68001FFA87FABEE72046FFF764FD3DB9ADF8B6
:103B78002490CDF82880ADF82C608DF82E50204682
:103B880009A96EF0F9F807460028DFD19DF82E3014
:103B98000135002BAFD0D8E76FF01B07D6E76FF0E1
:103BA800150530E725370A00985D09002DE9FF471C
:103BB8001E46837C04460F469046BDF8309043B9B4
:103BC800274828496EF000F86FF00C0004B0BDE8F3
:103BD800F0870821C06A6EF00FF8E368A3EB400392
:103BE800B3423AD34FF0000A65680195204602AA0D
:103BF80001A96EF077F80028E8D1BDF80830BB427B
:103C080006D102A9A8B26DF0E3FF50441FFA80FA6A
:103C1800019B62689A4219D0CA4515D9BDF80C3083
:103C2800C3B1CA4516D3BDF80A10B3426FF30F05E6
:103C380028BF33464246204629446DF0D2FE00286C
:103C4800C4D1BDF80C00C1E71D46CFE7BDF8083068
:103C5800BB42E3D06FF00100B8E76FF01500B5E79D
:103C6800985D090025370A002DE9F0470446074604
:103C78004FF00109DFF84C8094FAA4F5B5FA85F500
:103C880009FA05F32E0108EB05156FEA030A24EA81
:103C980003042B7B63B158F806301B696BB94644A3
:103CA800736802222846196807EA0A076EF0DFF9E6
:103CB800002CE1D13846BDE8F0872846984700280F
:103CC800F6D1ECE7A85E090010B5002288B00E49CD
:103CD8000E4875F0B9FF002200230024CDE9062321
:103CE8000E234FF44072CDE90334CDE90144084B6B
:103CF8000849009408482EF0D5FE0849064875F092
:103D0800FEFD204608B010BD293D0000682A0020AD
:103D18004940000040AE002080250020F7370A0007
:103D280001482EF039BB00BF6C1E00202DE9F0477A
:103D3800804621480F466EF07EF90646002833D0AB
:103D480000252846BDE8F087237B83B12368DB681C
:103D58000BB120469847636883F8069023681B696F
:103D6800D3B963680222204619686EF080F90136DB
:103D780010345445E8D3B8F1000FE2D0002DDFD05D
:103D88002846FFF771FF0546002FF7D0002140F2C3
:103D9800391075F0B6FEF1E7204698470028E0D0C4
:103DA80009FA06F31D43E2E705464FF00109034C03
:103DB800DFF80CA0DDE700BFE0430020A85E0900A3
:103DC800B85E0900014B53F820007047DC62090017
:103DD80008B5034608462BB1044A136000F04CFCB2
:103DE800002008BD6FF01500FBE700BF9C03002012
:103DF80010B5044C237813B903482EF0CDFA0123EB
:103E0800237010BDE6A700206C1E002010B50446E4
:103E180009486EF010F93CB1084BD3E8EF1F01399F
:103E2800C3E8E21F002AF8D105482FF05DFCBDE881
:103E3800104004482EF0B0BAD8430020DC430020DC
:103E4800682A00206C1E00200022044BD3E8EF0FE4
:103E5800C3E8E12F0029F9D1704700BFD8430020FB
:103E680070B5FFF7F1FF0546074C084EB44200D382
:103E780070BD63685B792BB123685B6813B1294611
:103E8800204698471034F1E7A85E0900B85E09009B
:103E980010B5044C044920466DF0D8F9034B1C605A
:103EA80010BD00BF1C1D0020C8620900D0430020BF
:103EB80000230D4A10B513700C4A0D4913600D4AC2
:103EC8000D481360FFF784FFFFF7E2FF0B4B0C4927
:103ED80018468B4200D310BD1A1A5C6812110132C1
:103EE80022711033F5E700BFE7A70020D843002070
:103EF80040420F00DC4300203B200700A85E090079
:103F0800B85E0900014647F61222002301486DF009
:103F1800BEB900BF1C1D002001486DF054BA00BF97
:103F28001C1D0020024B014618686DF0A7BA00BF9F
:103F3800D043002001486DF0DCBA00BF1C1D0020F2
:103F4800F8B5284B1B78002B4AD0FFF7E5FF04464D
:103F5800002842D1244B254D1B68002B19DD75F034
:103F68002BFE4FF47A76A0FB060747F612220023B1
:103F780006FB0171FDF7D0F8D5E90032C01A40F20E
:103F8800E93361EB0201984271F1000101D3FFF7B7
:103F980067FFD5E9003213F57A7342F10002C5E9EB
:103FA8000032ECB1BDE8F840FFF7C4BF6B685B793D
:103FB80023B12B68214628461B6898471035B5421F
:103FC800F4D32046FFF7AEFF094BD3E8EF1F0139C2
:103FD800C3E8E21F002ABDD0F7E7064D064EEEE71C
:103FE8000020F8BDE6A70020D8430020602A002062
:103FF800DC430020A85E0900B85E090070B50D4DCD
:10400800297861B90120FFF791FE0B4C0B4EB442A1
:1040180006D3FFF795FF0028FBD101232B7070BD55
:1040280063685B791BB1236820469B689847103406
:10403800EDE700BFE7A70020A85E0900B85E090009
:1040480000212DE9F8430846FFF770FE044648B3FF
:1040580040F21B684FF0000901F0D8FB1A4B1B4ACD
:104068001B58136033B11A4B1B68092B02DD194822
:104078002EF092F90025184F44B12046FFF7F4FDC1
:10408800044618B94FF0FF384FF0FF39FFF758FFD3
:10409800064628B9B5B90F4842464B462EF0B8F93E
:1040A8003546E9E74FF0FF384FF0FF39D4E72B6882
:1040B8009B691BB100222846114698471035BD421E
:1040C800F5D3E8E7054DFAE708000000D4430020DF
:1040D800DC4300206C1E0020B85E0900A85E0900C1
:1040E80013B518486DF0A7FF174B1B7873B1EFF3A2
:1040F8001184202383F31288BFF36F8FFFF720FF0B
:1041080084F31188BFF36F8F02B010BD0F4B1B688B
:10411800002BF9D050B9002200230D48CDE9002327
:1041280047F6122200232FF0B9FAEDE70928EBD160
:1041380007482FF0D9FA074802B0BDE810402EF022
:104148002BB900BFDC430020E7A70020D4430020A0
:10415800682A00206C1E002010B5064B04461B6818
:1041680098472146A06004486DF00EF9BDE810405C
:10417800FFF7B6BF9C0300201C1D0020044A054B16
:104188009B1AB1EBD30F34BF52F8310000207047AF
:10419800A85C0900A85E09002DE9F04F8FB0C1F3B3
:1041A8004A2604AF0D469046B8607B600C0D002E81
:1041B80061D04FF000090A234FF0040B07F1140AED
:1041C800FE60C7E90799C7F824900093CDF808B0B6
:1041D800CDF804A007F11C034A464046F968FEF7EB
:1041E80031FFB0F5006F03461CD36C468AB0D8F88F
:1041F800041004AB24481A46C3E9050140F2FF71D4
:10420800D9614FF400711984204B42F8103F4FF4E4
:1042180012514B461E48FFF7BFFFA5462C37BD4637
:10422800BDE8F08FC0F30A0604F11700184420F027
:10423800070080083B60FFF765FE66F353250446D8
:1042480080B13B6800F11001C7E908390A23F96118
:10425800CDE901AB009340460E4AF96807F11C030B
:10426800FEF7F0FE66F353252A4620467B68B968B8
:104278006DF01DFFD2E704F1170020F00700800859
:10428800FFF740FE0446EDE708380A000400000185
:10429800B85D0900892007002DE9F04F87B0054671
:1042A800DDE9106BDDE9127A884614469946BFB1FC
:1042B80010213B465A460020CDF800A0CDF814A0A6
:1042C8006CF0AFFCB0F5006F01460BD340F2FF7302
:1042D8000221184A184807B0BDE8F04F6DF040BFFA
:1042E8003946384604F0070305F00704E40044EAB9
:1042F800831444EA402444EA065406F117000844AB
:1043080020F0070080080391FFF7FCFD054640B147
:104318003FB13B465A460399CDF800A010306CF0E7
:1043280080FC4B4622464146284607B0BDE8F04F80
:104338006DF0BDBE47380A00B85D0900406820B17D
:10434800034BC01A40F3CF0070474FF0FF3070475F
:10435800A85C09000EB403B503AB53F8042B01465F
:104368000448019301F086FC02B05DF804EB03B049
:10437800704700BFCB210700CA0605D48B064CBF87
:1043880002490349FFF7E6BF704700BF02840A00ED
:10439800327A0A002DE9F04F8BB099469DF8588083
:1043A800179B044607930D46DDE918A31A9F06924A
:1043B8000593B8F1000F00F0BC80834B07F0020BA7
:1043C80013F80830089307F4807309936DF04DFED5
:1043D800024600287AD020467C49FFF7BBFF0646F4
:1043E800BBF1000F08D017F0440F71D12A462046C0
:1043F8007749FFF7AFFF064407F0010353B1754B48
:10440800204653F82820744B7449002A08BF1A46DE
:10441800FFF7A0FF07F48073002B07F0080318BF0D
:104428004FF00009002B7FD06D4B204653F8282011
:104438006C49FFF78FFF0546069B2BB11A462046AD
:104448006949FFF787FF0544B9F1000F0DD0089BB4
:10445800002B6CD06549664BB8F1040F18BF19469C
:104468004A462046FFF776FF054462483544079BD5
:104478001BB1224660496CF07CFD059B002B00F0C7
:104488008E80059B3946102B28BF1023204699465D
:104498000026FFF771FFB54252DC0026334620465E
:1044A8001AF803205549FFF755FF0136102E4DD055
:1044B800710703D120465249FFF74CFF4E4533465A
:1044C800EDD320464F49FFF745FFEEE7064687E75D
:1044D8004D4B186800288ED04C4B4FF47A7B1B68E4
:1044E8004FF03C0CB5FBF3F5B5FBF0F14FF461630D
:1044F80000FB11550BFB05F5B1FBF3F2B5FBF0FE24
:1045080003FB121100FB1E55B1FBFCF30BFB05F579
:10451800B5FBF0F50CFB131120460091CDE901E540
:104528003B49FFF717FF66E707F0080584E73049BE
:1045380096E7B9F1010F45460CBF2E48354896E776
:1045480020462F49FFF706FF0136A4E7002620463C
:104558003149FFF7FFFE33461AF803202046A2F13F
:1045680020035F2B28BF2E222C49FFF7F3FE0136CC
:10457800102E0DD0720703D120462149FFF7EAFE1D
:10458800B1453346E8D820461D49FFF7E3FEEEE77C
:10459800059BCA44B3EB090305937FF472AFB8F1E6
:1045A800000F0AD0FB0704D520460B4A0B49FFF73A
:1045B800D1FE39462046FFF7DFFE20460BB0BDE8A6
:1045C800F04F6DF0F1BD00BF3FBA0A008D380A0008
:1045D80091380A00EC6209007F380A00B8820A00A4
:1045E80000630900B7380A00BD380A0084380A0099
:1045F80088380A00CB2107007D5C0000C1380A001A
:104608005BB90A0059B90A00E8430020E4430020D6
:104618009B380A00F9210700C7380A0003820A00FC
:1046280042F20F7373B58B4228BF0B4605680446E8
:10463800052168460D4A68F00FF906466368284662
:104648000B225B680A496DF0A1FD63683246694632
:1046580028465B686DF09AFD63681B2228465B68F4
:1046680004496DF093FD02B070BD00BF35840A00A7
:1046780033BA0A0017BA0A0000210123064A9042F9
:1046880006D8064A01B901231360054B1860704724
:10469800012140085B00F2E740420F00E44300209C
:1046A800E8430020F8B50D460446064F4618B442C4
:1046B80001D12846F8BD14F8011BBB6801485B68A6
:1046C8009847F4E768590900014B036000207047D8
:1046D8004863090070B5104B0D461C68B4B10F4B08
:1046E800196800238B4202DB6FF0010070BD22467F
:1046F80012F8146B864202D014460133F2E7E068E0
:1047080074F063FD28B100202C60EFE76FF00C0017
:10471800ECE76FF01200E9E7A803002048630900FE
:1047280010B5436888B0029383680C46CDE903321C
:1047380000230A68C068CDE90623054901AA059344
:1047480073F006FA079808B9059B236008B010BDF6
:104758008B23070010B54FF42814DFF820C086B06B
:10476800CDE904C40824029404AC0194BDF82040A7
:10477800009471F0E3FA06B010BD00BF18002800DD
:104788002DE9F8430646FCF733FD0546EFF311889B
:10479800202383F31288BFF36F8F114B1C68D3F863
:1047A80004909C4208BF002434B988F31188BFF3F1
:1047B8006F8F2046BDE8F883A7683846FCF718FDD8
:1047C800A84206D12A463946304690F054FD0028C2
:1047D800EBD04C4501D02468E6E70024E5E700BFAC
:1047E800C40300202DE9F0410E461546FFF7C8FF27
:1047F800044628B3C3681BB35F690FB3062E07D0FE
:10480800072E20D02A4631463B46BDE8F0411847DE
:10481800838A3BB92A463146B84750B9A38A01333F
:10482800A38206E04FF6FF72934204D00133A382BD
:104838000020BDE8F0810121114A12486DF087FC83
:104848006FF01500F5E745B12A7832B1002282826F
:1048580031462A465B699847EAE7A38A012B08D1C3
:104868002A4607212046B8470028E2D1A38A013BFF
:10487800D6E70BB1013BDAE70221034ADDE700BFC7
:104888001D390A00805D09003F390A0010B5044649
:1048980008B1806838B9104A104801216DF057FCFA
:1048A8006FF0150010BDFFF76BFF08B10C4AF3E776
:1048B800A082EFF31181202383F31288BFF36F8F57
:1048C800084B5A68C4E9003214605C6081F31188AF
:1048D800BFF36F8FE6E700BF5D390A00805D09000E
:1048E80076390A00C40300202DE9F0410C4B054637
:1048F8001C680E4617467CB100F06AF963682046CA
:10490800D3F8108032463B462946C047044600F09B
:1049180069F92046BDE8F0816FF00104F9E700BFAE
:104928001844002000230360044B5A6812B9C3E9F5
:104938000000704710605860704700BF1C4400209A
:10494800014B1860704700BF18440020002330B5A1
:1049580085B0CDE902330546019000F039F9094BDD
:104968001C6844B9284600F0D5F8044600F03AF926
:10497800204605B030BD636820461B6801A99847EA
:104988002468EEE71C4400201FB5CDE9010103921D
:1049980000F01EF9074B1C6824B900F023F92046E3
:1049A80004B010BD636820461B6801A998472468B5
:1049B800F2E700BF1C4400200022024BC3E900229A
:1049C800704700BF1C4400200022024BC3E90022AC
:1049D800FFF7F2BF244400202DE9F74307460C46B1
:1049E80009B100230B6000261E4DDFF880904D456D
:1049F8000FD31D4B1D6885B355F8188C38464146B2
:104A080001AA183D6DF0A3FD10B3D6B914BB2E460C
:104A18001EE0D5F800803846414601AA6DF097FDA2
:104A280050B116B954B92E4606E000224046316806
:104A38006DF08DFD0028F5D11835D8E7019B23606E
:104A4800F1E70022404631686DF081FD0028DDD194
:104A5800AD69D0E7019B2360D9E7304603B0BDE8D4
:104A6800F08300BFB85E090024440020485F0900B5
:104A78002DE9F04784B002AFD7F8289004460D46D8
:104A8800164698467860B9F1000F07D0D9F800109B
:104A980031BBD9F804A0BAF1000F28D12046391D3E
:104AA800FFF79AFF08B3D0F80C90434632462946E0
:104AB8007868C847C8B16D468AB002AA124BD0615F
:104AC800C2E905344FF400731384104B42F8103FC9
:104AD80000234FF411510E48FFF75EFBAD4604E08A
:104AE8003A1D6DF034FD0028D3D1002007E0D9F835
:104AF800083032460093294643467868D04708373D
:104B0800BD46BDE8F08700BF9F390A0004000001D8
:104B1800F85D09002DE9F04780464FF00047002670
:104B2800DFF8A490DFF8A4A03D46264C4C450DD3F1
:104B3800DAF80040002C40D0183CB8F1000F24D11E
:104B4800226952BBA469F5E72F46EDE7B8F1000FDB
:104B580003D122694AB91834E8E70022414620689F
:104B68006DF0F5FC0028F4D1F5E76368BB4206DD7B
:104B7800AF4202D0AB42A8BF2B461D46EBE7EAD1B5
:104B88009047002E08BF0646E5E700224146206808
:104B98006DF0DDFC0028D3D1D4E76368BB4206DDA5
:104BA800AF4202D0AB42A8BF2B461D46CAE7C9D1C7
:104BB8009047002E08BF0646C4E7AF42C4D130462E
:104BC800BDE8F087B85E0900485F0900244400206A
:104BD8004FF0FF324FF0FF3301482DF0E5BA00BF28
:104BE800F81D002001482DF051BB00BFF81D002022
:104BF80038B5094DFFF7ECFF2B785BB9FFF7E4FEFA
:104C080000F06AF8044608B901232B70FFF7EAFFA1
:104C1800204638BD0024F9E7E9A700202DE9F04334
:104C280006460F46048F99B00134A4B200F1080873
:104C3800651EADB2B5F5004F4AD04A23294605AAEC
:104C480040466DF0DDF904F57F543F34A4B2814647
:104C58002146012340460DF10B026DF0D1F9B9F15F
:104C6800000F014610DC002810DC338FAB4209D15D
:104C780032466B1E22F8383F4FF40041022340466B
:104C8800FEF7B2FE2C46D3E7002808DC294640464A
:104C98006DF0B2F9214640466DF0AEF9E5E7B9F19D
:104CA800490FEFD809F160030DEB03090023094A06
:104CB80009F84C3C05A8009703ABCDF80C80ADF87B
:104CC8001040FFF7D5FE0028DCD019B0BDE8F0830E
:104CD8000020FAE7C72507007FB5012369460420AD
:104CE8000193FFF7F7FC044668BB042002AA01A958
:104CF8006DF069FB044610B110F10C0F23D1039934
:104D0800B1F5803F24D200231846009A94680844DD
:104D180084421BD30133B3F5807FF8D10E4D69610E
:104D28002B8353682846AB60D368EB636DF0DFFCD8
:104D3800044640B9094E28466E60FFF7F3FD284641
:104D48006E60FFF7FDFD204604B070BD9BB2E5E73D
:104D58006FF02004F7E700BF2C4400203C640900F2
:104D68002DE9F04F8BB09146D0F808A01E4600AF51
:104D7800DAF8103080460D469847B9F1000F05DA89
:104D88002B4A01212B486DF0E2F90AE0036846EA54
:104D980009045A1E14400BD00121274A25486DF0FA
:104DA800DFF96FF0150528462C37BD46BDE8F08FB2
:104DB800DAF80CB0BBF1000F06D0294633464A4654
:104DC8004046D8470546EEE7202B01D91B4AD8E7CD
:104DD8002946202207F1080090F028FA2546A64225
:104DE800E1D9331B202B28BF202309EB040BDAF869
:104DF80004505946404607F108027B60A847051E43
:104E08007B6812DA6C4688B06A460D4BCDF81CB048
:104E1800CDE90538042342F8103F00234FF401512F
:104E28000448FFF7B9F9A546BDE71C44D7E700BF1A
:104E3800C4390A00885D0900E1390A00133A0A00FA
:104E4800393A0A0080B505460E46174698462EF0B0
:104E580049F9034600F0DAFC0446DFF818904246A8
:104E680049F8003039463046A84754F8090000F0A0
:104E780045FC00BF0800000008B50348034A0021AC
:104E8800121A6DF070FC08BD4022002040AE0020D0
:104E9800074808B5074A0849121A6DF066FCBDE8CC
:104EA80008400648064A0749121A6DF05EBC00BF62
:104EB8000000002024220020ACF10A00000000209D
:104EC80000000020ACF10A002DE9F84F80460C469E
:104ED80000AF00296AD0D1E90012E9468AB0A36878
:104EE8006D464FF0050A6E463948CDE90723CDE9EE
:104EF800050146F810AF002332464FF421513548DA
:104F0800FFF74AF9D4E90312CD466369AD46324842
:104F1800C5E90723C5E90501C5F810A000233246F5
:104F28004FF421512B48FFF737F9CD46E3690121AA
:104F38002A4A28486DF014F90121294A25486DF0BC
:104F480006F9264600254FF00A0ADFF8A4B0E9461C
:104F5800D6E908C0D6E90A138EB06A46CDF81CC057
:104F680005F1010CCDE908C0A81CCDE90A01E91C2E
:104F7800CDE905B5CDE90C1342F810AF002345F291
:104F8800400114480435FFF707F9102DCD4606F106
:104F98001006DCD1236E0121124A0E486DF0E0F8AC
:104FA800A3690121104A0B486DF0DAF8B8F1010F36
:104FB80007D1EFF305830D4A41460648103B6DF0D3
:104FC800CFF8214640462CF01FFEBD46BDE8F88FBD
:104FD800603A0A00E85D09008F3A0A00BE3A0A0002
:104FE800CD3A0A004A3B0A00593B0A00873B0A00AF
:104FF800073B0A0030BFFFF7FDBF00BF2DE9F041B6
:1050080005460B4EDFF83080324606EB0807CC1B0E
:105018002046084990F0E4F8A01942460021083CCF
:1050280090F004F9C5F8904007F10800BDE8F08158
:1050380000000000485F09000800000010B5244C7B
:10504800244925486DF09EFBA36A99013ED5224864
:1050580022496DF097FB1E20A36ADA0104D51E4889
:105068001F496DF08FFB1F20194CA36ADB0204D582
:1050780019481C496DF086FB0220A36A1C0304D55D
:10508800154819496DF07EFB2120114CA36A59037C
:1050980004D5114815496DF075FB2220A36A9A03BF
:1050A80004D50D4812496DF06DFB2320084CA36A06
:1050B800DB0304D508480F496DF064FB2420A36A7C
:1050C8006FEA03436FEA1343A36210BD1D20C3E7D1
:1050D80000ED00E09A3B0A00E85D0900B23B0A00D7
:1050E800C53B0A00DF3B0A00093C0A00273C0A00CE
:1050F8004C3C0A00663C0A0070B506460D46294C31
:1051080029492A486DF03EFBA36ADB0647D52748A4
:1051180027496DF037FB1120A36A1C0704D52348E3
:1051280024496DF02FFB12201E4CA36A990712D553
:1051380021491E486DF026FB636BA26A120609D549
:1051480001211E4A19486DF00BF81EB1A36A23F01D
:105158008003A3621320134CA36ADE0704D5134807
:1051680017496DF00FFB1420A36A9C0604D50F485D
:1051780014496DF007FB15200A4B9A6AD10658BFEF
:105188009A6A9A6A920642BF5A6A22F400525A628E
:105198009A6A42F0FF029A6200232B7070BD1020B9
:1051A800BAE700BF00ED00E0913C0A00E85D0900A5
:1051B800A73C0A00DA3C0A00ED3C0A00053D0A005B
:1051C8001B3D0A003A3D0A0070B506460D46284CBC
:1051D800284929486DF0D6FAA36AD9043CD526484F
:1051E80026496DF0CFFA1720A36A1A0504D522487C
:1051F80023496DF0C7FA18201D4CA36A9B0512D5E8
:105208001D4820496DF0BEFAA36BA26A100409D5A7
:1052180001211D4A18486CF0A3FF1EB1A36A23F4AC
:105228000043A3621920124CA36A590504D51248F9
:1052380016496DF0A7FA1A20A36ADA050ED50E48AA
:1052480013496DF09FFA1B20094A936A43F47F4380
:10525800936200232B7070BD1620C5E7A36A9B04D8
:10526800F2D505480B496DF08DFA1C20ECE700BF1C
:1052780000ED00E0693D0A00E85D09007F3D0A0095
:10528800DA3C0A00903D0A00A93D0A00BE3D0A002A
:10529800D93D0A003A3D0A00F0B59DB0664B054677
:1052A8005868002600AFC0F3080386F31188BFF3DF
:1052B8006F8F02F07F44B4F17F4F07D102F00C04E6
:1052C800082C0ED15D495E486DF05CFA5D495C487A
:1052D8006DF058FA00210846FFF7F6FD7437BD4611
:1052E800F0BD14074CBF0D460126002DEED000225C
:1052F800FA71DA1E092A7ED8DFE802F0057578719E
:105308007D7D7D7D7D7B50494D486DF03BFA0023C6
:10531800494CFB71E36A9A0705D54C4948486DF03A
:1053280031FA00242DE0E36A002B01DA4849F5E759
:10533800E36A5B00F5D5474941486DF023FA636994
:10534800AA6943F480736361BFF34F8FBFF36F8F14
:1053580032F8023C626922F480726261BFF34F8FB7
:10536800BFF36F8F03F47F42B2F55F4F21D1DBB2F9
:10537800022B1ED12B680121374A31486CF0F0FE10
:105388002C68FB79002BA9D16822294607F108006F
:105398008FF026FF7B6A002E4AD0C3F3080222B999
:1053A8006FEA53236FEA43237B62204607F1080123
:1053B80092E7214B9A6AD2B222B10120F91DFFF778
:1053C8009BFE0EE09A6A12F47F4F04D00120F91D6B
:1053D800FFF7FAFE05E09B6AB3F5803FA1D3FFF71C
:1053E8002DFE0446CDE70020F91DE8E70020F91D51
:1053F800EEE71A4992E71A4A6C4610F4F87F8AB029
:10540800184918BF11466A46103B07934FF40073BA
:105418001548ADF82030154BCDE9050142F8103F8D
:1054280000234FF411510648FEF7B6FEA54678E76B
:105438006FF30803B8E700BF00ED00E01F3E0A0065
:10544800E85D09004A3E0A00863E0A009D3E0A00C1
:10545800BE3E0A00CC3E0A00EB3E0A00073F0A00A7
:10546800063E0A00F13D0A002B3F0A000400000135
:10547800064B5A6942F010025A615A6942F4806236
:105488005A615A6922F008025A61704700ED00E03B
:10549800EFF30880EFF3098101B57246FFF7FCFED0
:1054A80001BD00BF0B4880F308882AF0B1FD202019
:1054B80080F3118808484FF40061401880F3098888
:1054C800EFF314800221084380F31488BFF36F8F31
:1054D80000F068F89049012070E100201EF0040FE8
:1054E8000CBFEFF30880EFF30980816911F8021C03
:1054F8000229FFD001B572466DF039F901BD00BF30
:105508000028ACBF00F16040064B4FEA4111C9B218
:10551800ABBF00F5614000F00F0080F8001319548C
:10552800704700BF14ED00E000B2002807DB01233C
:105538004109034A00F01F00834042F821307047B8
:1055480000E100E000B200280CDB01220649430913
:1055580000F01F008240203341F82320BFF34F8F13
:10556800BFF36F8F704700BF00E100E0054B4209B1
:1055780053F82220012300F01F0003FA00F0104026
:10558800704700BF00E100E0044B054A23F07F03A9
:105598009360BFF34F8FBFF36F8F70470000000019
:1055A80000ED00E008B5FFF7EFFF104BD3F88820B7
:1055B80022F47002C3F88820D3F8882042F4A002AD
:1055C800C3F888204FF04042C3F83422BFF34F8F0E
:1055D800BFF36F8F0023E1EE103AFFF74DFCFFF7A2
:1055E80057FC00F0F3F82CF03BFC00BF00ED00E0A6
:1055F8008189203A41F0020181814FF47D41C0F850
:10560800DC101360009B08495360019B21F00101E5
:105618009360029B9161D3604FF08073D361002344
:105628000265C0F8943070474D4E0000104B9B68DF
:1056380083421AD1EFF30580B8B9EFF31181202224
:1056480082F31288BFF36F8F9A8922F002029A813F
:10565800EFF3148323F0040383F31488BFF36F8FED
:1056680081F31188BFF36F8F70476FF01500704793
:10567800A08000200E461546002300B5E1EE103A42
:10568800EFF3148323F0040383F31488BFF36F8FBD
:10569800BFF36F8F0C4BD0F8902098600B4B1A60BB
:1056A800D0F8803083F30B882C4686F309880020D5
:1056B800034B98472046002100220023014C204735
:1056C800B32707004D4E0000A08000206C44002046
:1056D8001022014B1A61704700ED00E0054B9A69F2
:1056E8009B689A421FBF044A536843F08053536033
:1056F800704700BFA080002000ED00E0084B9B68C9
:1057080083420BD1EFF3058343B1064B5A6842F04D
:1057180080525A605A6A22F400425A6274F0F4B80D
:10572800A080002000ED00E025498A6882F8DDE0CD
:105738004FF030001044EFF3098C80E8F01F1EF0A2
:10574800100F03D102F19C0080EC108A202080F316
:105758001288BFF36F8F1B4F4FF000668A698A600B
:105768003E60D2F89000184C206092F9DDE0D2F843
:1057780094000023C2F8943080F311881EF0100FB3
:1057880003D00023E1EE103A03E002F19C0090EC14
:10579800108AEFF3148323F0040383F31488BFF310
:1057A8006F8F02F1300090E8F01F8CF3098802F146
:1057B800000004B56CF0F2FFBDE80440704700003B
:1057C800A080002004ED00E06C440020002320218C
:1057D8000448C2180133B3F5917F82F80013F8D159
:1057E800704700BF00E100E008B5EFF30583064A03
:1057F800103B02EBC30152F8330049688847BDE803
:105808000840FFF76BBF00BFE8130020014800689D
:10581800704700006C4400201FB50121094B0A4A5B
:105828000A4800F00FF90023064A0393084B0121A8
:10583800019301A8D31A029300F00EF905B05DF8A0
:1058480004FB00BF00FC072000000020586409008A
:10585800402200200A7A0B6810B562F304031C4644
:10586800CB68520923F01F0343EA4203044A43F07A
:105878000103C2F89800C2F89C40C2F8A03010BDDD
:1058880000ED00E010B50A4BD3F89030C3F30723BE
:10589800013B984208D901210346064A06486CF0A4
:1058A8005FFC6FF0150010BDFFF7D4FFFBE700BFEA
:1058B80000ED00E0423F0A00D05D09002DE9F04FFD
:1058C8008946144606464FF000084F4D85B0C84536
:1058D80027DAD6F804A0BAF1000F44D0BAF11F0FA6
:1058E80017D91AF01F0F14D1D6F800B01BF01F0FEC
:1058F8000FD158466CF07CFF07460AEB0B000138C5
:105908006CF076FF874210D06FF015073F4A3B4690
:1059180001E043463E4A01213E486CF021FC6FF00D
:105928001504204605B0BDE8F08F17F1160FEDD02D
:10593800BC42EBDDC5F89870D5F89C10C5F8987096
:10594800D5F8A03021F01F0143F01F0BD6E9003233
:105958001A44994202F1FF3A1AD1D34507D1314688
:10596800F8B26CF04EFF08F101080C36AFE731468B
:10597800C5F89870D5F89C30E0B263F30402C5F816
:105988009C206CF03EFF10F1160FC8D0441CEAE7CB
:10599800C5F89870D5F8A020013B23F01F0302F04A
:1059A8001F021343D3453146E0B2C5F8A030E8D012
:1059B8006CF027FF10F1160FB1D0C5F89870D5F824
:1059C8009C209DF808300BF1FF3B62F304038DF82F
:1059D8000830D5F8A0309DF808205B0863F347121B
:1059E8008DF80820D6E900321344009323F01F03F2
:1059F8005B44A3EB0A03013023F01F036946C0B2DE
:105A08000393FFF73FFFBEE700ED00E08E3F0A007B
:105A1800683F0A00D05D09000522044BC3F89420B2
:105A2800BFF34F8FBFF36F8F704700BF00ED00E0EB
:105A3800BFF35F8F0022024BC3F89420704700BF6A
:105A480000ED00E010B5034C2278FFF737FF207017
:105A580010BD00BFEAA700202DE9F74F294D8A465F
:105A680006464FF00008AB46274FD0451BDAD6F85C
:105A78000490B9F1000F3FD03168084601916CF0ED
:105A8800B7FE0199044609EB010001386CF0B0FE3D
:105A980084424FF014021D4B08D002FB08F36FF04C
:105AA80015024BF8032003B0BDE8F08F14F1160F70
:105AB8002C60F8D01978A142F5DD02FB08B0C7F8D0
:105AC8009840C7F89840D7F89C4000F10801007B3F
:105AD80064F304000871D7F8A0000C79400860F35B
:105AE80047140C71D7F89C1021F01F016960D7F892
:105AF800A01021F01F01296108F1010814350C36A6
:105B0800B3E700BF7044002000ED00E0EAA70020E2
:105B1800F0B55349534DD1F890302C68C3F307239F
:105B28009C4287B000F299800020FFF781FF4E4B1E
:105B3800C1F8C030844216D14C4D01A82C70FEF734
:105B4800C3FD002607464A4CB74213D100202B78E4
:105B58004349D1F89020C2F30722934277DBFFF73D
:105B68005BFF002046E0696801EB0011FFF772FE59
:105B78000130DFE70199300101EB0613DA682240B2
:105B8800B2F1807F52D00AD8B2F5001F34D0B2F5F6
:105B9800800F3ED0B2F5801F12D00136D4E7B2F1A3
:105BA800006F43D0B2F1805FF7D15A689B680958FB
:105BB800013B22F01F00034423F01F03012032E0C1
:105BC8005A689B680958013B22F01F0003440120D2
:105BD800844623F01F0340EA4C10CDE902218DF8DA
:105BE800100002A928780593FFF74CFE00282ADA4E
:105BF8006FF0150007B0F0BD5A689B680958013B63
:105C080022F01F0003444FF0020C012023F01F0371
:105C1800E1E75A689B680958013B22F01F000344DA
:105C2800022023F01F034FF0000CD4E75A689B684A
:105C38000958013B22F01F0003444FF0030C0120D8
:105C480023F01F03C7E72B7801332B70A5E7C1F8B2
:105C58009830C1F8A00001337BE74FF0FF30C9E767
:105C680000ED00E064640900AAFF4400EAA70020F0
:105C78000000F0FFF0B587B007460E461446002135
:105C8800102268461D468FF0D1FA02238DF80230A3
:105C9800054B2A4621466846CDE90476019366F00D
:105CA8006DFF07B0F0BD00BF4328070008B5024BE1
:105CB8001B689847002008BD84440020034B044A11
:105CC8001860937843F0020393707047844400206F
:105CD800CC03002008B505486BF09DF9002383F339
:105CE8001188BFF36F8F0423184602DFC03F0A00F4
:105CF80008B50549054A21F007010548521A6AF016
:105D08003EFF002008BD00BF938E012000FC072045
:105D1800884400204FF0FF324FF0FF3301482CF049
:105D280043BA00BFDC03002001482CF0AFBA00BF23
:105D3800DC03002038B50546FFF7ECFF2A460821AA
:105D480007486AF062FE044628B925B1FFF75EFDF0
:105D58000C22044B1A50FFF7E7FF204638BD00BF5E
:105D6800884400200C00000038B504460D46FFF7B3
:105D7800D1FF21462B46082207486AF0C8FE044690
:105D880028B925B1FFF742FD0C22044B1A50FFF742
:105D9800CBFF204638BD00BF884400200C0000001F
:105DA80010B50446FFF7B6FF21460348FDF78AF809
:105DB800BDE81040FFF7B8BF8844002070B5A0FBCD
:105DC800015434B92846FFF7B5FF064640B93046B6
:105DD80070BDFFF71BFD0C22044B00261A50F6E796
:105DE8002A4621468FF022FAF1E700BF0C00000096
:105DF80070B541690446867A0A4D59B1437ADB0782
:105E080006D42C2303FB06535B6A1B689B689847E0
:105E1800002363612C20214600FB0650BDE870403A
:105E280073F0E2BBD81E00202C22024B02FB00308C
:105E3800704700BFD81E00202C21827A054B01FB39
:105E480002339A6A1B7F801A1B3323F00303B0FBCB
:105E5800F3F07047D81E002038B52C24827A064B00
:105E680004FB02335B6AD3E901240C601568FFF771
:105E7800E3FF04FB005038BDD81E00202DE9F04395
:105E880085B00546684690461C46039173F096FE19
:105E9800DDE90067EFF31189202383F31288BFF34C
:105EA8006F8F6B8B002B41D02A8B9A4225D9002209
:105EB800002328462CF03AFA0446F0B189F31188F9
:105EC800BFF36F8F039B002B41D032463B46684699
:105ED80073F099FE2C21A27A254B204601FB023350
:105EE8005B6A03A91B681D68DDE90023A847606198
:105EF80070BB2046FFF77CFF24E0698B4B1E6B8349
:105F080089F31188BFF36F8F2B7F2A8BAC6A1B3301
:105F180023F00303521A02FB0344154B154AEB1AEC
:105F28009B105343A3722B7FE372CBE789F311884D
:105F3800BFF36F8F2346424628462CF0F7F90446F4
:105F48000028BFD10024204605B0BDE8F083636176
:105F5800012300252381039B29466382E27A656039
:105F680004F118008FF062F963692582E360EAE7BB
:105F7800D81E0020A38B2EBAF8B500242C260F4D6E
:105F880000B9F8BD476800F10802D2E8EF3F591E92
:105F9800C2E8EC1FBCF1000FF7D1DBB2012BF0D146
:105FA800837AC46006FB035344601B6A13B19847A5
:105FB8003846E5E7FFF71CFFFAE700BFD81E0020C8
:105FC8002DE9F84F06460D4617460446A346646871
:105FD800002CFBD14FF02C09DFF878A0BBF810306B
:105FE800BBF81220DBF81410D21ADBF80C300BF1D6
:105FF8000C005B1AD21AAA4228BF2A461FFA82F856
:10600800394642466CF0CAFCB5EB0805444447449F
:106018001DD00C9B53B1DDE90A010D9A98478346C0
:10602800A8B1014630466CF07BFCD7E7B07A09FB93
:1060380000A0436A9B6843B1AB4228BF2B46194670
:10604800DDE90A23FFF71AFFE9E72946F8E72046C2
:10605800BDE8F88FD81E002008B5244A244B1A60E2
:1060680028F0C2FA4FF47A612248D0F82436C3F3F4
:106078000802C3F309434B4382F480721E498832F5
:1060880001FB02334FF4FA215B00B3FBF1F201FB91
:1060980012331A49B3F57A3F28BF0132C1F80429EF
:1060A800D0F820364FF47A60C3F30802C3F30943EB
:1060B800434342F21C5082F4807202F2172200FB22
:1060C80002334FF47A701B0AB3FBF0F200FB123371
:1060D8000020B3F5FA7F4FF0010328BF0132C1F861
:1060E8001C27C1F80009C1F8003608BD0020A10727
:1060F8000C0E002000C0FF00F82A0080000012509B
:1061080048B1054B054A1B68B3FBF2F35843044BEF
:1061180043F00103184770470C0E002040420F005F
:1061280010600900BFF34F8F0549064BCA6802F497
:10613800E0621343CB60BFF34F8F00BFFDE700BFA2
:1061480000ED00E00400FA05F7B506460D461446D2
:10615800124F384673F039F8E0B1BB68314638461B
:106168001B68AAB29847002802DB002003B0F0BDE4
:10617800002CFBD1AC42F8D22F1B042F28BF0427D8
:1061880072F0B0FB3A46019001A930198FF028F857
:106198003C44EFE76FF01200E8E700BF4C590900F4
:1061A80038B504462CF07AFF20466CF061FCA069F3
:1061B800C8B194F86C30DB070DD50221154A164892
:1061C8006CF054FC6FF07705201D6CF058FC2CF037
:1061D80079FF284638BD72F0F8FF38B901210F4A17
:1061E8000D486CF043FC6FF01205EDE7204600F017
:1061F800B5FF05460028E7D10146242204F128000E
:106208008FF014F894F86C3043F0010384F86C3084
:10621800DAE700BFDC3F0A00685E090006400A00B2
:1062280070B504462CF03AFF20466CF021FC94F837
:106238006C30DA070DD40221254A26486CF016FC8A
:106248004FF0FF35201D6CF01AFC2CF03BFF284660
:1062580070BDC3F340019B0707D502211E4A1D48A4
:106268006CF004FC6FF07705ECE7A06970F073FE42
:106278000646A06970F0FFFE054628B10121174ABD
:1062880014486CF0F3FBDDE7A36F4BB131462046B1
:106298006CF0CFFD0546A0B1A06970F014FFD1E7FE
:1062A800A06970F090FEA0670028EFD101210C4A88
:1062B80008486CF0DBFBA06970F005FF6FF00B0578
:1062C800C0E794F86C3043F0020384F86C30B9E707
:1062D80029400A00685E09004F400A0075400A001C
:1062E80091400A0038B590F86C3004469B0708D4F2
:1062F8000221144A14486CF0B9FB6FF07705284660
:1063080038BD6CF0B5FB0021204601F0C1F820B182
:1063180001210E4A0C486CF0A9FBA06970F0D3FE6D
:10632800054620B101210A4A07486CF09FFB94F802
:106338006C30201D23F0020384F86C306CF09FFB56
:10634800DDE700BFAD400A00685E0900D4400A00DE
:10635800F2400A002DE9F04385B006460C46904607
:106368006CF08FFB0546B8F1000F07D030466CF093
:106378008DFB012810D1B5FA85F56D090134294640
:106388003046E2B26CF06EFD814650B901212346D9
:10639800324A33486BF0E4FE0024204605B0BDE8DD
:1063A800F0834768B8F1000F09D03868796801AB05
:1063B80003C33A7A01AF1A7007238DF80530F18DBF
:1063C8007B883046994228BF19466CF09DFE0446EA
:1063D8000028E1D0038A428A4169D21AC36800F1D1
:1063E8000C085B1AD21A3B7839469A4228BF1A46DB
:1063F80040466CF0D3FAD9F80C90B9F1000F08D1E7
:10640800218AF38D9942C8D94046C91A6CF0EDFA31
:10641800C3E7D9F8040083681B6B13B9D9F8009057
:10642800EBE7294698470028F8D0071F57F8041FBC
:106438000029F3D008780028F0D0628A238AA2EBDA
:10644800030C6269E3689B1AACEB0302904294BFA9
:10645800024692B240466CF0A1FAE7E722410A00F0
:10646800485E090038B50446806F6CF041FA05466D
:106478006CF0F7F92046294601F052FA044638B183
:1064880004480121044A6BF062FE2846FFF774FDB8
:10649800204638BD485E090048410A0038B58021C9
:1064A8000446806970F0B2FD054678B10146204681
:1064B80001F036FA044638B106480121064A6BF065
:1064C80046FE2846FFF758FD204638BD6FF00B04FE
:1064D800FAE700BF485E090067410A0000232DE97A
:1064E800F04F93B005930B7E044633F080060F46B9
:1064F80015460AD00121AD4AAD486BF028FE6FF071
:106508000406304613B0BDE8F08F82B10846FFF7A5
:1065180033FD7B7EDA0704D49D07F2D53B7E002B42
:10652800EFD1204613B0BDE8F04FFFF79BBF4A7E7E
:1065380000F12809900705D5802B09D13846FFF7C7
:106548001BFDDEE7910700F03884002B40F035840E
:10655800D3071ED53B8A082B12D1FA68394613682F
:106568000020A3625368C9F804306CF0EBF9059079
:1065780080B18F4801218F4A6BF0E9FD059805E04D
:106588008B4801218C4A6BF0E2FD3846FFF7F4FC9A
:106598001EE00597FFF73AF9002394F82850874A38
:1065A80015F0600F8350C5F341131CD0032B40F046
:1065B80064836FF08505FFF729F9804B1B58002B82
:1065C80000F0A183002D00F0698305980028DDD133
:1065D80048466CF08EFB0346A069002B00F0288427
:1065E800802100F02EBC48466CF083FB94F82930DB
:1065F800002840F02C81013B0A2BDAD801A252F87E
:1066080023F000BF4B670000BB650000D1670000A6
:10661800BB65000039660000BB650000BB65000073
:10662800BB6500009F660000BB65000013670000A3
:10663800A069618D03697F2993F88030B9D8A28D4C
:10664800002AB6D1E28D002AB3D1EE06B1D194F872
:106658003020022A02D14FF0FF35ACE71D070BD5D9
:10666800C9B26CF07CFB054648B1638D0121544AE0
:106678004F486BF075FD9EE7012384F8393094F894
:106688003030012B05D1638D1BB984F830300025DB
:1066980091E70123F9E720466CF0F3F9628D014692
:1066A800FF2A86D8E38D002B83D194F82830D806AA
:1066B8007FF47FAF94F83030002BCCD092B9618D45
:1066C80094F838308B42E2D02046C9B200F0E0FEA0
:1066D800638D054668B1012100903A4A34486BF051
:1066E80049FD68E72046D2B26CF0E2FB0028E6D10B
:1066F800B1E7002B14BF02220122052184F83020C3
:1067080020461A466CF049FDC1E705F01F05012D2A
:106718007FF44FAFE38D002B7FF44BAF628DFF2AE0
:106728003FF647AFA18DFF293FF643AF94F83030CD
:10673800022B90D12046D2B2C9B26CF069FC054652
:1067480039E7E38DA68D002B7FF433AF94F8303012
:10675800002B80D0012B02D1002E7FF47CAF15F0E6
:106768001F0515D0022D92D1B4F82A80B8F1000F78
:106778008DD1F6B23146204601F03AF9421C054661
:106788003FF419AF4246314620466CF0B8FA12E79A
:10679800002E7FF460AF638D012B7FF478AF94F8FF
:1067A8006C3066F3C30384F86C3070E78A410A00E2
:1067B800485E0900C2410A00AB410A000C00000013
:1067C800E4410A0006420A00A38DE28DDEB2002AE7
:1067D8007FF4EFAE628D022A11D105F01F05354313
:1067E8004FEA13217FF4E5AE0122A0696CF097FA15
:1067F80000287FF4DEAE012384F8393047E794F8A7
:10680800301000293FF427AF012902D1002B7FF473
:1068180022AF15F01F050FD0022D7FF438AF002AE4
:106828007FF435AF3146204601F0C0F8431C0546D9
:106838003FF4C1AE0122A6E7002B7FF40CAF012A7A
:106848007FF425AF94F86C3043F00803ABE70A2BCC
:1068580063D8DFE813F00B00620062006200620098
:1068680062003A006200DD016200F201E38D022B52
:1068780053D194F83030002B4FD0012BA18D01D18A
:1068880000294AD115F01F050ED0022D17D0002679
:10689800022120466CF038FC054618B131460C3010
:1068A8006CF08DF80595F2E6002936D194F86C3035
:1068B8009E0806F00206C3F300131E43E8E72046CD
:1068C800C9B26CF045FC0646E2E7618DED064FEA79
:1068D8001123C9B207D0002320460AA90A936CF0F5
:1068E80057FA0A9DDEE7013B0E2B16D8DFE813F0B6
:1068F8000F003000380015001500D20036001500D2
:106908001500150015001500150015000F0120468B
:106918006CF0B7F818B1012818D00025C2E7266F27
:10692800002EFAD0B4F82E8033782046984528BF38
:10693800984641466CF0E8FB05460028B2D042462E
:10694800314605F10C006CF029F8ABE7666FE7E714
:1069580000222046FFF7FEFC0546A3E70122F8E7E0
:106968000A46204603216CF018F980460028D4D046
:106978006CF0BAF9E58D98F81530B8B998F8146044
:106988008DF82930AE428DF8286028BF2E46D8F8F9
:10699800103031461B882046ADF82A306CF0B4FB25
:1069A80005460028B9D032460AA9CAE74FF0000ABE
:1069B800B44A8DF81130D8F808308DF810A01A4074
:1069C800B14B9A4255D1102106A828F0E5FC061EC5
:1069D80036DB0AAB102E984628BF1026AB4806AA0D
:1069E800564503F1020334D8B6000236F6B28DF8E4
:1069F8001060AE4228BF2E46204631466CF084FB1C
:106A08000546002889D0022EB34628BF4FF0020B56
:106A18005A46A6EB0B06C34600F10C0A504604A9D9
:106A28006BF0BCFF730808EB56025A4528D1F007F3
:106A38007FF538AF504618F803106BF0B8FF31E710
:106A480058367FF46AAF0121914A92486BF07FFB78
:106A580063E712F8011B0AF1010A4FEA111C01F061
:106A68000F0110F80CC0415C03F802CC03F8011CBC
:106A7800B6E798F81460D8F810808DF81060B8E779
:106A880050461BF8011BCDE902236BF098FFDDE9A6
:106A98000223CAE720466BF0F4FFD4E91C53002810
:106AA80008BF1D460A2300268DF8283006232046F5
:106AB800CDF82A60CDF82E608DF829306BF0E6FF0E
:106AC80001287FF42AAF002D3FF4ECAE6B882046F6
:106AD800ADF82A302B798DF82C306B798DF82D3064
:106AE800AB798DF82E30EB798DF82F306B7C8DF8E3
:106AF8003030E68D9DF828309E4228BF1E4631462C
:106B08006CF002FB054600287FF44DAFCAE620462C
:106B18006BF0B7FF20B101287FF4FFAE636F00E090
:106B2800236F002B3FF4F9AE5B88B3F5007F7FF647
:106B3800F4AE594B04F14C060A9300238DF82C301F
:106B4800E36C9E4208BF0023BDF82A2093B1597D0B
:106B58000F2908D1197D0A44ADF82A209DF82C2068
:106B680001328DF82C20226D9A4201D01B68EBE788
:106B7800BDF82A20B4F82E802046904528BF9046BC
:106B880041466CF0C1FA054600283FF4C6AE9DF8B0
:106B9800282000F10C0A424528BF424650460AA95F
:106BA8006BF0FCFE9DF82830434594BFA8EB030822
:106BB800A8EB0808B8F1000F3FF474AED4F84CB055
:106BC800B3453FF46FAEBBF1000F3FF46BAE9BF8DB
:106BD80015300F2B15D19BF814205046424528BF7D
:106BE8004246DBF810106BF0D9FE9BF81430434591
:106BF80094BFA8EB0308A8EB0808B8F1000F3FF40E
:106C080051AE236D5B453FF44DAEDBF800B0DAE7DB
:106C180094F83030002B3FF480AEE18D01297FF4E9
:106C28007CAE94F8386020466CF06EFA0546002871
:106C38003FF438AE31460C30FFE605F01F05012D54
:106C48007FF46BAE20466CF021F900283FF465AE66
:106C5800A38D4268FF2B3FF660AE12799A42FFF48B
:106C68005CAEDAB20F2A3FF658AEE18D01297FF407
:106C780054AE234493F83A60D5E7204605A96CF052
:106C880087F85CE500FF02000003020044BA0A002E
:106C980029420A00485E0900050F050072F08CFFC2
:106CA8004FF47A76A0FB060C47F61222002306FB67
:106CB80001C1FAF731FA654BD3E8AF1F41F28732C9
:106CC800461A9642624A39D9D3E8EF6F8E4204D108
:106CD800C3E8EC0FBCF1000FF6D12FD1D2E8EF3F9B
:106CE800C2E8E15F0029F9D123B10221594A5A4883
:106CF8006BF036FA0221594A57486BF028FAFEF72A
:106D080085FD574B1D58002D7FF45FAC7B7EE28DCF
:106D1800D9071BD548466BF0ECFFB8B9BAB129467C
:106D2800A06970F05FF90146059000283FF450AC67
:106D3800204613B0BDE8F04F00F0F2BDD2E8EF3FB7
:106D48000133C2E8E13F0029D9D0F7E73AB9204634
:106D5800FFF7A4FB00287FF43BACFFF7E2BB4846F3
:106D68006BF0C7FF059D18B92846FFF705F9EEE750
:106D7800002D3FF42DAC2946204600F0D1FD08B186
:106D8800284603E4A069036993F8801011F0040110
:106D98007FF4C7AB70F03AF9054600283FF418AC09
:106DA8000146204600F0BCFD00283FF4BAAB0121A3
:106DB8002C4A29486BF0CBF9E2E752077FF508AC7B
:106DC800002B3FF4BBAB3846FFF7D6F894F83930C0
:106DD800002B3FF496AB94F82930052B0CD1618D2C
:106DE800A069C9B26BF0BBFF054628B1638D0121CC
:106DF8001D4A19486BF0B4F994F82930032B11D1C6
:106E0800638D022B0ED1A18D00220E0A3146A06996
:106E18006BF085FF054628B101213346134A0E4819
:106E28006BF09EF900232E4684F83930FFF769BBD2
:106E3800E38D002B3FF4D4AB0599003918BF01212D
:106E4800C9016FF0E6FFFFF76CBB00BF9844002054
:106E5800944400204B420A00485E09005F420A0041
:106E68000C00000088420A00E4410A00AC420A0013
:106E78000B7810B4062B14D10369D3F89C20EFF3D8
:106E88001184202383F31288BFF36F8F00204B688F
:106E98001860506A60B9C2E9083384F31188BFF3F7
:106EA8006F8F0022002304485DF8044B72F08CBAFF
:106EB80003605362F1E700BF3C1E002030B589B083
:106EC800002200230024CDE906236FF007034FF4C6
:106ED8008062CDE90334CDE90144154B154900948E
:106EE80015482BF0DFFD1549134872F008FD144BC7
:106EF80014498B4207D30020134B14498B420CD3FF
:106F0800002009B030BD03F11402D2E8EF0FC2E847
:106F1800E54F002DF9D11833EBE703F11402D2E85D
:106F2800EF4FC2E8E50F002DF9D11833E6E700BFAF
:106F3800B16F000040B10020A02A002047800A005D
:106F480064210020C4210020C42100202422002024
:106F580038B50D466BF09AFF30B90121BDE83840CD
:106F68000F4A10486BF0F3B8C46804B938BD2B78E1
:106F7800032B05D0052B0ED0022B08D02468F4E78C
:106F8800606883685B69002BF8D09847F6E760680B
:106F980083689B69F7E760688368DB69F3E700BF8C
:106FA800D3420A00585E09002DE9FF4120274FF01F
:106FB800FF334FF0FF32644801A92BF091F8039B8F
:106FC8001B69D3F89C40236A93B1EFF3118287F3CE
:106FD8001288BFF36F8F216A29B1606A0B688142FA
:106FE800236208BF636282F31188BFF36F8FC9B948
:106FF8009DF80430062BDAD0072BD8D801A252F816
:1070080023F000BF51700000457000007970000047
:1070180057700000AD7000009B700000B76F000053
:10702800417100000B7E20465D06D1F81E2002D17A
:10703800FFF754FAC7E76BF079FFC4E70022012194
:1070480020466CF0AAF8B2E700221146F8E794F857
:107058006C3043F0040384F86C3094F83030022B21
:1070680003D1204601A9FFF773FF00220321E7E7B8
:1070780094F86C3023F0040384F86C3094F83030C2
:10708800022B03D1204601A9FFF762FF002202214B
:10709800D6E794F83030022B89D1204601A9FFF7B2
:1070A80057FF84E794F86C30A66923F0040384F84A
:1070B8006C30D6F808803369A033D3E8AF3F9A071D
:1070C8001ED53046D8F83C309847D8F824300021EF
:1070D800304698470546D8F840303046984795B12D
:1070E8001A4A01211A486BF032F80022042120467E
:1070F8006CF053F8002D3FF45AAF2A4607219FE75A
:107108004FF0FF35ECE72946204600F0C1F9054667
:1071180008B1104AE5E7A0696FF097FF831E58424F
:10712800584194F86C3084F8305023F0680343EAEF
:10713800401384F86C30D8E70121074A04486BF003
:1071480006F80621029A7BE73C1E002002430A004B
:10715800585E090030430A005C430A0038B502460D
:1071680005460C4980696FF0CEFF044630B1012115
:10717800094A0A486AF0EBFF204638BD85F838000E
:10718800284600F043F904460028F5D0A8696FF0B6
:10719800E9FFF1E7796E00006C430A00585E0900C8
:1071A800F8B501231D460C68002C35D063F07F022A
:1071B800D6B202F07F02103224FA02F7FF0716D582
:1071C800046824FA02F7FF0708D43346134801215C
:1071D800134A6AF0C5FF6FF01500F8BD05FA02F210
:1071E80024EA020404600C6824EA02040C60DC400F
:1071F800E6070ED5026822FA03F4E40700D4E5E7AF
:1072080005FA03F422EA040202600A6822EA040288
:107218000A600133102BC6D10020DEE7885E090022
:1072280093430A002DE9F04F0026536891B0D468C3
:107238000A900891069202930E96039674B9039BDE
:10724800029A09339BB293701B0AD370069B16717E
:10725800DC68002C40F0C780A346AEE04FF0000A7F
:107268006068CDF83CA083681B6B002B00F0AC80F5
:1072780008999847002800F0A7803546C4E903AA72
:10728800A0F1040959F8043F0BB11A789AB9B5422C
:1072980040F29780E3680F9A1343E360606883685D
:1072A8009B6A002B00F0928098478346002800F0E4
:1072B8009080534A7DE05A780B2A08BF9D70D9F810
:1072C80000305A78042A10D1E2680F990A43E26024
:1072D800DA78002A5CD101229D702369AA40134301
:1072E80001352361EDB2CDF83CA0D9F800707B7868
:1072F800052BC7D16FF0120B4FF001080A9B9B6951
:10730800099379793A790E9B42EA0122ADF8362041
:1073180097F902205FFA88F1002AACBF424641F093
:1073280080010493B7BF4BB24FFA88F321F0800273
:107338000793A8BF0793049BB8BF103223FA02F043
:10734800C0072CD40F9B23FA02F20593D30726D447
:10735800BB79FA78099800930DF136030B916FF019
:10736800CEFC0B998346D0B9079BB970002B4FF020
:107378000103BCBF21F0800110318B4004980599AE
:10738800BDF8362019431843CDE90E01BA8079E7D4
:107398006A1E9A700FA90EA8FFF702FFA3E708F16B
:1073A8000108B8F1100FACD1BBF1000F3FF46AAF80
:1073B800144A012114486AF0CAFE584611B0BDE8C3
:1073C800F08F6FF0150BF3E7354667E76FF0850B25
:1073D8006FE7606808996BF079FD039B2E460344BC
:1073E800246803932AE7E36804F10C01A3600EA85C
:1073F800FFF7D6FE08B924682BE76FF0150BDCE71A
:10740800D4430A00B0430A00885E090070B5836956
:1074180005461B69026F93F88030C3F34113022BB2
:107428000CD0032B0CD0012B0CBF10230823D371D5
:10743800EE6D3EB96E6DBEB9344611E02023F6E715
:107448004023F4E7324601212846FFF7EBFE0446C5
:1074580040B173685B790B4A01210B486AF080FEE2
:10746800204670BD3668E4E7324600212846FFF71B
:10747800D9FE044618B173685B79044AECE73668AC
:10748800D9E700BFF8430A00885E09001B440A00D8
:107498002DE9F04105460E466BF0F3FA95F83830C1
:1074A800804633B328466BF0F1FC0746F0B101463D
:1074B80028466BF05BFD10220446002105F13A00D6
:1074C8008DF0B4FE002385F83830FF683FB984B1E9
:1074D80019491A486BF0B9FC2046BDE8F081786874
:1074E80083685B6A03B198473F68EFE76FF03C0435
:1074F800EEE71EB985F838600024EDE732464146CC
:1075080028466BF0AFFC074690B1024628466BF060
:1075180057FD04460028DFD185F83860FC68002C48
:10752800EAD0606883681B6A03B198472468F6E765
:107538006FF03C04D0E700BFD4400A00405E090069
:107548002DE9F04105460F461446D2F804806BF049
:1075580080FC95F86C30D9070BD5474947486BF044
:1075680074FC6FF00F07281D6BF07AFC3846BDE8F5
:10757800F081012F0AD128466BF088FA30B94049CA
:107588003E486BF062FC6FF08507ECE798F807302F
:107598009A0607D5AB691B6993F880309B0701D41D
:1075A8003849EDE71FB1012F06D03749E8E7EB6D01
:1075B8002BBB05F1540603E06B6DABB905F15C0616
:1075C800002233680BBB002FD5E91C2308BF1346E4
:1075D8005B7C626803F10103DBB25371D5E91C12CD
:1075E80008BF0A46537422E09C4206D12749234823
:1075F8006BF02BFC6FF01507B5E71B68DDE79C42C5
:1076080001D12349F3E71B68D2E79C4221D12368C3
:10761800CAB972683360944200D173600023236052
:1076280063685B7902211B4A14486AF099FDA168D6
:10763800B9B128466BF0CBFA074668B116490F482E
:107648006BF003FC8FE7136073689C4208BF72609D
:10765800E4E71A461B68B5E7A0686BF045FB88F8B5
:1076680006000023236073681BB9C6E9004400279D
:1076780079E71C607460FAE76C440A00405E090010
:107688008E440A0048440A00AC440A00CC440A006C
:10769800E9440A0006450A0023450A00F8B50546EC
:1076A80000AF29B301290BD1184C194E2BE06368A0
:1076B80028461968F9F78AFDB8B11834B442F6D3E8
:1076C8006C4688B06A46134BCDE905354FF4007314
:1076D800ADF81C30104B42F8103F00234FF4E25134
:1076E8000E48FCF759FDA54600242046BD46F8BDC6
:1076F8000B4C0C4EE2E7636828461968F9F766FDFB
:107708000028F2D01834B442F5D3D9E7C4210020B8
:10771800242200205A450A0003000001505E090097
:1077280064210020C421002070B5012501F07F03E9
:1077380011F0800F18BF10339D4090F83030044688
:10774800022B06D001210C4A0C486AF000FD0020EB
:1077580070BD90F838606BF094F9324601462046C7
:107768006BF080FB0028F2D0C0680028EFD0836857
:107778001D42EDD10068F8E778450A00505E09001F
:107788002DE9F84305460846114616469846FFF780
:1077980085FF0446002843D028466BF090FB95F8F7
:1077A8006C30DA0702D5204A012109E0D4F80490A8
:1077B80004F11407D7E8AF3FDB070CD502211B4AB9
:1077C8001B486AF0C4FC6FF00F04281D2AF05EFD08
:1077D8002046BDE8F883D9F804301BB1AB4201D08C
:1077E800144AE1E74246314628466BF03BFBA0B11C
:1077F8000023236003696BB9C0E90344D7E8EF3F6E
:1078080043F00103C7E8E23F002AF7D10024C9F892
:107818000450DAE71C600461F0E76FF03C04D4E739
:107828006FF01204D4E700BF6C440A009D450A00BB
:10783800505E0900BF450A002DE9F04F83B000AF44
:107848007B6097F830304C680E463B608146904626
:107858006BF017F9A36801461B6B33B96FF0150479
:1078680020460C37BD46BDE8F08F204698470028D3
:10787800F4D00024051F06F10C0A55F8041F09B1BD
:107888000B782BB9002C14BF00246FF03C04E7E7F9
:107898004B78042B0ED1002C3CD18B787A6893421C
:1078A800EBD1CB783A689342E7D10B79002BD7D04C
:1078B8000124E2E7052BE0D1002CDED0B8F1010F5E
:1078C80091F802B009D0B8F1020FF1D152465946E9
:1078D800D9F818006BF002FC04E05246D9F81800F9
:1078E8006BF0E0FB04460028E2D06D468AB06A4699
:1078F800F368CDE907B3062307490990CDE90518D0
:1079080042F8103F00234FF441510448FCF744FC6F
:10791800AD46A5E70024A3E7FF450A00805E0900FD
:107928002DE9F0410B7E0C465906054637D16BB35D
:107938006BF0E7F840B11B4801211B4A6AF007FCCD
:107948004FF0FF30BDE8F0812846D5F87080268AD0
:10795800EF8D6BF096F8F8B1421E534253419B01EC
:10796800228A9AB1BE42324628BF3A46E98D9142F0
:107978000CD9B2FBF3F103FB11223AB994F9183090
:10798800002BBEBF637E43F0080363762146A869D7
:10799800BDE8F0416FF099BA98F80730E0E76FF06A
:1079A8001500CFE7705E09003B460A0070B5064631
:1079B80080690C466FF02DFA054638B1022123463E
:1079C800094A0A486AF0CCFB284670BD012214F027
:1079D800800F18BF24F08004736B18BF1034A240C6
:1079E8001A437263F0E700BF4F460A00705E090051
:1079F80070B5054680690E466FF036FA044638B110
:107A080002213346054A06486AF0AAFB204670BDA3
:107A1800314605F134006BF037FBF7E766460A009C
:107A2800705E090070B50646EFF31181202383F3D9
:107A38001288BFF36F8F1B4D2A6881F31188BFF33B
:107A48006F8F526892F86C20D20705D4BDE8704059
:107A5800202200232AF076BFEFF3118283F31288E5
:107A6800BFF36F8F2C682CB1696823688C422B6038
:107A780008BF6B6082F31188BFF36F8F44B16068F1
:107A880004F10801C36998472146074871F039FC99
:107A98002B6833B13046BDE87040002200232AF03D
:107AA80019BF70BD9C440020B41D002030B585B0BE
:107AB800CDE90012054600220023144803A92AF044
:107AC80075FA0246E8B9DDE90001039B5D600833F9
:107AD80083E80300EFF31180202383F31288BFF3B8
:107AE8006F8F039B1A600A4A516861B9C2E9003373
:107AF80080F31188BFF36F8F0022002305482AF016
:107B0800E9FE05B030BD0B605360F1E7B41D0020FD
:107B18009C4400200000002073B5202504698DF8DE
:107B28000710EFF3118685F31288BFF36F8F0122D8
:107B3800206C0DF1070169F0E9FE86F31188BFF3A7
:107B48006F8F012812D071F0D4FEC8B10122104BFA
:107B5800D3E8EF1F002903D1C3E8E02F0028F7D1AD
:107B680004D102210B4A0C486AF0F1FA237F2BB1A9
:107B78002022002304F148002AF0ACFE02B070BDB8
:107B8800A37E002BE2D00021202071F0BAFFC8E7C5
:107B9800A444002090460A00385E090038B5002445
:107BA80005690E492B6C05F14800C3E90144DC6006
:107BB800AB6BC3E90144DC6071F043FE05F178006A
:107BC800074971F0E1FD074905F1280071F0DCFD76
:107BD80028466BF007FB204638BD00BF117D00002A
:107BE800597E0000257F00002DE9F3410369064610
:107BF8000D46D0F804801C690F7E002A32D00B8A0B
:107C080071323E480BBF022101213D4A3D4A009393
:107C18003B466AF0AFFA30462F7E6BF04CFB87424A
:107C280004D1042104F188006BF0F2FB30462F7E6A
:107C38006BF04FFB874204D1052104F188006BF0FB
:107C4800E7FB30462F7E6BF028FB874203D104F117
:107C58008C002AF003FC2946404602B0BDE8F041FA
:107C68006BF073BA6BF027FBB84214D12A8AE96823
:107C7800A06B69F04BFE28B1236A1BB104F1280000
:107C88002AF0B8FD04F1880004216BF0C1FB04F16F
:107C980078002AF0AFFD30462F7E6BF01AFB874242
:107CA80015D1236A1BB104F128002AF0A3FD052190
:107CB80004F188006BF0ACFB237F9BB9002340F6EE
:107CC800354204F148002AF005FE012323773046A7
:107CD8002F7E6BF0E2FA8742BDD104F18C002AF0C6
:107CE8005BFBB8E7236C5A89DB889A42EFD0002205
:107CF800002304F148002AF0EDFDE8E7385E0900AA
:107D0800AF460A00D3460A002DE9F04750F8483C30
:107D180000F140075B68054600213846D3F800901B
:107D28006BF0B5FA002864D0012138466BF0AFFA41
:107D3800804600285DD155F8083C5A89DB889A426C
:107D480003D115F82D3C002B53D0D7E8EF4F44F062
:107D58002003C7E8E23F002AF7D114F0200448D1F5
:107D680048466BF0B6FA00228246002322486AF0A1
:107D78007DFD064650B9384605216BF049FB28467B
:107D8800BDE8F047202200232AF0A4BD80F818A0FF
:107D980015F82C3C33B1428AC16855F8080C69F0D3
:107DA800D5FD0446214606F10C006AF0F1FD5CB1F0
:107DB800D9F804006BF00AFBB4FBF0F303FB1044A2
:107DC800B4FA84F84FEA58183146484605F82D8C1D
:107DD8006BF0A3F968B10121084A09486AF0B7F9BC
:107DE8003046FEF7C9F83846BDE8F04705216BF084
:107DF8000FBBBDE8F08700BF301F0020F4460A0023
:107E0800385E090038B503461B6940685D68AC6890
:107E1800A37A84F8223094F82D3084F82330A3769E
:107E2800696849B1237C3BB96AF0D1FE30B10121C0
:107E3800054A06486AF08BF9002038BD68686AF080
:107E480053FF2074F8E700BF06470A00385E0900B0
:107E580070B550F8782C00F11004526803460021E0
:107E6800204615686BF013FA00284DD001212046F2
:107E78006BF00DFA002847D153F8402C68689388B6
:107E8800918916695B1A9BB2F61A6BF09FFAB04299
:107E98003AD8D4E8EF3F43F01002C4E8E12F0029B4
:107EA800F7D1DB0606D5BDE870400221174A18480D
:107EB8006AF04DB928466BF0FEF900220646002309
:107EC80014486AF0D3FC0446F0B1067668686BF093
:107ED8007DFA638A984203D268686BF077FA83B2B6
:107EE8002146284663826BF018F968B128466BF082
:107EF800E2F9034606480121074A6AF031F92046AB
:107F0800BDE87040FEF738B870BD00BF30470A00C2
:107F1800385E0900301F002050470A0038B550F875
:107F2800083C044633B9BDE8384001212A4A2B48A9
:107F38006AF00DB950F8283C00F160055B68022131
:107F48001A6800238382838328466BF0A0F9B8B1AE
:107F580054E9023110699847637D1BB104F1500060
:107F68002AF048FC052128466BF091F998B9637FFF
:107F78006BB10022002304F120002AF0ABFC0AE0D8
:107F8800032128466BF083F90028E1D1E4E714F8CF
:107F98000D3C002BEDD1022128466BF078F938B161
:107FA8002369DA885B899A4202D020462AF022FCAB
:107FB800032128466BF06BF960B1A2699388918917
:107FC80012695B1A9BB29A4204D02046BDE8384039
:107FD8002AF010BC38BD00BF75470A00385E09009A
:107FE800D3B5002600270446CDE9006705486AF0A6
:107FF80041FC28B1230658BF0023047658BF0382EA
:1080080002B0D0BD642000202DE9F04383B00023E6
:108018004FF0010805691C4C1C4E02AF28602B77F5
:1080280085F8203005F12409B442234601D3002005
:1080380019E095F820201034CAB16C4688B01B6846
:1080480002AA1349C2E905134FF400739383114B35
:1080580042F8103F104800234FF4E251FCF79CF817
:108068006FF00B00A5460437BD46BDE8F08385F8E0
:10807800208054F8043C4846009354F8101C54E9F6
:1080880003236BF091FCCFE7D0130B00E0130B0038
:10809800D7470A0003000001905E09001FB5CDE92B
:1080A800010103924FF0FF324FF0FF3301A903485B
:1080B80071F08AF9002005B05DF804FB0C1E002061
:1080C8001FB500230190CDE902334FF0FF324FF086
:1080D800FF3301A9024871F077F905B05DF804FB98
:1080E8000C1E00202DE9F041044617460E46006894
:1080F8006BF0C2FA31463A468046FFF771FFD4F872
:108108007B300546DB1B0146C4F87B3020686BF0EA
:1081180004F888B10B4A434601210B486AF020F85D
:10812800314620466BF073FB2846FDF725FF2046B5
:10813800BDE8F0416BF037BBA37F0133A377BDE8FF
:10814800F08100BF50470A00905E09002DE9F84F02
:10815800044600686BF0A5FA4FF030090746E37F44
:10816800012B1ED82368D3F810B0D3F804A09BF8CD
:10817800616009FB06B6243630466BF03BFC31469D
:108188000246804650466BF0A2FA9BF81F3005461F
:1081980033B1A8EB0002314650466BF098FA054619
:1081A8000DB9BDE8F88F20466BF04EFA2A46014615
:1081B80006463846FFF714FF0546014620686AF070
:1081C800ACFF80B101213B46094A0A4869F0C8FF63
:1081D8002846FDF7D1FE314620466BF018FBBDE876
:1081E800F84F6BF0E0BAE37F0133E377B7E700BFFE
:1081F80050470A00905E09002DE9F04FB94F89B049
:108208004FF0FF324FF0FF33B74805A929F068FF58
:10821800059E069D3469002D40F09080257704F175
:10822800240694F820309D42C0F2828004F118039D
:10823800D3E8EF2F22F00202C3E8E12F0029F7D19B
:10824800D3E8EF1F21F00401C3E8E21F002AF7D1A9
:1082580004F11803D3E8AF3FDB07D1D5237F022B06
:1082680000F08E81032B00F0878153BBDDF814A04A
:10827800DAF81050EB7F23BB50466BF012FA8146B8
:1082880028466BF0E1F94FF400720146064648466D
:10829800FFF7A6FE8046014650466AF03EFF0028DA
:1082A80000F0668101214B46904A914869F058FFD9
:1082B8004046FDF761FE314628466BF0A8FA6BF0A0
:1082C80072FAA37F002B9BD1237F012B40F07D8185
:1082D800302304F1630694F86150304694F8621034
:1082E80003FB054500F060FA243502463146236950
:1082F800284600F077FA0646C4F8840028466BF052
:108308006FFB814628466BF070FB804628466BF071
:1083180071FBE26D3044002A40F03B81002840F0B8
:10832800338128466BF08DFB003818BF01202CE103
:1083380030466BF04CFB0135303672E7DDF81C80B7
:10834800D6F804A095F81890B8F1000F21D02B8A20
:1083580018F1710F6648009308BF02214B4616BFFB
:108368000121644A644A69F005FF304695F818808F
:108378006BF097F9804540F0EF80E37F013BE377AE
:10838800204669696BF043FA294650466AF0DDFEDB
:108398005EE730466BF085F9484540F09580237FCD
:1083A800D5F80C80B5F810B0002B49D1BBF11F0FE0
:1083B80042D1D8F80030BB423ED1414604F15403C3
:1083C80008F11C0251F8040B914243F8040BF9D14F
:1083D8000A881A808A7842219A70552384F8733063
:1083E800532384F8743084F87630A36DE26DC4F8B2
:1083F80077300023C4F8803094F86030C4F87B20CC
:108408009A0684F875100FD194F8612094F82030FA
:108418009A4209D294F86230013B0F2B04D8012309
:1084280084F87F302377A0E720686BF030F90223C7
:1084380084F87F300423F5E720466BF0B4F994E71D
:10844800032B92D1302394F8619003FB0949D4F8A7
:10845800803009F124095B44C4F88030BBF1000F77
:1084680016D048466BF0C6FA90B141465A4648467F
:108478006BF0D2FA804628B902215B461F4A1C4895
:1084880069F06EFED4F87B30A3EB0803C4F87B30A8
:10849800D4F88020E36D9A420DD248466BF0AAFAD0
:1084A80000287FF462AFD4F88020E36D9A4202D2AC
:1084B80020686BF002F948466BF0C3FA003818BF21
:1084C800012084F87F00B5E7304695F818906BF0E6
:1084D800D3F881457FF449AF237F052B10D184F869
:1084E8001C8042E7555342430C1E002050470A00A7
:1084F800905E0900AF460A00D3460A00EE470A001C
:10850800022B7FF432AF4FF030092A8AD4F880303A
:1085180094F861801344C4F8803023681969D3F84B
:1085280004B091F8613009FB031124310846039126
:108538006BF060FA0399024658466BF0C8F80028B9
:108548007FF413AFD4F87B3013B120686BF09FF839
:1085580009FB08402430AFE7304695F818806BF0E7
:108568008BF8804502BFA37F03F1FF33A37707E7AA
:10857800EB7F0133EB77A4E62046FFF7E7FDA0E6A3
:1085880020466BF054F99CE6022084F87F0004230F
:108598001AE094F9601040B90029206802DA6BF0FB
:1085A80076F8BEE66BF089F8BBE6002914DA90424B
:1085B80002D8B9F1000F06D120686BF068F80223E1
:1085C80084F87F30E3E702232377237F022B0ED141
:1085D80020466BF02CF913E6904202D8B8F1000F50
:1085E80003D120686BF069F8E9E70323ECE7032B74
:1085F80003D12046FFF7AAFD02E6042B7FF400AE64
:10860800A37F2BB101211D4A1D4869F0A0FDF7E5A4
:1086180020686BF031F8804620466BF015F8054667
:10862800024604F1730304F17F0153F8040B8B42F3
:1086380042F8040BF9D11B782946137040460D22E5
:10864800FFF7CEFC0646014620686AF066FD78B161
:108658000C4A434601210A4869F082FD3046FDF77D
:108668008BFC294620466BF0D2F86BF09CF8C7E5E6
:10867800A37F0133A37705232377C1E514480A00B4
:10868800905E090050470A00802938B50D46144607
:1086980021D083290DD019BB802353718323032054
:1086A800117193710023E07023706570A37004301A
:1086B80038BD0223137101235371002393710A23D8
:1086C800D37108224168A0188CF0E7FD064B0E20F4
:1086D8001B882382E6E7044B02201B889380E1E78E
:1086E8006FF08500E4E700BF5AB90A002DE9F041B0
:1086F8008769D0F82480BA4228BF3A46B2FBF8F41A
:108708000646C2692346006869F003FF0546C0B9FA
:10871800B7FBF8F7A7420BD1002205213068FCF718
:1087280061F828B101210A4A0A4869F010FD0125BB
:10873800F3692344F3613DB10020074BB362BDE800
:10874800F08100240125E7E7706A6043F7E700BF7E
:1087580035480A00905E09000203000C81420B466E
:1087680007B509D302210D4A0D4869F0F9FC6FF0ED
:10877800150003B05DF804FB6AB101391144814268
:1087880001D28B4207D90221009305481346054AB6
:1087980069F0F0FCEBE70020EBE700BF4C480A006B
:1087A800905E090063480A000C290346084616D162
:1087B8001B78252B12D009D8122B10D8084A42FA58
:1087C80003F313F0010F08BF0620704703F0FD0202
:1087D800282A03D05A2B08BF0A2070470A2070475E
:1087E800F6FFFBFF2DE9F041984690F82C3086B053
:1087F80023F00C0380F82C300023C0E90433836194
:10880800062A04460F460B7840F010810BBB4B79C3
:108818005B0724D490F82C309F070DD402234FF423
:1088280068521946002584F8283084F82910628592
:10883800284606B0BDE8F0816BF038F80028EDD185
:10884800002319461A46EDE70223052145F20232B4
:10885800E8E7032B36D14E7916F0040604D002233C
:1088680005214FF41052DDE790F82C308DF80760A1
:1088780043F0040380F82C307023ADF8043090F8EE
:1088880029300D7903F00F038DF806300A23122DD5
:1088980028BF12258DF80B30438D2A465BBA404617
:1088A80001A98DF808608DF809608DF80A600396B3
:1088B800ADF81030ADF81260ADF814608CF090FC93
:1088C800A662B5E71B2B00F0898009D8122B1AD0B5
:1088D8001A2B61D00121B24AB24869F041FCBEE7C7
:1088E8001E2BF7D14B795E07B9D40B7913F003032C
:1088F80000F09780012BA3D190F82C3043F00103AE
:1089080080F82C309CE74B795E07A8D490F82C307F
:1089180043F0040380F82C304A7812F002061FD185
:10892800D5078B7822D5B1F8035042461946FFF790
:10893800ABFE6DBAADB285420BDAB7F803506DBA2B
:10894800ADB200231A4684F8283084F8296062857D
:108958006EE742462046B978FFF796FE051EF0DA24
:10896800022305264FF410520025ECE72BB1022113
:108978008D4A8C4869F0F4FBF2E7B1F803504146A0
:108988006DBAADB26AF0C8FF232DD6D9414620464C
:108998006AF0C2FF2425D4E74D7915F004057FF469
:1089A8005EAF90F82C3043F0040380F82C308B78BD
:1089B8003F2B0ED1CE78002ED2D10D790323042D72
:1089C80028BF042540462A4601A901938CF008FCDB
:1089D800B7E7022305264FF41052B4E74B7959073D
:1089E8003FF53DAF3B791A090CD19A070AD5DB0749
:1089F80015D494F82C3003F00303032B3FF424AF71
:108A0800002305E094F82C209707C2F34003F0D523
:108A180094F82C2063F3410284F82C2010E70123FA
:108A2800F6E790F82C2063F30002F5E70A2A7FF4B2
:108A380051AF2A2B1AD8222B7FF64CAFA3F1230271
:108A4800072A3FF647AF01A151F822F0CB8A000070
:108A5800DD8800004D8B0000DD880000DD88000007
:108A6800B58B0000DD8800000D8C00005A2B7FF4C8
:108A780031AF4D7A15F004057FF4F1AE90F82C3043
:108A880043F0040380F82C308B783F2B40F0DD80D6
:108A9800CE78002E40F0D9804FF4C063CDE901367E
:108AA800B1F8075040466DBAADB2082D28BF082569
:108AB80001A92A468CF094FB3246334684F82820D4
:108AC80053E07B7A13F004037FF4C9AE01AEADF82E
:108AD8000430B370082390F82C208DF8073042F04A
:108AE800040280F82C206AF0E1FE0028B5BF4FF0A0
:108AF800FF3302220322236A8DF80C20A8BF1BBA79
:108B08000293636A31461BBA8DF80D30C3F307220E
:108B1800C3F307438DF80F3094F82C308DF80E20EE
:108B280043F0040384F82C30B7F8075040466DBA78
:108B3800ADB20C2D28BF0C252A468CF051FB002322
:108B4800A36275E67E7A16F004067FF488AE90F884
:108B58002C3043F004039D0780F82C3009D40226FA
:108B68004FF46853002584F8286084F829606385E9
:108B78005EE66AF09BFE0028F1D1236A03B1013B4F
:108B880094F82C10626A1BBA12BA41F0040184F8F6
:108B98002C100825C8F80030C8F804200023E2E7A4
:108BA800AA480A00905E09008D480A007B7A580797
:108BB8003FF555AE94F82C30D7F8026043F0040323
:108BC8009907B7F8075084F82C307FF527AE204670
:108BD8006AF06CFE00287FF421AE6DBA36BAADB2E9
:108BE8002A463146206AFFF7B9FD20B10223052144
:108BF8004FF4045216E6174B2361636AE6616B4330
:108C0800A3611DE67B7A5A073FF529AE90F82C3010
:108C1800D7F8026043F00803B7F8075080F82C3003
:108C28009B077FF5FBAD6AF041FE00287FF4F6ADA7
:108C38006DBA36BAADB22A463146206AFFF78EFDC4
:108C48000028D3D1044B6361D7E7022205264FF4ED
:108C5800105333E783390700F586000010B504691F
:108C68000346204640F8143B0122002170F0E0FC46
:108C780004F12C00024970F087FD002010BD00BFF0
:108C8800158E000038B503461B6940685C681B698F
:108C980025685A681AB19A680AB1DA683AB9134865
:108CA8000121134A69F053FA6FF0150038BD1033EB
:108CB800D3E8EF1F41F00101C3E8E21F002AF7D112
:108CC800216909B90020F1E72B7A002BFAD169F064
:108CD8007EFF28B10121074A044869F038FAF1E714
:108CE80020696AF001F82872ECE700BF785E090095
:108CF800C5480A0006470A0038B504694068006894
:108D080004F11005D5E8AF5FED071FD40BB15D681E
:108D18003DB9104A1048012169F019FA6FF01500A1
:108D280038BD90F820501DB1DD680DB90B4AF1E748
:108D380085791DB19D690DB9094AEBE7C4E90212AD
:108D480063600274120A42740020E9E76FF077004A
:108D5800E6E700BFEF480A00785E09000E490A00FE
:108D68002D490A002DE9F347D0F804A00669884682
:108D780015467768DAF8044006F11003D3E8AF3FE8
:108D88009B073BD5236960685B68D3F8009069F05E
:108D980078FE00220023012829460CBF99F81B9071
:108DA80099F81490DAF80C00CDE90023424669F0EE
:108DB80061FD054650B90121124A134869F0C7F907
:108DC8006FF00B04204602B0BDE8F087014680F83A
:108DD800189020466AF0A1F9044618B12846FDF714
:108DE800CBF8EFE7FB69002BECD14FF0FF324FF0E7
:108DF800FF3306F1140029F00BFBE3E76FF00C04D6
:108E0800E0E700BF4E490A00785E090070B550F8E7
:108E18002C3C5C6865681C38D0E8AF3F9B0725D5BB
:108E28002B6968685B681E6869F02BFE00220128C0
:108E38004FF00003A0680CBF96F8296096F82260EE
:108E480069F014FD044630B9094A0121BDE87040B3
:108E5800084869F07CB90146067628466AF05DF94B
:108E680020B12046FDF788F8034AEEE770BD00BF41
:108E780069490A00785E090083490A0070B50B78D1
:108E880092B006460C4607AD032B31D8DFE803F055
:108E9800022A2C2E19492846F8F7A2F90595637875
:108EA800174A0493A3781E210393E3780AA8029330
:108EB800237910AD019363790093A37963F0CCFC17
:108EC80032460AAB1C4603CCAC42106051602346C4
:108ED80002F10802F6D1206810603046A38893801A
:108EE80012B070BD0749D6E70749D4E70749D2E76A
:108EF8000A212846064A63F0AFFCCFE7B8490A00C2
:108F0800D3490A0099AB0A00BF490A00C9490A00B7
:108F1800746B0A000E4B402928BF402170B51D46CE
:108F28000C4C4618B04203F1020304D1002305F8A3
:108F38001130074870BD02781209A25C03F8022CB0
:108F480010F8012B02F00F02A25C03F8012CE9E7EC
:108F5800EBA700209DBA0A0010B50024094B86B083
:108F680009480393CDE9044470F064FC03AB009313
:108F78004FF440620A230549034829F041FC204682
:108F880006B010BDFD490A00602C002040BB00203F
:108F98000146014829F074BC602C002001460148B4
:108FA80029F09EBC602C00200146014870F017BCD7
:108FB800602C00202DE9F743064689461746984657
:108FC8003C4DD5E8AF3FDA0722D548B901213A4AE6
:108FD8003A4869F0BCF86FF0010003B0BDE8F083CF
:108FE80001A969F0D8FA022804462BD1024634496F
:108FF80030468CF023F90028EDD1D5E8AF3FC3F314
:10900800C0061B0706D52F4A21462C4869F09FF851
:109018000020E2E7A5F18804072221464046B84728
:1090280006280AD80121284A244869F090F845F80A
:10903800886CE671C4F80360EAE70723B0FBF3F035
:10904800E071E5E7042818D10246204930468CF043
:10905800F5F804460028BED11C22404605F1A001BF
:10906800B847031E05DA0121194A144869F078F84F
:10907800CEE72B4483F8A040CAE70A28ABD10246C2
:10908800144930468CF0DAF80028A4D1B9F1020F5F
:1090980007D00A480121104A69F059F86FF0150005
:1090A8009BE74A46404605F1BE01B84700EAE07032
:1090B80093E700BF08020020064A0A00485D09003D
:1090C800C6490A00274A0A004B4A0A0036500A00D5
:1090D800704A0A00A24A0A00AD4A0A002DE9F04384
:1090E80089B0DDF840909D795E791F7993F803C0C7
:1090F80093F802E093F801800C461B78B9F1000F51
:1091080015D0CDE90639CDE904E81346CDE9027C4E
:10911800CDE900560D4A63F09FFB002813DBA042FF
:109128002CBF6FF01500002009B0BDE8F083CDE931
:109138000583CDE903CE1346CDE90167044A0095BE
:1091480063F08AFBE9E76FF01500EDE7E44A0A00EF
:10915800084B0A0010B5FBF74BFD044628B1012166
:109168000346034A034868F0FBFF204610BD00BFD2
:10917800294B0A00485D090070B504461E4615468D
:109188008CB0AAB129B10A4602A8042168F0C9F92D
:1091980002A900912B462246242103A8FFF79EFF2F
:1091A80070B93146109A03A8FBF79EFB0CB070BD4E
:1091B80003462421044A03A863F04EFB2328F0D970
:1091C8006FF01500F2E700BF4E4B0A0007B50B4BD6
:1091D8000B48DA79C2EBC202009200221146FFF76F
:1091E800CBFF034638B10121064A074803B05DF8B2
:1091F80004EB68F0B5BF03B05DF804FB8001002004
:10920800C6490A00544B0A00485D090030B50446B7
:1092180015468DB09AB129B10A4602A8042168F012
:1092280080F902A900912B462246242103A8FFF7C2
:1092380055FF60B903A869F086F90DB030BD034643
:109248002421044A03A863F007FB2328F2D96FF00E
:109258001500F2E74E4B0A0007B5009313460A467D
:1092680001460348FFF788FF03B05DF804FB00BF21
:10927800B3680A000A4601460148FFF7C7BF00BFA6
:10928800B3680A0007B5009313460A460146034827
:10929800FFF772FF03B05DF804FB00BFAD680A007A
:1092A8000A4601460148FFF7B1BF00BFAD680A0092
:1092B80007B5009313460A4601460348FFF75CFFCB
:1092C80003B05DF804FB00BFDE660A000A460146EB
:1092D8000148FFF79BBF00BFDE660A0007B5002202
:1092E8000346009103481146FFF746FF03B05DF8B7
:1092F80004FB00BFA5680A0007B5002203460091D9
:1093080003481146FFF738FF03B05DF804FB00BFC0
:1093180036500A0007B5002203460091034811465B
:10932800FFF72AFF03B05DF804FB00BFA24A0A005A
:1093380008B5024829F05EFA002008BD5C08002044
:10934800F8B51E4DD5E8AF3F13F0010F2F4632D0C8
:1093580095F8A040A5F188063CB91C22184906F5E5
:1093680094708BF09AFF86F84441F3798BB902F038
:1093780039F8044630B10121124A134868F0E7FE73
:109388002046F8BDF37923B902F03CF804460028DA
:10939800F1D1D5E8AF3F5A0701D400F0C5FED7E8B0
:1093A800EF3F23F40062C7E8E12F0029F7D11B053E
:1093B80001D5FFF7BDFF0024E2E700BF0802002047
:1093C8006F4B0A00764B0A00485D090007B5009309
:1093D80013460A4601460348FFF7CEFE03B05DF880
:1093E80004FB00BFE46D0A000A4601460148FFF786
:1093F8000DBF00BFE46D0A0030B50378012B11D012
:10940800022B21D06BB90A46144B03F1100453F810
:10941800045BA34242F8045BF9D143881A0A8A70B4
:10942800CB7030BD0A460D4B03F1100453F8045BB2
:10943800A34242F8045BF9D143681A0C180E4A702B
:109448000870C3F30722EAE700F11003013913F8A3
:109458000129984201F8012FF9D1E2E7AEBA0A00D2
:1094680010B56AF051FD70F044FA044608B929F0C5
:1094780015FE064BD3E8AF3F0BB10A2098471CB93D
:10948800BDE8104029F01EBE10BD00BF6851002085
:1094980038B50446084869F0E9F9054648B1631E3D
:1094A800DBB21F2B96BF054A0021D15C0C3069F056
:1094B8007EFA284638BD00BFE01F0020BEBA0A0069
:1094C8000F2810B50CD80D280CD90A4869F0CEF928
:1094D800044618B104210C3069F069FA204610BD21
:1094E8001328F2D009B10448F0E70220BDE8104083
:1094F800FFF7CEBF902000205C1F0020C3681B78B8
:109508000221024A02486AF09DBD00BFB84B0A001A
:10951800105D0900F8B506460F4604F0F5FA044652
:1095280090B9394630460AF061FF0546F0B9394628
:10953800304608F0A9FF164B1B6823B153F80C49B5
:1095480004B10C3CB3B9F8BD83781321012B4FF05B
:10955800000312BF1D46D0F8A450C0F8A4306BF029
:109568009EF9204603F05CFE002DDAD028466DF007
:1095780014FADCE79B6813B13946304698472CB19A
:10958800E26802B10C3A23461446DBE72246FAE7C2
:109598003052002010B5002486B003AB00934FF47E
:1095A80080624FF0FF3305490548CDE9034405942F
:1095B80029F026F9204606B010BD00BF40C700209C
:1095C800602D002038B5C5682B7893B9B5F80140EF
:1095D8000F21204603F082FFEB78054650B90A4A6E
:1095E800118831B96FEA04506FEA10501080074AA9
:1095F800137038BD0373012103F05EFE2846BDE8F1
:10960800384003F00DBE00BFB8A500206CA80020AC
:1096180070B5C3681D787DBBB3F801600F21304673
:1096280003F05CFF044638B901213346BDE87040B9
:10963800124A13486AF006BD294603F03DFEA37896
:10964800012B04D02046BDE8704003F0E9BD201D81
:109658006AF0E1FCC307F5D50321204603F02CFE90
:10966800032002F019FF03460028EBD00221054A27
:1096780003486AF0E7FCE5E770BD00BFE04B0A006D
:10968800105D0900064C0A0010B5C3680121B3F843
:109698000140204603F022FF38B901212346BDE8E6
:1096A8001040044A04486AF0CDBCBDE8104003F0FD
:1096B800B7BD00BF2C4C0A00105D090010B5C36887
:1096C80001211C88204603F009FF38B901212346EF
:1096D800BDE81040034A04486AF0B4BCBDE8104035
:1096E80003F09EBD2C4C0A00105D090010B5012145
:1096F8000C3069F09AF903780121BDE81040024A5C
:1097080002486AF09FBC00BF504C0A00105D090077
:10971800014610B5084869F0C0F80849084870F0D3
:109728005EF8031E06DABDE810400121054A064826
:109738006AF088BC10BD00BF840200207C080020AD
:10974800602E0020724C0A00105D09000121024AB7
:1097580002486AF063BC00BF8F4C0A00105D090024
:1097680070B5C5680121B5F80160304603F0B6FE52
:10977800044638B901213346BDE870400B4A0C480D
:109788006AF060BC2B783BB9D5F80330C0F8993043
:10979800D5F80730C0F89D30201D4FF400316AF02D
:1097A80046FC2046BDE8704003F03ABD2C4C0A0048
:1097B800105D090008B502F025FE064B18466AF050
:1097C8002AFC00F00B00D3E8EF2FC3E8E10F0029D3
:1097D800F9D108BD080200200B46B0B50D8A00AFCC
:1097E80004462946D868FFF795FB8AB06A460A4BB3
:1097F800CDE90750CDE9053440F20243ADF82430F5
:10980800064B42F8103F00234FF432510448FAF750
:10981800C3FCBD46B0BD00BFA94C0A00050000014D
:10982800105D09002DE9F84FD0F80C90018A99F8DD
:10983800004000AFA30001338B4260D96D468AB067
:109848006A46CDE9073105232E48CDE9050442F8DB
:10985800103F00234FF421512B48FAF79DFCAD46E9
:10986800BD46BDE8F88F01212B46284A26486AF0F4
:10987800E9FB013699F800309E42F1DA09EB8603DC
:10988800B3F801500F212846B3F8038003F026FEF1
:1098980004460028E7D000F1C00AB8F1000F06D04E
:1098A800656945B901211A4A17486AF0B7FB20468D
:1098B80003F0B6FCDDE7A2692B6895422046636198
:1098C80008BFA36103F0CCFB28F066FDC5F800B023
:1098D800236A8BB9C4E90755DAE8EF3F013BCAE8C8
:1098E800E23F002AF8D10021204608F1FF3803F0B2
:1098F800C1FB1FFA88F8D0E71D602562ECE7002657
:10990800B346B7E7CB4C0A00105D0900F64C0A00D5
:10991800124D0A0080B500AF8AB06A46094BCDE9FE
:109928000530094B079340F20133ADF82030074B5F
:1099380042F8103F00234FF412510548FAF72CFC67
:10994800BD4680BD294D0A00377A0A00040000018F
:10995800105D090037B50446084602EBC3039A4276
:1099680002D16FF05E0010E0114611F8085BA542C5
:1099780011D1038A5178994209D908480121084A26
:10998800009468F0F7FB6FF0150003B030BD536822
:1099980098470020F9E70A46E1E700BF105D090093
:1099A800454D0A002DE9F0470C4629F077FBE5689C
:1099B8002B78022B72D0042B07D001213B4A3C485C
:1099C8006AF040FB6FF015040EE0B4F81080B8F1AF
:1099D800020F0ED84346374A354801216AF032FB58
:1099E8002046FCF7C9FA002429F06CFB2046BDE8A4
:1099F800F08768783E280CD1B8F1030F02D12E4ABF
:109A08004346E9E7EB78012B01D00A2B46D103271F
:109A180004E06AF0EDFA0746F8073FD504F10C06B2
:109A280001213046D4F814A068F0F7FF022130462F
:109A380068F0FBFF814600783E2807D1E3681B7871
:109A4800012B01D00A2B06D1032614E06AF0D0FAC4
:109A5800C10706460FD441F28A13184A1849194813
:109A680067F0E6FA002383F31188BFF36F8F0323AF
:109A7800184602DF0226144A0623214699F80000F8
:109A88006AF001FBB2070DD56369A5EB0A0513FA65
:109A980085F5E560A4F81080BB07A4D52046FFF73C
:109AA80037FEA0E72046FCF767FAF5E70D4E0A00F7
:109AB800105D0900674D0A00834D0A00A34D0A0096
:109AC800D74D0A00F04D0A008865090010B501213C
:109AD80004460C3068F0A9FF2146BDE81040022377
:109AE800014A00786AF0CFBAB865090073B53E48F4
:109AF80068F0E8FE0446002873D000F10C052846FB
:109B080068F09BFF0228034603D0042847D0374A51
:109B180003E0238A032B05D8354A012135486AF02A
:109B280091FA13E00421284668F07FFFFF2342885A
:109B380006882376238AC6F30B009A42608309D0ED
:109B4800012100922B482C4A68F014FB2046FCF7B0
:109B580013FA12E00F2103F0C1FC054610B9638B1C
:109B6800264ADAE703F0E0FC21462076320B284645
:109B780003F0D2FA284603F053FB214BD3F8043103
:109B88007BB3204920486FF02AFE031E29DA012101
:109B98001E4A184802B0BDE870406AF053BA284619
:109BA800022168F042FF054600783E2812D06AF08C
:109BB8001FFA10F002060DD140F6BC43144A1549AD
:109BC800154867F035FA86F31188BFF36F8F0323C2
:109BD800184602DF06232146104A28786AF053FA0D
:109BE800B4E702B070BD00BF84020020B64E0A0080
:109BF800214E0A00105D0900424E0A00664E0A0016
:109C0800800100207C080020602E0020724C0A0091
:109C1800A34D0A00884E0A00F04D0A00C8650900E5
:109C280010B5012104460C3068F0FFFE2146BDE85E
:109C380010400D23014A00786AF025BAF86509003A
:109C4800F8B50121044600AF0C3068F0EEFE067846
:109C5800002321463046114AFFF77CFE5F301AD1B7
:109C6800258AE0682946FFF755F96C468AB06A46A6
:109C78000B4BCDE90750CDE9053640F20243ADF86C
:109C88002430084B42F8103F00234FF43251064865
:109C9800FAF782FAA546BD46F8BD00BF606609001E
:109CA800CA4E0A0005000001105D09002DE9F74FB2
:109CB8000023804689461746DFF810A1DAE8EF4FFF
:109CC800CAE8E23F002AF9D1264644B901214346B1
:109CD8003A4A3B4803B0BDE8F04F6AF0B3B92046B2
:109CE800FCF7AAF84FF00C0B364D0BFB00504388DD
:109CF80043451BD02046FCF79FF80BFB00504388D8
:109D080001210093304A43462D4868F033FADAE8D7
:109D1800EF3FCAE8E26F002AF9D1002B4BD01E466C
:109D2800304603B0BDE8F04FFCF726B9A74208D08B
:109D3800204668F096FD3A8AF96804F10C0068F04C
:109D48002DFE2046FCF778F80C2707FB00504368E7
:109D5800ABB1B9F1000F12D12046FCF76DF8012123
:109D680007FB00504268536803F01F0081401068E9
:109D78005B0900EB8300137ACBB16AF058F92046EF
:109D8800FCF75AF80C2707FB00508368002BC7D054
:109D98002046FCF751F8784305F800902046FCF778
:109DA8004BF807FB0055A86828F0F6FAB8E7C9434E
:109DB8006AF04FF9E3E703B0BDE8F08FFC4E0A0004
:109DC800105D09006C510020244F0A008002002019
:109DD80073B5C5680121B5F80160304603F07EFB14
:109DE800044640B9012133463D4A3E4802B0BDE829
:109DF80070406AF027B92B78061D1A2B19D1C37841
:109E0800012B50D14FF4804130466AF010F94204DA
:109E18000FD4D4F88C3069460093D4F89430204697
:109E2800019304F09FFB204602B0BDE8704003F0A8
:109E3800F7B92B78BBBB40F2E242B5F803302A49A8
:109E48005343C4F88830B5F80520A4F89020B5F835
:109E58000720A4F89220A3F5EA520C3A8A4204D9C2
:109E68000221224A1F486AF0EDF8B4F89030B3F5A1
:109E7800FA7F04D302211E4A1A486AF0E3F840F632
:109E88007641B4F89230A3F10A0292B28A4204D918
:109E98000221184A13486AF0D5F86FF48051304609
:109EA8006AF0D7F814E030466AF0B5F8C304F4D580
:109EB8002B78202BF1D194F89830002BEDD0013B72
:109EC80084F898300C4A002304F1400028F002FD81
:109ED8002B78002BA7D1204603F0FCFCA3E700BF9A
:109EE8002C4C0A00105D090095F03C00574F0A0001
:109EF8007E4F0A00A54F0A005A62020010B5C1E958
:109F080000239DF808300C460B72FBF795FF0C22D6
:109F1800024B02FB00335C6010BD00BF6C51002097
:109F2800F8B502460B46104868F0A0FC0446C0B1DC
:109F380004210C3068F021FD2046FBF77DFF0C273B
:109F480000260A4D07FB005046802046FBF774FFA9
:109F580007FB005086602046FBF76EFF07FB0055A5
:109F68006E602046F8BD00BFB41F00206C51002071
:109F78000138C0B202289ABF014B185C0020704714
:109F880008BB0A0037B50C468DF8070000F0FF053E
:109F9800A0B929B1072220460A498BF04FF940B9E8
:109FA800002009490DF107020AF08CF9002003B0DE
:109FB80030BD21462846FFF7ADFAF7E76FF01500E8
:109FC800F5E700BF8ABA0A005140070029289ABF5E
:109FD800014B185C09207047DEBA0A0070B5C368E7
:109FE8000F21B3F801601D78304603F077FA044674
:109FF80038B901213346BDE87040184A18486AF05C
:10A0080021B865B12846FFF7E1FF294602462046F8
:10A0180003F018FD2046BDE8704003F001B98378CD
:10A02800012B07D10AF03AF8204669F0C9FF002849
:10A0380008BF05252846FFF7C9FF294602462046DE
:10A0480003F000FD002DE5D00121064A044869F01F
:10A05800E5FF052120466AF022FCDBE7E04B0A0019
:10A06800105D0900D14F0A002DE9F041C6680F21A3
:10A07800B6F801703578384603F030FA044638B936
:10A0880001213B46BDE8F0411E4A1F4869F0DABF8E
:10A0980065B12846FFF79AFF29460246204603F095
:10A0A800D1FC2046BDE8F04103F0BAB8F278C37A93
:10A0B800934205D10221154A134869F0C3FFF0E71E
:10A0C8008378C272012B08D10AB109F0E7FF204654
:10A0D80069F076FF002808BF05252846FFF776FFB8
:10A0E80029460246204603F0ADFC002DD9D00121B7
:10A0F800074A054869F092FF052120466AF0CFFB20
:10A10800CFE700BFE04B0A00105D0900F74F0A00D7
:10A11800D14F0A00034B0146D3F8240182689268A4
:10A12800104700BF8001002008B50421034869F0EA
:10A138007EFFBDE8084002F065B900BF08020020B4
:10A1480008B5034869F067FFC0F3800008BD00BF89
:10A158000802002038B50546F7F74AF81C280446D7
:10A168001BD829460E48F7F731F8A0B122462946F0
:10A178000B488BF035F800220A482146031900F5F0
:10A18800947083F82821FFF7B7F820B10221064A16
:10A19800064869F043FF002038BD6FF00B00FBE76D
:10A1A800A80200208001002026500A00105D090046
:10A1B80000487047A8020020014BB3F846017047D9
:10A1C8008001002037B50F4DADF80600B5F84631CF
:10A1D800834203D10024204603B030BD02210DF193
:10A1E8000600FFF797F8044630B101210346064AF6
:10A1F800064869F027FFEEE7BDF80630A5F84631B6
:10A20800E8E700BF800100203B500A00105D09000C
:10A21800014902486FF0E3BA6C080020602D002065
:10A2280070B505460C4639B1CB684A699B1A032BB1
:10A238000ED86FF0150509E04FF0FF304FF0FF31F1
:10A24800FFF76EFE044618B96FF06805284670BD22
:10A258002046FBF7F1FD0C22164BA61802FB003333
:10A26800032130465D8068F0C7FB0580238A012101
:10A27800033B8370304668F0C7FB40F635439D4288
:10A288000FD12046FFF746FF05460028DED0012102
:10A298000346094A094869F0D5FE2046FBF76CFEDB
:10A2A800D4E7214606486FF08CF90025FFF7B0FF88
:10A2B800CCE700BF6C5100206C500A00105D09000B
:10A2C8008C0200202DE9F04786B0804691460C4666
:10A2D80000AF71B94FF0FF304FF0FF31FFF720FEAC
:10A2E800044660B96FF0680528461837BD46BDE8D2
:10A2F800F087887AFBF798FD3C4B83426FD10122A7
:10A30800002138466FF094F92046FBF795FD0C23A1
:10A31800DFF800A103FB00A08760204668F0E8FA98
:10A3280001464046FFF77CFF054618B12046FBF77B
:10A3380023FED9E7002338462D4A28F069F8064657
:10A3480090B140F2E3132B4A2B492C4866F070FE7B
:10A35800324641462A4866F06BFE85F31188BFF302
:10A368006F8F0323184602DF2046FBF765FD0C2399
:10A3780058431AF8006066B36D468AB06A46214BA6
:10A388000796CDE90538204B089340F20243ADF813
:10A3980024301E4B42F8103F00234FF432511C4822
:10A3A800F9F7FAFE2046AD46093EFBF7E5FD092E12
:10A3B8000CD8DFE806F0050B0B08170B0B0B0B147A
:10A3C8006FF06E0590E76FF00C058DE76FF00405F0
:10A3D8008AE7B9F1000FA9D0C9F8004084E76FF007
:10A3E800150581E76FF00B057EE700BFB41F00205D
:10A3F800B4C40400A34D0A008E500A00F04D0A00B0
:10A4080097500A00DC500A00377A0A00050000015C
:10A41800105D09006C51002073B506460D4642F2E6
:10A428002F00002101AAFFF74DFF044638B1012192
:10A43800144A154869F0F2FD204602B070BD019833
:10A44800C368B3F801203280B3F803302B80FBF7E0
:10A4580093FD3388A3F11B02E02A04D902210B4A99
:10A46800094869F0EFFD44F248112B88A3F5A4725E
:10A4780092B28A42E0D90221054A034869F0E2FD16
:10A48800DAE700BFFB500A00105D09001B510A0003
:10A4980040510A002DE9F04385B004460DF103014F
:10A4A800002001F01DF8054600287CD14FF0FF3050
:10A4B8004FF0FF31FFF734FD0746002877D000F151
:10A4C8000C080A21404668F063FA064605604560B4
:10A4D8000581384D023095F8DA3095F8DB209A423C
:10A4E80094BF04F1700104F17E0169F099FD9DF8B3
:10A4F80003307370AB6813F002091DD101231021DA
:10A508004046737268F044FAAA890280EA89428058
:10A51800B4F88C208280B4F88E20C280B4F89020E1
:10A528000281B4F8922080F80C90428180F80D9056
:10A5380080F80E9080F80F90AB68DB071CD5737A13
:10A54800102143F004034046737268F021FA2A8A06
:10A5580002806A8A4280B4F88C208280B4F88E2007
:10A56800C280B4F890200281B4F89220428100227F
:10A57800027342738273C2730F4B384601930723E9
:10A58800029301238DF80C30FBF756FC0C220B4B81
:10A59800394602FB003301AA5A6042F24300002206
:10A5A800FFF790FE0546284605B0BDE8F0836FF03A
:10A5B8006805F8E780010020080200206C5100209F
:10A5C8003C2870B5054644D002283ED100210246F9
:10A5D800084603F01BFB044680B901211D4A1E48AA
:10A5E80069F01CFD032001F057FF034688B3BDE85E
:10A5F80070400221194A184869F024BD043069F0F6
:10A608000AFDC30707D50321204602F055FE204660
:10A6180002F006FEE6E704F140006FF01EF910F0C4
:10A628000C0607D10E4A29460B4869F0F7FC31465B
:10A638002573E9E72046FFF72DFF0028E7D0012121
:10A64800084A054869F0EAFCE1E7BDE87040FFF711
:10A6580061B970BD63510A00105D0900064C0A001B
:10A6680081510A00A7510A0030B54FF0FF304FF072
:10A67800FF3185B0FFF754FC0446B0B10C4B002500
:10A68800019307238DF80C500293FBF7D5FB0C229E
:10A69800084B214602FB003301AA5A6042F20E0021
:10A6A8002A46FFF70FFE05B030BD6FF06800FAE7E5
:10A6B800080200206C5100202DE9F0478CB00026DC
:10A6C80005466F4BB0F80190198849F470429142E1
:10A6D80004BF1E806B4B00AF08BF1E7800F074FDEE
:10A6E800EB7805F10408012B08BF674B404614BFFF
:10A6F800002493F8224069F003FC4146002841D029
:10A7080007F1080069F0F1FBD5F81130C7F80130FE
:10A71800B5F81530A7F8053001233B70E878002814
:10A728003DD1022207F1080103F070FA0446EB78E4
:10A7380023B96FF08001554869F08BFC002C43D198
:10A7480007F1100541462846FEF798FB6E4688B08B
:10A758006A464F4BCDE905354FF40073ADF81C3010
:10A768004C4B42F8103F4FF4E2514B482346F9F75F
:10A7780013FD1321B546484669F0C0FC3037BD4685
:10A78800BDE8F087204669F055FE014607F108004C
:10A7980069F046FC4146384669F042FCBEE70128AC
:10A7A80010D1DFF8E4A006229AF8220007F1080188
:10A7B80003F02CFA04460028B9D1052237499AF843
:10A7C8002200B1E70024B2E7204640F2E242B5F8A1
:10A7D800013007F1080120F8703B69F021FCB5F859
:10A7E80017305343C4F88830B5F81930A4F89030BE
:10A7F800B5F81B30A4F892300023EA782373012AB5
:10A80800E2702BD1394604F1770069F009FCD5F8DC
:10A818000B30C4F87F30B5F80F3084F87E20A4F8E8
:10A8280083300721204602F047FD26B1012120464A
:10A83800267302F041FD204602F0B2FEE3784BB9E0
:10A84800032001F029FE034620B10221144A1248D0
:10A8580069F0F8FB204602F0E3FC8FE7002AE0D11C
:10A86800394604F17E0069F0DBFB217A064BC1EB27
:10A87800C101194404F1770069F0D2FBD1E700BFA8
:10A88800B8A500206CA80020800100200802002044
:10A89800C3510A0003000001105D090083BA0A00D1
:10A8A800064C0A0000B5C16889B0087820B109B023
:10A8B8005DF804EBFFF784BEB1F801308DF80000B5
:10A8C800ADF80130CB7801A88DF80330B1F80B3022
:10A8D8000431ADF81730B1F80930ADF81930B1F8D6
:10A8E8000B30ADF81B304B7B8DF81D3069F098FBB1
:10A8F800084B68461A689B88CDF80B20ADF80F30D6
:10A90800CDF81120ADF81530FFF7D6FE09B05DF887
:10A9180004FB00BF97BA0A0010B5F6F7D1FD034B48
:10A928001B6813B1BDE81040184710BD90510020B6
:10A938002DE9F341344D0646D5F824016EF045FC67
:10A9480050B90121314A324869F068FB6FF01204AE
:10A95800204602B0BDE8F0816FF0020105F18800E1
:10A9680069F077FB012169F062FBC30748D4FEF761
:10A97800F1FB04460028EBD1264B1E60012205F1AD
:10A98800E80011466EF054FE234F05F586706EF010
:10A99800DAFD38466EF04EFF38466FF007034FF485
:10A9A80000621E49009427F02BFFD7F8E0001C49ED
:10A9B8006EF0A5FFD5F824010769D7F80080B8F133
:10A9C800000F15D1174B3B6083681B6898470446F6
:10A9D80028B986B902B0BDE8F041F6F771BDC7F8ED
:10A9E800008001212346104A094869F02BFBAFE794
:10A9F8006FF07704F5E705F1780027F0FBFEA7E78D
:10AA08006FF07704A4E700BF800100203F530A00DD
:10AA1800105D090090510020602E002040CB0020DE
:10AA280057530A00AD99000060530A00F0B5C56895
:10AA380001212F8887B0BCB2204602F04FFD0646A0
:10AA480040B901212346274A274807B0BDE8F0400E
:10AA580069F0F8BA02ACD5F80220D5F806300194AE
:10AA6800698900916BF0E3FD48B34FF0FF304FF078
:10AA7800FF31FFF755FA054648B901211B4A1A4824
:10AA880069F0CCFA304602F0CBFB07B0F0BD1221DA
:10AA98000C3067F07DFF0346224623F8027B1446FC
:10AAA80003CC596006A98C421860224603F10803BA
:10AAB800F5D1294642F21A00FFF7B2FBE2E74FF060
:10AAC800FF304FF0FF31FFF72BFA04460028D4D0AF
:10AAD80002210C3067F05CFF2146078042F21B0020
:10AAE800EAE700BF2C4C0A00105D09007C530A00FD
:10AAF80073B5C368D9789A781E8842EA0122ADF8FE
:10AB0800002059791A79B4B242EA0122ADF802203C
:10AB1800D9799A79204642EA0122ADF804201A7AB6
:10AB28005B7A012142EA0323ADF8063002F0D6FC35
:10AB3800054658B901211D4823461D4A69F082FA85
:10AB48000221204669F061FB02B070BD694602F03F
:10AB58000DFF38B91E21204669F057FB284602F040
:10AB68005FFBF1E74FF0FF304FF0FF31FFF7D8F907
:10AB780004460028F2D00E210C3067F009FF0023AC
:10AB88000680C0F80A30BDF8003021464380BDF881
:10AB980002308380BDF80430C380BDF806300381DD
:10ABA80042F22000FFF73CFBD8E700BF105D090028
:10ABB8002C4C0A0038B5042104460C3067F035FFE8
:10ABC800034640885D7818B122461978FFF76EF879
:10ABD80035B1044827F0E0FBBDE83840FFF718BB63
:10ABE80038BD00BF68020020B0B50446032100AF9D
:10ABF8000C3067F01AFFE2680346117840F63542D8
:10AC0800B0F80100904217D16C468AB06A46114BE1
:10AC1800CDE90531104B079340F20133ADF82030F0
:10AC28000E4B42F8103F00234FF412510C48F9F72D
:10AC3800B3FAA546BD46B0BD1D7810B12246FFF750
:10AC480035F8002DF6D0074827F0A6FBFFF7E0FA05
:10AC5800F0E700BF93530A00377A0A0004000001A6
:10AC6800105D09006802002038B528F017FA314D48
:10AC7800D5F80C31002B5AD00022002305F1E8004A
:10AC880027F0C6FB002852D10022002305F5867064
:10AC980027F04CFB044668B940F6CC43264A2749BE
:10ACA800274866F0C5F984F31188BFF36F8F032333
:10ACB800184602DFD5F800317BB1224A012122482B
:10ACC80069F0ACF90022214BD3E8EF0FC3E8E12F7C
:10ACD8000029F9D108B1FBF74FF9204667F008FEC3
:10ACE800C5F800012046FFF715FA0346C8B101214F
:10ACF800174A154869F0A6F9164827F04DFB204673
:10AD0800FBF79AF80C22144B02FB0033588818B151
:10AD180022461F21FEF7CAFF2046FBF72DF9FFF751
:10AD280077FAFFF775FABDE8384028F0CBB902F09A
:10AD380047FCF8E780010020A34D0A00AC4B0A004D
:10AD4800F04D0A00CB530A00105D09008002002074
:10AD58006C500A00680200206C51002070B54FF05A
:10AD6800FF320D464FF0FF3300210646FEF7A8FBE1
:10AD7800044660B91A230A4A0A490B4866F058F98A
:10AD880084F31188BFF36F8F0323184602DF022173
:10AD980004F10C0067F0FCFD06704570204670BD9C
:10ADA80033540A00AC4B0A00F04D0A00F8B50646C9
:10ADB8000024094DEF79E3B29F4202D86FF00100F9
:10ADC80007E02946304669F06AFA0735631C08B17E
:10ADD8002046F8BD1C46EEE78001002037B5044642
:10ADE8000D46B9B12846164969F059FA90B929466D
:10ADF8001448C4EBC404204469F04AFA124869F0C4
:10AE080044FA430703D5FEF793FA69F011F80020D6
:10AE180003B030BD684669F05AF80028F8D1684692
:10AE2800FFF7C4FF0028F5DA064BC4EBC4006946F7
:10AE3800184469F02DFA002DE0D001462846DBE7DA
:10AE48008ABA0A00800100200802002070B5174E57
:10AE58000622314605468AF0F1F910B34FF0FF306B
:10AE68004FF0FF31FFF75CF80446E0B106222946AF
:10AE78000C3067F093FD2146002242F20500FFF7EF
:10AE880021FA044648B110F10D0F04D10221084AF5
:10AE9800084869F00CFA204670BD28683060AB8815
:10AEA800B3800024F7E76FF06804F4E79C01002002
:10AEB80069540A00205D0900064BD3E8EFCF4CF433
:10AEC800806CC3E8E2CF002AF7D1037A19430172F4
:10AED800704700BF080200202DE9F3410021044615
:10AEE8000222084602F092FE054648B1204601219A
:10AEF800FFF7E2FF284602B0BDE8F04102F090B942
:10AF08008DF8000069464E4800F0ACFE9DF8003010
:10AF180033B101212046FFF7CFFF02B0BDE8F08131
:10AF2800484869F0B2F98106C0F3401708D545488A
:10AF380069F0ABF9420603D501212046FFF7BCFFB3
:10AF48000021414800F08EFE17B1002001F070FA90
:10AF58003E4D95F8DB309BB1002069F0E7F978B1F8
:10AF680002213B4A3B4869F0A2F917B1012001F0E0
:10AF78005FFA0021384802B0BDE8F04100F072BE27
:10AF880095F8DB2095F8DA309A4218D10221334A35
:10AF9800304869F08CF9002242F229001146FFF787
:10AFA80091F910B101212E4ADCE795F8DB30013325
:10AFB80085F8DB30237A43F004032372D5E7224671
:10AFC80004F10108414612F82E0B69F072F90646A1
:10AFD80010B1244A01210EE095F8DB30013385F8E1
:10AFE800DB30237A43F00403237295F85B305B0768
:10AFF80008D402211C4A174869F059F9012069F060
:10B0080095F9B2E74146684669F042F901234FF0E5
:10B01800FF304FF0FF318DF80730FEF781FF04460F
:10B0280060B1082269460C3067F0B8FC3246214608
:10B0380042F24E00FFF746F90028DFD00B4AC9E775
:10B048001D44070008020020ED430700800100208E
:10B0580078540A00205D0900674307009D540A00E0
:10B06800CE540A00EE540A000E550A0038550A005C
:10B078002DE9F743002104460222084602F0C6FDE6
:10B08800054648B120460221FFF716FF284603B0BF
:10B09800BDE8F04302F0C4B88DF807000DF10701D0
:10B0A800404800F0DFFD9DF8073033B1022120460B
:10B0B800FFF702FF03B0BDE8F0833B4869F0E5F80D
:10B0C8008206C0F3401808D5374869F0DEF8430611
:10B0D80003D502212046FFF7EFFE0021334800F098
:10B0E800C1FDB8F1000F02D0002001F0A1F9002045
:10B0F80069F01CF92E4D0646C0B1012103462D4AC0
:10B108002D4867F02DF895F8DB3013B1012069F070
:10B118000DF9B8F1000F02D0012001F089F90021E2
:10B12800264803B0BDE8F04300F09CBD95F8DB303D
:10B1380095F8DA209A420CD2013B85F8DB30237A65
:10B14800024623F0040302201D49237209F0DCF8AB
:10B15800D9E74FF0FF304FF0FF31FEF7E1FE04F181
:10B168000109074668B107210C3067F011FC494610
:10B1780069F08EF83246394642F22800FFF7A2F805
:10B1880028B101210F4A0C4869F091F8BBE795F8FE
:10B19800DB30013B85F8DB30237A23F0040323728C
:10B1A800B1E700BF1D44070008020020ED43070077
:10B1B8008001002053550A00205D090067430700FD
:10B1C8001F43070080550A00084BD3E8EF2F22F4ED
:10B1D8008061C3E8E01F0028F7D1530504D5002299
:10B1E8000220034909F090B8704700BF0802002008
:10B1F80065450700002307B50549CDE900036A4600
:10B20800022009F081F8019803B05DF804FB00BF43
:10B2180091430700034610B470B10B4991F8DA4026
:10B2280091F8DB200CB1944209D2013281F8DB207D
:10B238001A7A42F004021A725DF8044B70475DF8FE
:10B24800044BFFF749BE00BF80010020034610B43D
:10B25800A0B10C4C94F8DA1094F8DB2031B101312C
:10B268008A4204DC5DF8044BFFF702BF12B1013AD1
:10B2780084F8DB201A7A22F004021A725DF8044B73
:10B28800704700BF8001002038B50D460649CC79CB
:10B2980038B12B689C4228BF1C46C4EBC40289F015
:10B2A8009FFF2C6038BD00BF8001002070B50446A8
:10B2B80011BB20B3254968F0F2FF00BB2046FFF719
:10B2C80075FD00283BDA237853B92148C279002A52
:10B2D80035D1214668F0DCFF0123C371104670BDEB
:10B2E800012B04D1A37903F0C003C02B07D001219F
:10B2F800184A194868F0DBFF6FF01500EFE7144DA6
:10B30800EB79012B1ED005F1880068F0BEFFC3075A
:10B3180007D4002CF0D020460C4968F0C0FF002864
:10B32800EAD1EE792146731C3046EB71FFF756FDE2
:10B3380008B93046D3E7EB79013BEB71CFE76FF003
:10B348007700CCE76FF00B00C9E700BF8ABA0A00A4
:10B3580080010020A5550A00205D09002DE9F34170
:10B36800044640B91A4A02211A4868F0A0FF002092
:10B3780002B0BDE8F081002141F2090001AAFEF700
:10B38800A1FF054608B1144AEDE7019E0622D6F84A
:10B398000C80124908F10107384689F04FFF28B19F
:10B3A800062238460E4989F049FF18B93046FAF79F
:10B3B800E3FDDCE7D8F801303046C4F80130BB883B
:10B3C8002570A4F80530FAF7D7FD0120D0E700BFB3
:10B3D800D3550A00205D0900EC550A0097BA0A0007
:10B3E80091BA0A0007B56846FFF7B8FF044BD87151
:10B3F80018B169460020FFF7F1FC03B05DF804FBC3
:10B40800800100202DE9F041304E88B0F179002903
:10B4180054D196F8764014F0010411D12C4A022137
:10B428002C4868F044FF0024F471162500240127F5
:10B43800F379E0B283422BD8002B3FD000203AE0CA
:10B448006A464FF60940FEF73DFF08B1224AE6E793
:10B45800DDF800C0DCF80C5095F80180B8F1000F59
:10B468000ED0AB1C02AA1235174618685968083363
:10B4780003C7AB423A46F7D1186838609B88BB804F
:10B488006046FAF779FDB8F1000FCDD1134AC6E747
:10B4980008AB05FB003353F8182C33F8143C694605
:10B4A800CDF80120ADF805308DF80070FFF796FC57
:10B4B80001340028BCD008B0BDE8F081002108465E
:10B4C80008B0BDE8F041FFF7F1BE00BF80010020E1
:10B4D8000A560A00205D090036560A0056560A0028
:10B4E80038B50C4661B108480578012D05D1013001
:10B4F800FFF7ACFC00B9257038BD00200870FBE7E9
:10B508006FF01500F8E700BF800100202DE9F04139
:10B518001D460E461746034648B145B10A0311D5E4
:10B528004C0708D50121284A284868F0C0FE6FF06A
:10B538001500BDE8F08168F0EEFF0028F9D101237D
:10B548002B70F6E7B107047824D021492FB1B20651
:10B5580003D591F89020500632D5C4EBC40411F8F5
:10B568000480B8F1010F09D101341846214468F06C
:10B578006DFF0028DDD185F8008002E0B8F1000FEA
:10B58800F9D02FB1B30642BF2B7843F002032B70DA
:10B598000020CEE7720710D50D49C4EBC4040F5D37
:10B5A800012F07D10134214468F050FF0028C0D191
:10B5B8002F70E7E7002FE5D1FAE768F0ACFFBEE7A8
:10B5C8006FF08500B5E700BF7F560A00205D0900CF
:10B5D8008001002070B500F10F0604460D460722D1
:10B5E80030460C4989F02AFE0346207873B90522B3
:10B5F800094902F00BFB044658B10573002101F01C
:10B608005BFE2046BDE8704001F00ABE06223146C6
:10B61800EFE770BD8ABA0A0083BA0A00F8B5046970
:10B628000646456844B140F203432B4039D005F43F
:10B638008263B3F5806F34D015F4806302D115F4BA
:10B64800F84F2ED1184F3078FB79834229D9C0EBB7
:10B65800C00007221549384489F0F0FDA8B115F05B
:10B66800030306D197F82320082A02D8B2689F2A34
:10B6780017D915F0300F09D09CB1EB0608D405F4A2
:10B688006035B5F5603018BF0120F8BD002CF6D143
:10B69800D6E902239A4204D81F2A02D9B3F1807F3F
:10B6A800EDD30020F1E700BF800100208ABA0A002C
:10B6B80038B50E4D284668F070FF10F0010412D11D
:10B6C800A5F1180318465822214689F0AFFD034614
:10B6D800D5E8EF2F42F00102C5E8E12F0029F7D1A4
:10B6E80018465C7038BD0020FCE700BF782F0020AA
:10B6F800F8B5044614F80F7B154B06460D4607228D
:10B708002046144983F8227089F098FD70B93846AC
:10B71800114902F0CDF9044610B96FF00B00F8BDDD
:10B72800052101F0C9FD00202C60F8E721463846C4
:10B7380002F004FA40B92146307802F0B9F904461B
:10B748000028EAD00621ECE76FF01500E7E700BF14
:10B75800800100208ABA0A0083BA0A002DE9F04F56
:10B7680091B0154603905068002214460691824213
:10B7780012D1FB2C18D89F4BB3F8D8309C421ED955
:10B788009D480093022123469C4A66F0F3FC6FF023
:10B79800200011B0BDE8F08F2968023401EBC20126
:10B7A8004B7801321C44E2E7039B082103F118009F
:10B7B80068F0F6FE0028DED06FF00A00E9E7FB2CFF
:10B7C8006ED8039B0B2103F1180068F0E9FE10B94D
:10B7D8001F2C28BF1F244FF0FF304FF0FF31FEF71A
:10B7E8009FFB04F104080746002800F0FF8041464B
:10B7F8000C3067F0CDF84FF00009064642460021AC
:10B8080089F014FD4946D5F8008006F1040B6B68F1
:10B8180099450FD3039BF1705B78002233700323A3
:10B828003946737001230698B37011B0BDE8F04F24
:10B83800FEF748BD98F80120881C13189C4298F818
:10B8480000C013D2BCF1090FA4EB000201D1002AF9
:10B858000ADC694801216A4A66F079FC3846FAF739
:10B868008BFB6FF0150094E74FF0080C5FFA82FA33
:10B878000AF101030BF801300131C9B20BF801C01C
:10B88800C3B2D8F804105844049389F0A9FC049B67
:10B8980009F101099A445FFA8AF108F10808B6E744
:10B8A800002110220CA889F0C1FC0027012340F2D6
:10B8B80072600B933B4669680A958B4207D1002456
:10B8C8000123A046A34605935FB9384661E72A6875
:10B8D800023702EBC302527817448742C1D80133BA
:10B8E800EBE7FB2F4FF0FF304FF0FF31BA4628BF90
:10B8F8004FF0FB0AFEF714FB0AF104060490002837
:10B9080074D031460C3067F043F8039B81465B786E
:10B91800002603704FF000035FFA8AF283700792E3
:10B92800031D55F83B2005EBCB0102EBC80252780A
:10B938000232944209D14A6808F10108904509BFCA
:10B9480000240024A0460BF1010BBBF1010F12D01B
:10B9580055F83B204FEAC80112EBC80C0BD09819D8
:10B96800FCB901249CF8012001329A550136F6B23F
:10B97800079AB242D5D8059BBF1B002B31D0002FA8
:10B988000CBF0323012300220499069889F8036059
:10B9980089F80130FEF796FC00287FF4FAAE05908E
:10B9A80092E7012C05D1525C013602240270F6B2EE
:10B9B800DEE79CF80120AAEB0601121B02328A423C
:10B9C80028BF0A46DCF804C0A11E61440993089206
:10B9D80089F006FC089A099B14443244A4B2D6B2F2
:10B9E800C6E7B7FA87F35B095B00CCE76FF068003E
:10B9F800CFE600BF80010020A85C0900A4560A0019
:10BA0800D2560A002DE9F3470F690D46496890465A
:10BA18003A1E18BF01224C020646016505D5EB788F
:10BA28007F33DBB2932B00F2048130460DF1030320
:10BA3800FFF76CFD0446002840F0E88006F10F038C
:10BA4800002F00F0E7802A6911684FF0FF30C6F830
:10BA58000F109188998092794FF0FF319A71FEF713
:10BA68005FFA8146002800F0E78019210C3066F063
:10BA78008FFF04460021192289F0D8FB73782370C0
:10BA8800AB68E370C3F307221B0C22716371EB6888
:10BA9800A371C3F307221B0C2372E2716A6812F4C4
:10BAA800004F14BF06230723D00348BF03F0050344
:10BAB800910348BF03F0FB0363729DF80330A37240
:10BAC8006B685A0254BF7F2395F90330E37401234E
:10BAD80023756B6803F44063B3F5806F14BF0123CB
:10BAE8000223A3756B68DB0442BF03232375A37588
:10BAF8006A68C2F3802383F001031B0150049BB2E0
:10BB080048BF43F04003910448BF43F02003D205E7
:10BB180044BF012222766A6890077DD043F0010A6B
:10BB28001FB9510501D443F0030A900502D4B8F1B6
:10BB3800000F03D04AF0020A1FFA8AFA002F6DD0CC
:10BB4800D1062A6948BF4AF00403116858BF4AF071
:10BB58000C03C4F80B1091889BB2A4F80F109279CB
:10BB680062746A7801AFE275AA7849466275A4F8EA
:10BB780001303A4642F23600FEF7A4FB044600289C
:10BB880044D1019BDB6893F90130B370D7E8EF0F1C
:10BB9800C7E8E34F002BF9D108B1FAF7EDF906F140
:10BBA8001807D7E8EF3F43F00203C7E8E23F002A4F
:10BBB800F7D16FF01001384668F0F9FCC2062FD4AF
:10BBC8006A68092112F0030218BF0122384668F09A
:10BBD800F9FC0A213846CAF3400268F0F3FC2A79D6
:10BBE8000C213846C2F3800268F0ECFC6A790B211C
:10BBF8003846C2F3800268F0E5FC9DF80320032173
:10BC0800531E5A4238465A4168F0DCFC204602B0BE
:10BC1800BDE8F0870A4A17E79A4686E75346A0E741
:10BC2800304606F1090168F011FC0028C8D0044626
:10BC3800ECE76FF01504E9E76FF06804E6E700BF8A
:10BC48008ABA0A0008B520B9044868F0A6FCC307F8
:10BC580001D4002008BD0248FCE700BF782F00206F
:10BC6800602F0020034610B5044868F096FCC20710
:10BC780003D5BDE810400248184710BD782F0020B2
:10BC8800602F002010B5054CA06930B16FF001019C
:10BC9800183068F08CFC0023A36110BD80010020DF
:10BCA80010B5164B9C693CB90121154A154866F038
:10BCB8004EFA0024204610BD204668F009FD04F124
:10BCC80018020821104668F06BFC10B9FFF7DAFF7C
:10BCD800EFE70921104668F063FC18B100212046FF
:10BCE800FFF778FC00222046114668F0ACFC0446B9
:10BCF8000028DFD1FFF7C6FFDCE700BF8001002086
:10BD0800EB560A00A85C090010B50A4B20389B695D
:10BD180083420AD1FFF7C4FF034648B1BDE810408B
:10BD28000221054A054866F01BBA68F0D4FCF3E71F
:10BD380010BD00BF8001002022570A00A85C09003E
:10BD48002DE9F04FDFF888B10646DBF818400F46BA
:10BD58009046994685B0002C40F09E80FFF7A8FCDD
:10BD68000546CBF81800002800F099800BF18800F0
:10BD7800D6F810A0ADF808408DF80A40039468F092
:10BD88000CFC410774D573685A0574D432690AB13A
:10BD98009B0770D03046FFF741FC00286BD005F1B7
:10BDA800180B0821584668F0FBFB002866D1434869
:10BDB80068F0F3FB440501D5FFF706FA3378B9F1CB
:10BDC800000218BF0122314628462B70FFF71AFEE1
:10BDD800044660B9BAF1000F0CD10E9B424600939D
:10BDE80039464B46284668F0A1FC044680B1FFF767
:10BDF80049FF33E07368D8060AD48023ADF80830C9
:10BE0800DBE8EF3F43F08003CBE8E23F002AF7D1BD
:10BE18007368990716D10121284602AA68F013FC15
:10BE28000446B8B10121264A264866F090F9039ED7
:10BE3800002EDCD03046002101F03EFA304601F0F9
:10BE4800EFF9D4E7284603A9FFF752FC0446002877
:10BE5800E1D0CCE7039808B101F0E2F939460023B4
:10BE680040F2011098450CD1204605B0BDE8F08F8E
:10BE78006FF00A04BBE76FF01504B8E76FF07704BA
:10BE8800B5E70A88824204D14A6812B11278D2070B
:10BE980008D401330831E5E76FF07704E4E76FF081
:10BEA8000B04E1E72035284607496DF0CAFC00235A
:10BEB8002846064A26F046FDD6E700BF08020020BD
:10BEC80007570A00A85C090011BD00001C4E0E00AF
:10BED800800100202DE9F341C6687078FFF7B2FEB3
:10BEE800044638B90121364A364802B0BDE8F04167
:10BEF80066F02DB904F11808758868F0E9FB6FF44D
:10BF08008071404668F053FB33782F4F1BBB28469F
:10BF1800012101F0E3FA054650BB6FF0800140466D
:10BF280068F045FB03060ED5204668F00DFBFFF7C9
:10BF38004BF963683BB11B682BB1327920468DF809
:10BF4800042001A99847BB699C4235D102B0BDE8DD
:10BF5800F041FFF797BE0921404668F021FB18B170
:10BF680020463178FFF736FB3378002BD5D1CEE762
:10BF7800236D00F17E0213F4002F12D0A368C0F8DD
:10BF88007E30A3899380A37B937163682BB15B6830
:10BF98001BB12046019501A99847284601F040F9B0
:10BFA800BBE7037AC3EBC303F918FB58C0F87E302C
:10BFB8008B8893808B79E7E702B0BDE8F08100BFFA
:10BFC80041570A00A85C0900800100207FB5C568B8
:10BFD8002878FFF737FE044638B90121134A144878
:10BFE80004B0BDE8704066F0B2B843688BB19B6896
:10BFF8007BB10135284667F083FF02AE294650B170
:10C00800304667F072FF636820469B68019601A975
:10C01800984704B070BD207868F00CFA03460068B1
:10C0280002909A889B79B280B371ECE741570A0075
:10C03800A85C0900034B1A7A012A04BF02221A726B
:10C04800704700BF6DA8002008B509486DF007FCCF
:10C05800031E04DA0121074A074866F081F8002226
:10C06800064B99689A801960054B1A7208BD00BF83
:10C07800C802002055570A00405D09008C080020BE
:10C088006DA80020F0B505460F464FF0FF304FF081
:10C09800FF3187B01646FDF743FF0446C0B10621BD
:10C0A8000C3066F075FC46800026477005700671F6
:10C0B8004671094A204603A905230095FDF71EFF8E
:10C0C8003246214642F24200FEF7FCF807B0F0BDC6
:10C0D8006FF06800FAE700BF0802002038B505468F
:10C0E800407A0C46FDF744FF2073A87AFDF740FF1D
:10C0F800607395F90C30A37195F90D306371EB7A83
:10C108002371EB8963812B88103BDBB20B2B8EBF2D
:10C118000523054AD35CE3712B8883F0100303F0F1
:10C128001F03238138BD00BF0BBB0A0008B50C4BA9
:10C138000246400903EB800068F024FB02F01F036D
:10C1480040FA03F313F0010006D122B9054868F05C
:10C1580019FB40F3C01008BD6FF07700FBE700BF84
:10C1680094510020080200202DE9F04788B00022F1
:10C1780000238E4826F018F80646002840F0CB80A9
:10C188008B4868F0FFFA10F0010F894D7ED02B1D07
:10C1980093E8070008AB03E90700864868F0F2FA5D
:10C1A800C0F34013824868F0EDFA0446002800F016
:10C1B800A3808BB10C22804905A889F03FF804467A
:10C1C800002800F0A480002211461046FFF75AFF0D
:10C1D8000446002840F09B80764868F0D3FA410571
:10C1E80001D5FEF7F1FF9DF815502A0757BF9DF8B6
:10C1F800143000278DF80430BDF816305FBF01AF4A
:10C20800ADF80530BDF81830ADF8073015F0040565
:10C2180000F0C880BDF81C200AB9BDF81620BDF88A
:10C228001E300BB9BDF818309DF81410ADF80D206C
:10C238008DF80C10ADF80F3003AD002F6FD03B78A0
:10C24800012B71D0002D6AD10025BDF81A3006F0F7
:10C25800010043B1574BD3E8EF1F41F04001C3E859
:10C26800E21F002AF7D10DF1030168F087F90446AF
:10C2780000284CD14FF0FF304FF0FF31FDF750FE52
:10C288008046002852D16FF0680440E0494868F0C1
:10C2980079FA10F0800F494A0ED09089D189136934
:10C2A8004FF48072ADF81600ADF81420ADF81810F0
:10C2B800ADF81A60079370E7414C05AB20686168D8
:10C2C80003C3A068186092F8913039481F0744BF2B
:10C2D80005238DF8153068F055FA840706D5302304
:10C2E800ADF818306023ADF8163056E7304868F0DE
:10C2F80049FA4007F3D450E74BB102460146FFF72D
:10C30800C1FE044618B92C4B2861C3E9010027482F
:10C3180025F0BCFF2646304608B0BDE8F0872E78E9
:10C32800731E5E425E4190E71E468EE700F10C09DF
:10C338000321484666F02CFB9DF803309DF815A0B4
:10C348000370CAF3400306468470437037B1012373
:10C35800052283703946484666F020FB45B1B3781C
:10C36800052243F0040329464846B37066F016FBDD
:10C378000022414642F24100FDF7A4FF044600288E
:10C38800C5D10120BDF81A200AF00101FFF77AFE95
:10C3980004460028BBD1084B08AA12E9070083E825
:10C3A8000700B4E7002F7FF44AAF4DE7B0510020F3
:10C3B8009451002008020020A45100208001002090
:10C3C800905F0900002347F6122210B5064826F0B0
:10C3D800B9FA031E06DABDE810400121034A0448F1
:10C3E80065F0BEBE10BD00BFC802002082570A001B
:10C3F800405D09000022024B1A60FFF725BE00BF0E
:10C40800E051002010B544220021084888F00EFFB2
:10C41800064B03F11C001C466DF016F804F13000C1
:10C428006DF012F8BDE81040FFF7E4BF945100200A
:10C438000022044B801A597C18BF012001F0010129
:10C44800FFF720BE94510020032870B5054603D19C
:10C45800BDE87040FFF788BEFFF768FE0446B0B934
:10C46800012605F01F039E400A4B6D0903EB850565
:10C47800D5E8EF3F3343C5E8E23F002AF8D1FFF79C
:10C4880073FE044618B1F143284668F07EF9204649
:10C4980070BD00BF94510020032808B50AD00121BF
:10C4A80000F01F039940054B4009C94303EB800086
:10C4B80068F06BF9BDE80840FFF756BE94510020BC
:10C4C8002DE9F74F05465E4868F05CF900F0010871
:10C4D8005B4868F057F90E46144699468246B8F10B
:10C4E800000F03D00B895A0700F1A680284667F091
:10C4F80007FD6F46002868D02946684667F0F5FCB6
:10C50800B8F1000F02D11AF0040F28D14D4BD3F81F
:10C5180000B0BBF1000F13D02268A368B4F804A0E0
:10C52800A4F80490A2EB030838462346F27996F95A
:10C538000510D847A368A4F804A013FA88F3236069
:10C54800414B37601A6842B152F80889B8F1000FB8
:10C5580001D0A8F10808002A47D1002333603848E1
:10C56800338968F00FF910F0010665D1DB0763D550
:10C5780003223946304601F049FB044600285BD0C7
:10C588000220FFF789FF2B682046C4F87E30AB886D
:10C59800A4F88230AB7984F8843067F0ADFD0028C8
:10C5A80043D01F2331462373204600F085FE2046E2
:10C5B80000F036FEFFF7D8FD034600283CD00221E4
:10C5C800224A234865F0CCFD36E02B78FF2B07D1B3
:10C5D800204B186800909A889B79BA80BB718FE7C6
:10C5E800294667F027FF0346F3E713688BB12168F4
:10C5F800A368B4F804B0A4F80490A1EB030A304689
:10C60800136821469847A368A4F804B013FA8AF37C
:10C618002360B8F1000F06D0D8F8083003B1083B02
:10C628004246984697E74346FAE72046022100F03B
:10C6380043FE204600F0F4FD03B0BDE8F08F00BFD4
:10C6480094510020E0510020D8510020064C0A00E7
:10C65800405D09008ABA0A0010B50020FFF71CFFE8
:10C6680058B16DF070F90020FFF716FF034620B1AE
:10C678000221124A124865F073FD6FF0400111481B
:10C6880068F083F86FF480710E4868F07EF8FEF762
:10C698009BFD0D4B1B6823B153F8084904B1083CB6
:10C6A80003B910BD5B6803B198472CB1A26802B109
:10C6B800083A23461446F3E72246FAE7B3570A0036
:10C6C800405D090008020020D85100202DE9F04FF4
:10C6D80000F10C0989B00746484666F0AEF90646EF
:10C6E8005D4868F04FF800F001035B48039368F079
:10C6F80049F85A4DC0F38003DFF874A102939EB144
:10C70800039B53B13B8A172B11D80121544A554832
:10C7180009B0BDE8F04F65F01ABD2B7A0BB1FFF7F1
:10C7280093FC029B002BEDD109B0BDE8F08F1821D6
:10C73800484666F07AF93A8AC37DB0F800B0934269
:10C74800CBF3411804460BF0100B0FD94548009263
:10C758000221454A65F00EFD384666F082F8BBF1C5
:10C76800000FE1D102223D4B1A72DDE7BBF1000F49
:10C778000DD004A9FFF7B2FC4A46E37D04A9A01C2A
:10C78800FFF79EFE4846E17D66F047F929E095F8F7
:10C7980008B0BBF1000F37D0C27AEB799A4205D1C5
:10C7A800811C0722284688F049FD48B3B8F1000FDC
:10C7B80002D1204604A9DDE7BBF1010F27D10221F0
:10C7C8002A4A284865F0C3FCDCE72B7A022B3DD0C7
:10C7D8005046F96866F0E2F8B8F1010F04D1FFF7A6
:10C7E800F1FD013EF6B28AE7204604A9FFF776FC80
:10C7F8005246BAF8043004A9A01CFFF761FE28E0ED
:10C80800B8F1020F18D124E0B8F1000FD1D0B8F177
:10C81800020F1ED0BBF1020F01D1FFF715FCD4F8AF
:10C828000220E37A2A60E288EB710123AA80227A47
:10C838002B72AA71FFF7C6FDE27DBAF80430BAF888
:10C84800061013448B42C0DD02232B72B8F1010F8E
:10C8580098D0FFF7F9FB95E7945100206DA80020C8
:10C86800DC570A00405D0900F5570A001F580A0006
:10C878008C0800202DE9F04F00F10C0785B0064622
:10C88800384666F0DAF805462A4867F07BFF00F07C
:10C898000109284867F076FF4FF0010ADFF8A0B0D9
:10C8A800C0F3800815B905B0BDE8F08FB9F1000FE5
:10C8B80002D1B8F1000FF6D0338A082B07D801212E
:10C8C8001D4A1E4805B0BDE8F04F65F040BC09217F
:10C8D800384666F0AAF8037A328A01339A42044647
:10C8E800EDD37F23ADF80CA08DF80630037A6946A6
:10C8F80003445B7A01308DF80530FF238DF804304E
:10C908000023ADF80A3010F8012C013D042A98BF25
:10C918001BF802308DF80720ADF80830C3793A4685
:10C92800FFF7CEFD217A3846013166F076F8EDB290
:10C93800B8E700BF94510020DC570A00405D0900A9
:10C9480017BB0A00F8B50546224867F01BFF4307E6
:10C958000F463CD52A78012A03D96FF015042046E2
:10C96800F8BD6B780F2BF8D843F6FC746888031F62
:10C978009BB2A342F1D8A9880B1F9BB2A342ECD863
:10C988008842EAD37AB900220023134825F00CFC28
:10C9980004460028E3D1FFF7C9FB044640B10E481E
:10C9A80025F074FCDBE767F0CDFD0028EBD1D4E778
:10C9B80028686968094E0A4B03C6A8681F6030607A
:10C9C8002046FFF741FD044606F12400E8E76FF032
:10C9D8000A04C4E708020020C4510020985100202E
:10C9E800E051002008B5FFF705FD00220A4B6FF063
:10C9F80040010A481A6067F0C8FE430606D56FF47E
:10CA08008071064867F0C1FEFEF7DEFBBDE808400E
:10CA18000020FFF741BD00BFE051002008020020C0
:10CA28000A4A00F10803116831B98160516839B9BF
:10CA3800C2E90033002070478B4204D00968F3E74D
:10CA48000B605360F6E76FF010007047D851002074
:10CA580008B5034867F096FE00F0010008BD00BF66
:10CA68009451002070B59AB01422002104A888F0CF
:10CA7800DDFB47F21213ADF80C304FF4807344F22B
:10CA88000102ADF80E30364B01A903A8CDE9052304
:10CA98005DF016FC034618B3324A0121324865F0AE
:10CAA8005FFB1F25314BD3E8EF1F21F00101C3E8DD
:10CAB800E21F002AF7D12E4E26F0F0FA346804B1AE
:10CAC800043C002D2B4D18BF0025002C41D02368B5
:10CAD8000BB1284698476468002C3AD0043CF6E726
:10CAE80002AB4122019809A987F036FA034608B13A
:10CAF800214AD2E7214A0DF125030DF1650153F8CA
:10CB0800040B8B4242F8040BF9D102AB20221C49DA
:10CB1800019887F0C9F9034608B11A4ABDE7019898
:10CB280087F07AF9054610B1174A0346B5E7134965
:10CB3800104867F035FE1548203167F031FE144B78
:10CB4800D3E8EF1F41F01001C3E8E21F002AA9D083
:10CB5800F6E70023C6E9003326F0B4FA1AB070BD30
:10CB68000000020944590A00005D0900E451002050
:10CB7800EC510020BBA9002062590A007BA90020C3
:10CB88005BA9002085590A00A9590A00DBA90020E1
:10CB98000802002030B5A7B01422002108A888F0A8
:10CBA80045FB04233D22002116A8159388F03EFB7F
:10CBB80047F21213ADF81C304FF4807344F20102AF
:10CBC800ADF81E30284B2949CDE9092307A805AB44
:10CBD800202287F0EBF90346E0B1254A01212548D8
:10CBE80065F0BEFA6FF0040426F058FA224B1D686F
:10CBF80065B100201860214BD3E8EF1F21F0020136
:10CC0800C3E8E21F002AF7D144B3A84726F05AFA2E
:10CC180027B030BD1A4B0DF15502194603F14000FB
:10CC280053F8044B834242F8044BF9D106AB029304
:10CC380020230D48CDE9001315AA4123059987F053
:10CC480088FB034608B10F4AC8E7059887F0E4F85F
:10CC580004460028C8D00C4A0346BFE70DA8084977
:10CC680067F09EFD0DA8D0E7000002095BA900202F
:10CC7800C9590A00005D0900E8510020E45100206C
:10CC88007BA90020FF590A001B5A0A00402208B558
:10CC9800034988F0D3FAB0FA80F0400908BD00BF14
:10CCA8001CBB0A0010B598B004461422002102A843
:10CCB80088F0BCFA44F21213ADF804304FF48073D4
:10CCC8004FF48042ADF80630144B2146CDE90323DA
:10CCD80004230DF11D008DF81C3067F061FD04F18F
:10CCE80020010DF13D0067F05BFD6B46412207A96D
:10CCF80001A887F05BF9044601A887F050FC2CB91D
:10CD0800009887F089F8012018B010BD0448234620
:10CD18000121044A65F024FA0020F5E70000020921
:10CD2800005D0900385A0A0010B5002834D01D4AA1
:10CD3800136823B1043B984231D05B68F9E71A4B7A
:10CD4800D3E8AF1F890707D518480221184A65F0AC
:10CD5800FEF96FF00F0010BD1468011D44605068A3
:10CD6800116000B95160D3E8EF2F42F00101C3E828
:10CD7800E01F0028F7D1D30701D50020EBE70D4BC2
:10CD8800D3E8EF1F21F01001C3E8E21F002AF7D112
:10CD98000948FCF709F9F0E76FF01500DBE76FF0D9
:10CDA8007700D8E7EC510020E4510020005D09002D
:10CDB8005C5A0A0008020020A8080020044BD3E8A7
:10CDC800AF3F13F0100F034808BF0020704700BFA3
:10CDD80008020020BBA9002070B505461948036861
:10CDE8008B4228D0184BD3E8AF3FDA0626D5036824
:10CDF80013B16FF00F0070BD144AD2E8AF3FDB07E4
:10CE0800F7D4D2E8EF3F43F00204C2E8E64F002E21
:10CE1800F7D113F00204ECD1016029460C4867F001
:10CE2800BFFC0C4805F1200167F0BAFC0A48FCF782
:10CE3800BBF82046DFE76FF07700DCE76FF07C0097
:10CE4800D9E700BFE851002008020020E451002083
:10CE58007BA900209BA900209808002070B50546F2
:10CE68000B4B1C6844B154F81C3C1C3C13B12846BD
:10CE7800297B9847E469F5E7064C074EB44200D38E
:10CE880070BD236813B12846297B98472034F5E7FD
:10CE980028520020585C0900985C090010B5044627
:10CEA800F8F7CAFF044901EB0011204667F069F85A
:10CEB800BDE81040FDF7ACB9F4510020002270B570
:10CEC8000446D1E901560748C1E901226CF079FB13
:10CED8003DB1314620462B46BDE870406FF06D02EB
:10CEE800184770BDC01E002030B5051D04464FF41C
:10CEF8008061284685B067F07DFC400533D428461C
:10CF080067F073FC810321D5E17871B3637B072B4C
:10CF180029D1224B93F890309B0624D567F0C1F8AD
:10CF280008B30DF10E0103A8FDF776FAD8B920462B
:10CF3800BDF80E20BDF80C1067F01FF9034690B13C
:10CF48000121174A174867F053FC0CE0204667F0A8
:10CF5800F9F8034620B10121134A124867F048FC4A
:10CF6800637B072BD0D005B030BD0C4B93F89130C4
:10CF7800DA0706D4022319460C4A0A4867F038FC37
:10CF8800C4E7022320461A46009167F015F90346C4
:10CF98000028BBD00121064AEFE700BF800100202E
:10CFA800DB5A0A00C05C09008A5A0A00AB5A0A0018
:10CFB800C45A0A0070B50546002200230E4825F021
:10CFC80027FAB8B90D4B1C6834B154F8143C1C3C12
:10CFD80003B19847E469F7E7094C0A4EB44204D311
:10CFE8002846BDE8704025F005BCA36803B1984702
:10CFF8002034F3E770BD00BF9C1E0020285200209B
:10D00800585C0900985C09002DE9F0410446202786
:10D018000025EFF3118287F31288BFF36F8FE16960
:10D0280029B1206A0B688142E36108BF236282F359
:10D038001188BFF36F8F71B1D1E901680748C1E961
:10D0480001556CF0BEFA1EB1002241462046B04799
:10D05800FDF7DEF8DDE7BDE8F08100BFC01E002067
:10D068000348B0F8BC30C030002B08BF0020704720
:10D078008001002030B50446F8F7C8FB0D460D4A7C
:10D088000D498BB00858D2F8E010884205D12046E7
:10D098000BB0BDE83040FFF7B7BF24342146104637
:10D0A8006CF09DFB1DB1694620466CF0A8FB0BB0E7
:10D0B80030BD00BF783E00200800000038B50022CF
:10D0C80004468A4202D10024204638BD012004F1DA
:10D0D800C803D3E8EF5F002D04D1C3E8EC0FBCF11F
:10D0E800000FF6D102D0D0340244EAE7002CEAD08F
:10D0F800C8220021204688F099F804F1400004492C
:10D108006CF09FFB034904F124006CF03DFBDBE766
:10D1180051DF00001F480700F7B516460D460121EC
:10D128000446FFF7A7FF012E23D0022E52D1236910
:10D138003BB135480121354A65F009F8204667F0CA
:10D1480088FB25612269138A012B5AD9D268128873
:10D15800043292B2934254D343D9012100922A480F
:10D168002B4A65F007F8204603B0BDE8F04067F0A9
:10D1780070BB206940B9274A3146234864F0E7FF6D
:10D18800204667F066FB01E02A8A2AB9284603B0E0
:10D19800BDE8F040F8F7F0BE018A438A47695B1A98
:10D1A800C168C91B5B1A9A420CD91B4A31461648FA
:10D1B80064F0CDFF00222046216901F0A7F9002381
:10D1C8002361E3E7E9680C3065F0E8FB2846F8F7E7
:10D1D800D3FEB7E701213346104A0B4867F008FB36
:10D1E800CEE7002204F11003D3E8EF1FC3E8E02FD5
:10D1F8000028F9D10122204603B0BDE8F04001F033
:10D2080085B903B0F0BD00BFC05C0900F75A0A0039
:10D21800775B0A00145B0A00325B0A00595B0A005C
:10D2280008B500F1C803D3E8EF2F013AC3E8E12FAE
:10D238000029F8D1AAB90B4B984212D303F1D002B6
:10D2480090420ED2C01AD023B0FBF3F203FB1200B7
:10D2580038B9054825F0A0F8BDE80840034825F08E
:10D26800C9BA08BDB82F00209C1E0020C80800209D
:10D2780010B5044667F0FCFA25F010FF0C4B04F1DA
:10D28800BC01D3F8DC3043B90A4867F093FA25F0BB
:10D2980019FFBDE81040FCF7BBBF994201D01B68DD
:10D2A800F1E725F00FFF2046FFF7BAFFF1E700BFCF
:10D2B800800100205C020020F8B5457B04468D42C1
:10D2C8000E4600AF1CD1082D98BF694B6C4688B03C
:10D2D80094BF53F82530674B6A466749CDE9051373
:10D2E8004FF40073ADF81C30644B42F8103F002334
:10D2F8004FF4E4516248F6F74FFFA546BD46F8BD26
:10D308004173DDB1022D1CD0637B082B00F2AD8088
:10D3180001A252F823F000BF7FD3000019D4000007
:10D32800E9D3000005D3000005D3000005D30000B1
:10D3380005D3000059D3000005D3000067F098FA20
:10D34800E2E78378012BDFD140306CF088FADBE725
:10D358000023C4E90D33E378012BCFD1A378494AE0
:10D36800012B04BF032384F89830002304F1400004
:10D3780025F0B0FAC2E7082DC0D8DFE805F02A0585
:10D3880021172626212A2A0004F1400528466CF098
:10D3980066FA01212046FFF76DFE204667F059FA2C
:10D3A80000220023284625F0CDFAA7E70220FFF740
:10D3B80073F8034620B10221334A314867F018FA5E
:10D3C800237B13B12046FFF749FD2046FFF728FFCE
:10D3D80094E733462D4A0221294867F009FA8DE778
:10D3E800A378012B8AD12A4B9D8A002D86D00A2347
:10D3F80040F2E730002147F612265D434FF47A7277
:10D408000023E5FB0601F3F787FE02460B46ADE76E
:10D41800237B3E2B0FD16D4688B06A461D4BCDE964
:10D428000534032342F8103F00234FF4C451144835
:10D43800F6F7B2FEAD46164D05F1C006616911B9A1
:10D44800FCF7E6FE5AE7A2690B68914208BFA361A0
:10D4580020466361FFF732FDB5F8BC30002B14BFDE
:10D468003046002024F098FFE8E70B4A3346B2E73D
:10D4780074660900925B0A009C5B0A0003000001C5
:10D48800C05C09005A620200AD5B0A00DE5B0A005C
:10D4980080010020F55B0A001C5C0A00F8B507460D
:10D4A80009480D46164667F0E3F9044650B18378FB
:10D4B8001F4203D1BDE8F840FFF7B2BE3146A84786
:10D4C8002046F7E7F8BD00BFB82F00200022012052
:10D4D8000149FFF7E3BF00BF1348070070B50546D1
:10D4E8000E480E4667F0C4F90446A0B1437B012BF1
:10D4F80002D0073B012B0CD82388AB4208D1A37874
:10D508001E4209D102212B46054A064867F070F9E8
:10D518002046FFF785FE0024204670BDB82F002066
:10D52800385C0A00C05C0900034BC01A034B0011A9
:10D538005843C0B2704700BFB82F0020C54EECC496
:10D5480070B51C46144305460E460DD0F8F75EF933
:10D558000E49D1F8E0400E4909588C4206D1022103
:10D568000C4A0D4864F0F3FD002213460B49002DC8
:10D5780014BF2846084665F079F9044618B1711DAC
:10D588000C3065F0FAF9204670BD00BF783E0020E7
:10D59800080000004F5C0A00C05C0900D81E00208B
:10D5A80010B50446054825F025F9204600F0A8FEE8
:10D5B8002046BDE81040FFF751BC00BFB808002066
:10D5C8002DE9F04F002387B000AFFB607B61B94BBA
:10D5D8005A8B3AB1B84DD5F8DC403CB91C37BD463A
:10D5E800BDE8F08F1B68002BF4D1F7E754F8BC397D
:10D5F80003B1BC3B0026B14901E01C461346B5F80F
:10D60800BC20002A00F05481D5F8C8204AB904F19A
:10D61800BC06002BE2D0D3F8BC20002AEDD0BC3ADF
:10D62800EBE70A68002AF2D0D4F8A820002AEED046
:10D63800D4F8AC20002AEAD0D4F8B020002AE6D0EA
:10D64800637B072B6AD120469047002866D004F1F7
:10D65800C00067F0CAF8022860DC204667F008F9C5
:10D6680004460028BAD0637B072B40F01E81204671
:10D67800D4F8A830B5F8BC1007F1100298478146D5
:10D68800002800F00581B5F8BC203B699A4208D310
:10D698000146D4F8AC60204607F1140307F10C02E8
:10D6A800B0477B69D7F80C803B60B9F81030002B85
:10D6B80000F0F5804846D7F810A066F078FC78604E
:10D6C800002840F0EF80B5F8BC30DFF800B2002B3E
:10D6D80014BF584600200022002324F099FE78B990
:10D6E80000220023754824F021FE064600283BD17D
:10D6F800B5F8BC30002B18BF5E46304624F04CFE0F
:10D708006FF00B054846F8F737FCB8F1000F00F04A
:10D71800AA802A4620463968C047A4E0D4F8BC301D
:10D7280004F1BC02C6B9D5F8E010C5F8DC308A426D
:10D7380001D1C5F8E03000232046C4F8BC30D4F845
:10D74800B030984700288ED0637B072B40F0AD801F
:10D758002046FFF78DFD86E73360D5F8E0309A4222
:10D7680008BFC5F8E060E6E73B68C0F8048083605E
:10D77800B5F8BCB00022DA454FF000034FF00001C5
:10D788004C4898BF1FFA8AFBF8F778FB804650B1DF
:10D79800F8F752FB4A4B5A4603EB001349464046FA
:10D7A80066F0CAFB8046B5F8BC3094F8C4909A4538
:10D7B80084BF01237B607B689CBF09F102095FFA83
:10D7C80089F984F8C43004F1C00ADAE8EF3F01337C
:10D7D800CAE8E23F002AF8D104F1140B3146584652
:10D7E80066F0E8FFA378012B56D108F10C03042159
:10D7F80018467B6065F000F9228809F0FD0942EAC5
:10D8080009320280B8F810207B68043A428002216D
:10D81800184665F0F9F84046FCF77CFC814600287C
:10D8280043D0DAE8EF3F013BCAE8E23F002AF8D1EB
:10D838003146584666F0F2FF224A4B4601212248FB
:10D8480066F0D6FF4046F8F797FB20463146FFF7CB
:10D8580035FBB5F8BC301D48002B08BF002024F06C
:10D868009BFD6FF004056E4688B0194A0423CDE984
:10D8780005256A46079442F8103F4FF401511248B3
:10D888000023F6F789FC1321B546204667F007F810
:10D898002046FFF7C5FCA1E66FF01509C1E76FF058
:10D8A80079052FE76FF004052CE7FCF7B1FCEFE7EB
:10D8B8009368FFDE881F002080010020C01E002022
:10D8C800F45100206C500A00C05C0900400200209E
:10D8D800785C0A0040F2E2432DE9F041D0F8886014
:10D8E8000446B6FBF3F6031D184666F07EFF820475
:10D8F800B6B213D5B4F88C20B2420FD8B4F88E2043
:10D90800B2420BD3D4E92412914207D1D3E8EF1FD6
:10D9180021F40051C3E8E21F002AF7D1104B1D681B
:10D9280065B155F80C7C1C3D37B131462046B4F83A
:10D938009230B4F89020B847ED69F1E7094DDFF867
:10D948002880454501D3BDE8F0812F6937B13146BC
:10D958002046B4F89230B4F89020B8472035F0E764
:10D9680028520020585C0900985C09002DE9F04114
:10D97800074608460D4666F096FB064618B9002687
:10D988003046BDE8F081144B1C6884B154F8103C53
:10D998001C3C0BB9E469F8E7294638469847002843
:10D9A800EDD0284666F07FFB0028F3D1E7E70B4C63
:10D9B800DFF82C804445E3D2E3680BB92034F9E75B
:10D9C8002946384698470028D9D0284666F06BFB88
:10D9D8000028F3D1D3E700BF28520020585C090083
:10D9E800985C09002DE9F041C37804468BB900F131
:10D9F8007E06114B1D687DB11C3D04F170076B69F3
:10DA08001BB13A46314620469847ED6925B11C3D81
:10DA1800F5E700F17706ECE7084D094F04F17008C7
:10DA2800BD4201D3BDE8F0816B691BB14246314666
:10DA3800204698472035F3E728520020585C090013
:10DA4800985C0900F8B5437A04468372164667F075
:10DA5800F8F8144B1D684DB155F8043C1C3D1BB13A
:10DA680032462046617A9847ED69F4E70E4D0F4F2C
:10DA7800BD420DD3A6B9637A012B11D9A378012B26
:10DA88000ED1207A04F17001BDE8F84006F0ACBE72
:10DA9800AB691BB132462046617A98472035E7E7E3
:10DAA800F8BD00BF28520020585C0900985C0900A6
:10DAB80038B505460C460F480121FFF7FFFAC0B1FB
:10DAC800057223680367A388A0F87430A37980F8E7
:10DAD80076300123437283728370074BC0F8A830F5
:10DAE800064BC0F8AC30064BC0F8B030054BC0F858
:10DAF8008C3038BDB82F002009E20000DD47070050
:10DB0800D14707001800280070B505460A480E4698
:10DB180066F0AEFE044620B18378012B04D0FFF7EF
:10DB28007FFB0024204670BD3246294666F0ABFFD5
:10DB38000028F7D12046F2E7B82F0020F0B589B0C9
:10DB480000AF0D46FFF7E0FF044618B329463846F4
:10DB5800FBF794F9637B6D46082B98BF0F4A8AB090
:10DB680094BF52F823300E4B6A46CDE907730D4B2C
:10DB78000D4909930D4BCDE9051442F8103F0023D8
:10DB88004FF442510A48F6F707FB2046AD46FFF727
:10DB980047FB01202437BD46F0BD00BF746609006D
:10DBA800925B0A00010302049B5C0A000500000264
:10DBB800C05C090038B50446134866F016FE4207F3
:10DBC80002D46FF00A0038BD084666F06CFA10B946
:10DBD8006FF01500F7E7FEF73BFF0028F1D10A4880
:10DBE80066F003FE0306C0F3C0150AD466F0AAFC6B
:10DBF8000028EDD021462846FFF7A0FF0028E2D0F4
:10DC0800E6E76FF07700DEE708020020F8B5054682
:10DC18000E480E46174666F02BFE044620B1837860
:10DC2800012B03D0FFF7FCFA00240DE036B1324691
:10DC3800294666F028FF08B92046F3E7637BBB4214
:10DC4800FAD1237AAB42F7D12046F8BDB82F00208D
:10DC580070B58B780646012B0C4692B042D191F8EC
:10DC6800703007AD032B37D8DFE803F002303234C9
:10DC78001E492846F3F7B4FA059594F871301E2129
:10DC8800049394F872301A4A039394F873300AA8EC
:10DC9800029394F87430019394F87530009394F8D3
:10DCA80076305EF0D9FD32460AAB10AD1C4603CC87
:10DCB800AC4210605160234602F10802F6D1206898
:10DCC80010603046A388938012B070BD0949D0E730
:10DCD8000949CEE70949CCE70A212846084A5EF0F7
:10DCE800BBFDC9E700238DF82830DCE7B8490A00F6
:10DCF800D3490A0099AB0A00BF490A00C9490A007A
:10DD0800746B0A00002210B5837804460B70C37840
:10DD18004B70037A8B70437B81F82320023BDBB284
:10DD2800062B8EBF13462848C35C204681F8203056
:10DD3800A378012B14BF0023637A81F8213066F0A1
:10DD480034FE81F82200A378012B3AD104F1700344
:10DD58008B60237A1D4AC3EBC30313444B60E278FC
:10DD680004F1770304F17E0012BB1A460346C1E9A9
:10DD7800032340F2E242D4F888304B61B3FBF2F35C
:10DD88000B83B4F890304B83B4F892308B83D4F87B
:10DD9800A4302BB15B7CDA0644BF012381F8233021
:10DDA800D4F8A43013B15B7C9B0603D4002010BDCB
:10DDB8000246DCE791F8233043F0020381F8233070
:10DDC800F4E76FF01500F2E75CBB0A008001002061
:10DDD8002DE9F04104460F4615469846002B6ED0B3
:10DDE8001B6823B10221394A394864F0B0F9294641
:10DDF8002046FFF7DFFE064600283FD12046294689
:10DE080066F017FE044600285CD097E80F00314DF5
:10DE180005F1080C8CE80F00AB8A002B08BF4FF403
:10DE28009673AB822B8A03B9AB892B826B8A03B9B1
:10DE3800EB8929486B8266F0D8FC430501D5FDF7CC
:10DE4800C3F995F8DB2095F8DA309A4219D90321FD
:10DE58002046FFF731FA0220FEF7F6FA054658B1D8
:10DE68000220FEF719FB20460021FFF725FA20467D
:10DE7800FFF7D6F92E4601E0C8F800403046BDE865
:10DE8800F08102212046FFF717FA204666F034F9A0
:10DE980005460028F0D0002120462173FFF70CFA30
:10DEA8002046FFF7BDF90320FEF7CEFA0346002807
:10DEB800E0D00221094A064866F09AFCDAE76FF0DA
:10DEC8001506DBE76FF00B06D8E700BFD45C0A0045
:10DED800C05C09008001002008020020064C0A00EE
:10DEE80038B5044608460D4666F0DDF838B3154BDC
:10DEF80093F89030990707D4E37873B12946204600
:10DF0800BDE8384000F02EBB94F899309A07F3D555
:10DF1800201D66F06AFC4304EED42946204666F0CC
:10DF2800D8FD58B92B88A4F88C306B88A4F88E30AB
:10DF3800AB88A4F89430EB88A4F8963038BD6FF01D
:10DF48001500FBE780010020F7B510F8333C0446C4
:10DF5800A0F140060BBB304666F016FE3C4B1D6830
:10DF68004DB155F8183C1C3D1BB1304614F8341C13
:10DF78009847ED69F4E7374D374FBD4205D3304632
:10DF880003B0BDE8F040FFF74BB96B681BB13046F2
:10DF980014F8341C98472035EFE710F83E3C012B65
:10DFA80053D110F83D3C8BB9FCF75EFB69304CD17E
:10DFB80002212A4A2A4864F0CAF840F2391200239A
:10DFC800204603B0BDE8F04024F0BCBCA0F13C05FD
:10DFD800D5E8EF3F23F40052C5E8E12F0029F7D137
:10DFE80099041FD5E36C69460093636D304601932D
:10DFF800FFF776FF034678B9D5E8EF3F23F480535F
:10E00800C5E8E23F002AF7D14FF40061284603B083
:10E01800BDE8F04066F0EEBB124A0221104866F0F7
:10E02800E7FBF1E74FF428130F4A69463046CDE97C
:10E038000023FFF755FF034628B94FF480512846BF
:10E0480066F0D8FBE0E7094AE7E703B0F0BD00BF98
:10E0580028520020585C0900985C0900095D0A00F4
:10E06800C05C09003C5D0A0018002800615D0A00D8
:10E0780008B568B1094B00F10C011A6822B90748C4
:10E0880066F098FB104605E0914204D01268F5E767
:10E098006FF0150008BD6FF07700FBE730520020E5
:10E0A80038B517486BF04FFA164915486BF089FADE
:10E0B800154913486BF085FA144911486BF081FA39
:10E0C80067F0CBF904F0C4FA0446B8B906F094F83E
:10E0D800044698B966F017FE0D4866F0C9FB054678
:10E0E80060B1043066F081FBC30704D503212846DC
:10E0F8002C72FFF7E1F82846FFF792F8204638BD62
:10E10800C01E002004520020105200201C52002083
:10E11800B82F002003460121014A024864F020B8C4
:10E12800145E0A00305D090080B500AF88B06A4609
:10E13800074BCDE90530032342F8103F00234FF485
:10E14800C2510448F6F728F86FF00B00BD4680BDB1
:10E158003C5E0A00305D090008B5064A136823B919
:10E168000548506018460A6008BDFFF7DDFF6FF0EC
:10E178000B00F9E73C520020C066090070B5044660
:10E1880052EA030008D0F7F741FB074D074ED5F8D0
:10E19800E0503058854201D1002213462046BDE8A0
:10E1A80070400431FFF7CCB9783E00200800000029
:10E1B80038B5054618462B68DBB15B7B072B18D1B1
:10E1C8000B7A012B07D001210B4A0C4863F0C8FFDA
:10E1D8006FF0150038BDCB7A072BF9D9C8618A6171
:10E1E80005F130006BF0EDF9284666F0A4FC00203C
:10E1F800F0E76FF07F00EDE7635E0A00305D09002D
:10E208002DE9F84F88469146D0F8B44000AF44B1A4
:10E21800483C236B63B92068B43066F0ABFCA46C4F
:10E22800F5E7FBF7F5FF00263046BD46BDE8F88F59
:10E2380004F1300A50466BF0E9F905460028F0D0A1
:10E2480065F0B5FE80B16C4688B06A46294BCDE9C9
:10E258000535032342F8103F00234FF4C2512648E6
:10E26800F5F79AFFA546DEE7284664F041FBE56C22
:10E2780006469DB9A38C058A403B9BB23F2B03D829
:10E28800238D9D4228BF1D46042106F10C0064F031
:10E29800B3FB0580A38C04354380E56445451FD84E
:10E2A800B6F810B0AB4506D100220023504624F042
:10E2B8003DF8F7F761FEA38CA3F140023F2A06D888
:10E2C800AB451ABF002213460C4AF361B2612068BD
:10E2D800B43066F04FFC236B13B1204666F02BFC7C
:10E2E800E36C98452CBF0021A3EB0801C9F8003066
:10E2F800E16499E77B5E0A00305D0900C14C0700C4
:10E30800F7B504460026234D234FBD4201D303B081
:10E31800F0BD2988204666F0C6FC6B68019001A90B
:10E3280020469847002830DB019B2A889A829A84E5
:10E3380003F11002D2E8EF1FC2E8E06F0028F9D11C
:10E348009E64DE649E60A16B03F10802F9B9C4E91A
:10E358000D221C60DE6003F130006BF0F4F80198C8
:10E3680043681B6803B19847019B1033D3E8EF1F3C
:10E3780041F00101C3E8E21F002AF7D10198436880
:10E38800DB6913B100F1100198470835BDE70A6051
:10E39800A263DEE7405C0900585C09007FB50D46C2
:10E3A8000646042105F10C0064F03FFB2A8A4388E5
:10E3B8000446934208D000931346444A0121444836
:10E3C80063F0D8FE04B070BD417839B90121414AE3
:10E3D8003F4804B0BDE8704063F0B9BE0278122A25
:10E3E80022D0132A1AD0012AECD002211346384829
:10E3F800394A63F0B5FE617802220120356866F07B
:10E4080038FC04460028DDD002210C3064F0C0FA44
:10E418000023214603704370284624E0022BD1D004
:10E42800022200922D4AC9E7082B03D00822009245
:10E438002B4AC3E73468637B072B02D00221294AA1
:10E44800C6E7E378A3B10222012066F012FC054674
:10E458000028B7D002210C3064F09AFA002329462C
:10E4680003704370204604B0BDE8704066F031BCCC
:10E47800EB6813201A88ADF808205A88ADF80A20EE
:10E488009A88ADF80C20DB880222ADF80E3066F0D1
:10E49800F0FB0546002895D002A92046FFF766FA4A
:10E4A8000646022105F10C0064F072FA86F00103B9
:10E4B800DBB203802946204666F00BFC002E81D093
:10E4C800204602A966F005FB7CE700BF935E0A00C0
:10E4D800305D0900B45E0A00405F0A00D55E0A009C
:10E4E800005F0A00325F0A0008B50B8A032B06D8C2
:10E4F8000121044A044863F02AFE002008BDFFF702
:10E508004DFFFAE7685F0A00305D090038B50B8AED
:10E518000546032B0C4609D801210F4A0F4863F022
:10E5280016FE2046BDE83840F7F726BD042104F161
:10E538000C0064F07AFA4188284666F0DBFB30B9B3
:10E54800074A0B460548022163F00AFEE9E74368DB
:10E5580021465B699847E4E7865F0A00305D090059
:10E56800A35F0A0070B5134A0C46137806460133B8
:10E5780013F0FF010ABF01230B461946137012203E
:10E58800082266F076FB054688B108210C3064F055
:10E59800FFF922882946028062884280A288828008
:10E5A800E288C2803046BDE8704066F092BB6FF0EA
:10E5B8000B0070BDFBA9002023281FD81A2804D8F7
:10E5C800431E182B0ED906207047A0F11B03082BF9
:10E5D8001ED8DFE803F0051D1B231D19251D0500A6
:10E5E8000320704701230F4A83401A40C2B90E4ADC
:10E5F8001A40002A0CBF06200120704700F07F0354
:10E60800522B05D100207047012070470520704724
:10E6180010F0400F14BF00200620704704207047F8
:10E6280002207047AAAA8A02545545012DE9F74FDE
:10E63800064608460C46F7F7FFFB182343432D4FC1
:10E648000546FA1891680191E16806F15400D0E88E
:10E65800AF0FC0070AD40121274A284866F076FB85
:10E668006FF01509484603B0BDE8F08FE068007800
:10E6780010710022FA500B78D22B0FD13368214643
:10E68800186868F041F8814640B101211C4A1B48CE
:10E6980066F05CFB2046F7F76FFCE3E7182303FB03
:10E6A8000573D4F80C80D4F814B0B4F810A09E60A8
:10E6B800002321461A46301DFFF77AFD81460028BF
:10E6C800D0D010F1690F04D101210E4A0B4866F031
:10E6D8003DFB6269A8EB0B0812FA88F2E260182287
:10E6E8005543019B7A19A4F810A0936047F8059048
:10E6F800B8E700BF94520020DF5F0A00B05C090051
:10E70800F95F0A000C600A0008B5EFF311812023B5
:10E7180083F31288BFF36F8F002303600F4B5A688F
:10E72800C2B9C3E9000081F31188BFF36F8F0C48A9
:10E7380024F060F8031E0CDA01210A4A0A4863F043
:10E748000FFD002383F31188BFF36F8F032318464F
:10E7580002DF08BD10605860E5E700BF8C5200205A
:10E76800000900202F600A00B05C0900094B011F56
:10E778009A680948914204BF00229A601A6A914235
:10E7880004BF00221A629A6B914204BF00229A6366
:10E798006AF0B7BD945200207C1D00200121024A76
:10E7A800024866F0D3BA00BF58600A00B05C09009E
:10E7B80010B5044600F15003D3E8EF1F41F0010102
:10E7C800C3E8E21F002AF7D1201F66F0E8FA04F137
:10E7D800740004496BF035F82068BDE8104003F078
:10E7E8008DBD00BFF5F7000073B50E46438D418B14
:10E7F80001328B4228BF0B469A42054609D90221AD
:10E8080000921D481D4A63F0B5FC0024204602B062
:10E8180070BD3046FFF7D0FE6FF01403034113F0CC
:10E82800010310D0F6F7F2FF154B1958154BD3F822
:10E83800E03099421DD0144B1B685A1A18BF4FF08C
:10E84800FF32134600E0114A00211148FFF796FCF9
:10E8580004460028DAD0F7F7EFFA18220D4B012109
:10E8680002FB003304F10C009D6064F091F806701F
:10E87800CCE70022E5E700BFB05C090075600A003C
:10E8880008000000783E0020DC5200201C4E0E00DC
:10E89800041F00209452002070B5044601F10C00BA
:10E8A8000D4664F0D2F8266801462B8AEA6830687B
:10E8B80067F0C3FC1E2100222046FFF795FF0146A2
:10E8C80030B90121044A054866F040FA002070BDBD
:10E8D800204666F056FAF9E79A600A00B05C09002B
:10E8E800F0B51D4603680E460039044618BF0121DD
:10E8F80087B01868174667F0B1FC40B904F15400B6
:10E9080066F07EFB002846D0002007B0F0BD002D41
:10E9180043D018220021684686F088FC6FB1002297
:10E9280013212046FFF760FF019030B91C480121F0
:10E938001C4A66F00BFA1120E7E7236829461B6892
:10E94800284600930023ADF812300C9B164A039317
:10E95800BDF834308DF80860ADF8103001238DF81B
:10E9680014306B4666F0F4FA9DF8143063B1002F4A
:10E97800CAD00198F7F700FB2A46314620469DF891
:10E98800143066F048FBBFE701990029BCD0204647
:10E9980066F0F7F9B8E71220B7E70120B5E700BF3E
:10E9A800B05C0900B7600A000F4E07002DE9F3417B
:10E9B8000B8A04460D4643B90121294A294866F0C5
:10E9C800C5F9002002B0BDE8F0810768012105F112
:10E9D8000C0064F02AF87B7B0646072BF1D154F82B
:10E9E800043C002BEDD0002203781F4F043C17F89D
:10E9F80032004FEAC208984207EBC20114D12A8AB2
:10EA08004878904226D90121009316481346174AA0
:10EA180063F0B0FB04234744BA78012AD1D1002B14
:10EA2800CFD00022317811E001321C2ADFD1104A00
:10EA380002210C4863F094FB31780846FFF7BCFDCF
:10EA48002122C24012F00102BBD10623204666F003
:10EA5800E2FAB6E74B682046294698470346DAE7C4
:10EA6800D0600A00B05C0900E866090005610A0088
:10EA7800EB600A00F8B5124A0746002311480D4614
:10EA880063F0F4FE044638B901212B460E4A0F48BC
:10EA980063F066FB2046F8BD00F10C0609213046FC
:10EAA80063F06BFF2046F7F7C7F91822084B0121DE
:10EAB80002FB003330469F6063F06AFF0570E9E7A8
:10EAC8001C4E0E00041F0020145E0A00B05C0900F2
:10EAD800945200202DE9F0410E8A0446043EF6B215
:10EAE800022E08468CB001D0102E64D104210C30BF
:10EAF80063F09BFF0DF1080805884788011D324621
:10EB0800404665F0C4F9002857D0A5B300268FB356
:10EB1800AF4230D34FF42053404601A98DF804602A
:10EB2800ADF8063065F086F948BB1422002107A825
:10EB380086F07CFB11212046FFF79CFF09900028F6
:10EB480037D001210C30CDE9074863F021FF0023BD
:10EB58000A90394603701A4A0B93284607AB66F0A9
:10EB6800F7F9DDE909131B78FBB90846F7F704FA4A
:10EB78000A2301E03D4601232A4610210EE042F611
:10EB88000103404607A98DF81C60ADF81E3065F0FA
:10EB980051F90028C9D010232A461946204666F0A4
:10EBA8003AFA00200CB0BDE8F081204666F0E9F89A
:10EBB800F7E71120F6E70420F4E70E20F2E700BF9C
:10EBC80021F100002DE9FF41036804460D4618684D
:10EBD800012167F043FB40B904F1540066F010FAD4
:10EBE800A0BB122004B0BDE8F081102200216846C5
:10EBF80086F01CFB21212046FFF73CFF029038B32A
:10EC08004FF00108009405F10C072B8A012B04D85A
:10EC18002046029966F0B5F818E0384663F015FF0B
:10EC28006B4601460B4A06468DF80C8066F090F953
:10EC38009DF80C30002BE8D00298F7F79DF9324682
:10EC4800202120469DF80C3066F0E5F90020C9E740
:10EC58001120C7E7815207002DE9FF4103680446E8
:10EC68000D461868012167F0F9FA40B904F154001B
:10EC780066F0C6F9A0BB122004B0BDE8F0811022EE
:10EC88000021684686F0D2FA0F212046FFF7F2FEEF
:10EC9800029038B34FF00108009405F10C072B8A55
:10ECA800012B04D82046029966F06BF818E0384624
:10ECB80063F0CBFE6B4601460B4A06468DF80C8086
:10ECC80066F046F99DF80C30002BE8D00298F7F76B
:10ECD80053F932460E2120469DF80C3066F09BF918
:10ECE8000020C9E71120C7E705530700F0B51D4606
:10ECF800036804460E4685B001211868174667F078
:10ED0800ADFA38B904F1540066F07AF950BB122014
:10ED180005B0F0BD65B310220021684686F086FA7A
:10ED280039462046FFF7A6FE029018B3BDF82830F2
:10ED38002946ADF80430012328468DF80C300E4AD8
:10ED48006B46009466F004F99DF80C3002995BB1AB
:10ED58000846F7F711F92A46314620469DF80C3047
:10ED680066F059F90020D3E7204666F00AF8F9E77B
:10ED78000120CDE71120CBE7055307002DE9F0412D
:10ED88000E8A0446043EF6B2022E08468CB001D024
:10ED9800102E76D104210C3063F047FE0DF10408E3
:10EDA80005884788011D3246404665F070F80028FE
:10EDB80069D085B377B3BD422DD80121606867F06B
:10EDC8004DFA064678BB42F602038DF80000694604
:10EDD8004046ADF8023065F02DF820B342F6030343
:10EDE800404606A98DF81860ADF81A3065F022F88B
:10EDF800C8B1012D03D14FF6FF739F4213D004F120
:10EE0800540066F0FDF8002814BF002012200CB052
:10EE1800BDE8F0813D4601232A460821204666F0D8
:10EE2800FAF80020F3E7182200210DEB020086F023
:10EE3800FDF909212046FFF71DFE0890F8B10121D0
:10EE48000C30CDE9064863F0A3FD00230990037058
:10EE58000A2339468DF82C30284606AB0B4A66F053
:10EE680077F89DF82C3008992BB10846F7F784F805
:10EE78009DF82C30D0E7204665F083FFD1E71120BC
:10EE8800C5E70420C3E70E20C1E700BFD9F10000A1
:10EE98002DE9F0430F460446062187B007F10C0020
:10EEA80063F0C3FD0588EDB1B0F80280B8F1000F3A
:10EEB80017D0454516D8002382888DF800308DF884
:10EEC80004304FF42053684601A9D7F80C90ADF8E8
:10EED8000220ADF8063064F0ADFF064660B10A23A3
:10EEE80001E0454601232A460621204666F093F8AC
:10EEF800002007B0BDE8F0830146142201A83F7C3A
:10EF080086F094F907212046FFF7B4FD0290D8B1A6
:10EF18000A2341468DF81530284601AB0B4ACDE946
:10EF2800036901948DF8147066F012F89DF8153095
:10EF380002992BB10846F7F71FF89DF81530D2E76C
:10EF4800204665F01EFFD3E71120D2E7C5EF000089
:10EF58007FB5CB6804461D888DB15E8876B1B54211
:10EF68000DD810220021684686F060F90521204658
:10EF7800FFF780FD019058B9112007E035460123BD
:10EF88002A460421204666F046F8002004B070BDE9
:10EF98006B4631462846084A009465F0D9FFDDE9FA
:10EFA800011323B90846F6F7E7FF0A23E8E72046E6
:10EFB80065F0E7FEE9E700BF814E07002DE9F04361
:10EFC80042F60103002591B0D2F8008006460F46AC
:10EFD80000680BA9D8F8049014468DF82C50ADF8A9
:10EFE8002E3064F027FF00286DD04FF4205330688E
:10EFF8000BA98DF82C50ADF82E3064F01BFF38B1FA
:10F00800A3681BB15A88BA4200D25F80012010E081
:10F018006168084665F082FEB8F82A20B8F81A3008
:10F028009A4294BFC0EB0200C0EB0300032803D848
:10F03800002011B0BDE8F083084663F060FC054687
:10F048006168084665F06AFE6B8A2A8AA3EB020C9F
:10F058006B69EA68D21AACEB0203B8F82AC0B8F8B0
:10F068001A20944594BFC0EB0C00C0EB0200834209
:10F0780028BF03466BB9887AF6F7D6FE002200232C
:10F0880063F0F4FB05460028D2D00146606863F0BF
:10F0980047FC002300933146D6F8048010234846E5
:10F0A80002AAC047061E0EDB227CE068964227D0E3
:10F0B80001460BA864F0EBFE40B9237C134A0221F9
:10F0C800134863F04DF80023A3609FE7F2B202A94A
:10F0D80006A864F0DCFE10B90E4A3346EFE706A92D
:10F0E8000BA864F0A7FE0028EDD100230421637467
:10F0F80005F10C0063F04CFCA0600780A36884E76E
:10F10800324602A986F09AF8EDE700BF24610A00AA
:10F11800B05C090043610A002DE9FF414FF0000887
:10F128004FF4205305460E46006802A91446176896
:10F138008DF80880ADF80A3064F07CFEA0B142F684
:10F148000103286803A98DF80C80ADF80E3064F02F
:10F1580071FE48B123691BB15A88B24200D25E8061
:10F16800012004B0BDE8F0816168286864F062FE9F
:10F1780010B100232361F3E7E368A0681A786AB145
:10F18800B7F81AC0798D038A8C4594BFC3EB0C037A
:10F19800C3EB0103934201DA0020E2E704210C30BB
:10F1A80063F0F6FB20610680236929465E80074BE1
:10F1B8000194009338460023A26865F0D4FF002824
:10F1C800EADB2069003818BF0120CAE7394F070079
:10F1D8002DE9F347176805468946006851681446C3
:10F1E800D7F804A064F026FE804600284BD195226B
:10F1F8002946504666F093FE0646207540B1E368FE
:10F208001B780BB184F81480002002B0BDE8F087A9
:10F218002946504667F05BF810B908232375F3E7D1
:10F22800A068267563F06BFB02210C3063F0B0FB1D
:10F23800164B2061A0F800900093019433462946AC
:10F248003846A26865F08FFF002807DA10F1FF0F33
:10F2580032BF0E204042C0B22075D5E72369002B8B
:10F26800D2D0A06865F05AFD7B8D7A8B9A4294BF04
:10F27800C0EB0200C0EB0300E3681B78984294BF20
:10F2880000200120C1E70120BFE700BF354D07007E
:10F298002DE9F04182B000AF0446884600220023E1
:10F2A80039463B4822F082FE0546B0B16D4688B02B
:10F2B8006A46384BCDE90534032342F8103F002352
:10F2C8004FF4C2513448F4F767FFAD466FF00B06B0
:10F2D80030460837BD46BDE8F081F6F797FA2F4B60
:10F2E80029461A582E4B38681A602C2285F09EFF42
:10F2F8003B6800221C603C680023C4E90155C4E94E
:10F3080009552848391D7D6022F050FE064688B10F
:10F3180023686C4688B06A462349CDE90513032360
:10F3280042F8103F4FF4C4512B461B48F4F734FF02
:10F33800A546CBE70146B022786885F077FF786864
:10F348001A4B83605C306AF0FEF87B685433D3E86C
:10F35800EF2FC3E8E16F0029F9D17B681C60636A6D
:10F368007D681BB904F10C006AF0EDF8626A05F1DA
:10F37800A803C5F8A820A26A636202B9A36217228B
:10F388007B685A855A830433C8F80030A0E700BF69
:10F39800601D002062610A00B05C090008000000DE
:10F3A800DC5200207C1D002087610A00D80800205C
:10F3B80008B5437B072B06D002210C4A0C4865F0A0
:10F3C800C5FC002008BD042165F094FC10B9094A69
:10F3D8000121F3E700F15003D3E8AF3FDB0701D485
:10F3E800054AF5E750F8040CECE700BF325F0A0065
:10F3F800B05C0900AC610A00DF5F0A002DE9F04F3C
:10F4080085B000AFB860EFF31188202383F312882A
:10F41800BFF36F8F584C204665F076FC266805468A
:10F4280088F31188BFF36F8F00285FD0F6F704FDCB
:10F43800182202FB00F35149C81851F803A00369C8
:10F448000021D0E90248FB6090F80490B0F806B0BB
:10F4580085F0ECFEA87AF6F7E7FC6969034659B12E
:10F468006A7AD00706D45A6A284612687B6092687E
:10F4780090477B6800226A61294618466AF0B4F80A
:10F48800B9F1000F0DD064B1236853B11B6843B1C3
:10F49800BAF1000F2ED001215346394A394862F09B
:10F4A8005FFE1EB30020B9686AF099F900281DDADA
:10F4B8006C468AB06A46344B0593344BCDE9063026
:10F4C8004FF40073ADF82030314B42F8103F002361
:10F4D8004FF411512B48F4F75FFE0023A54683F340
:10F4E8001188BFF36F8F0323184602DF1437BD4618
:10F4F800BDE8F08F201D65F031FF4846FFF75CF846
:10F508000528CED801A353F820F000BF59F5000014
:10F518002DF50000ABF4000059F50000ABF4000035
:10F528002DF5000004F15403D3E8AF3FDA0705D402
:10F538000121184A134865F009FCB2E7A36D002BB6
:10F54800AFD00023144A04F1780023F0FBF9A8E7B0
:10F5580054F8543B1D68D4E8AF3FDB07E8D5B8F151
:10F56800000F9ED0002403E02846F968C047013404
:10F57800A3B29B45F8D894E78C52002094520020FF
:10F58800C7610A00B05C0900E6610A0067BB0A00AF
:10F5980004000001DF5F0A001C4E0E00F8B50F469C
:10F5A8001646FFF705FFB0B1446A20461CB150F873
:10F5B800A84904B1A83C731C194638B1428B458D43
:10F5C800AA4228BF2A469A4207D264B902210A4AA7
:10F5D8000A4862F0C5FD0020F8BD32463946BDE84C
:10F5E800F840FFF701B9D4F8A85005B1A83D204666
:10F5F8000B462C46E2E700BF01620A00B05C090036
:10F6080007B50B4600210246F6F700F901910E49AD
:10F6180009580E480068884204D00D48D0F8E00028
:10F62800884201D10022134601A90A4822F0BEFCF3
:10F63800014638B91C22019885F0F8FD019803B0FD
:10F648005DF804FB0020FAE708000000DC52002007
:10F65800783E0020981D002010B50022044600F1D5
:10F668000803D3E8EF0FC3E8E12F0029F9D108B167
:10F67800F6F782FC2146BDE81040014869F041BE1A
:10F68800981D00202DE9F743044678300F46904630
:10F698001E466AF0E4F8A06D50B90221144A1548D4
:10F6A80065F054FB204603B0BDE8F04300F086B88F
:10F6B800114B98424FF0000317D045684360A06D86
:10F6C800D0F81890FFF7C8FF00232068A36565F0FD
:10F6D80076FE3DB12068CDF8009043463A46314663
:10F6E8000068A84703B0BDE8F0831D46ECE700BFFB
:10F6F8001C620A00B05C0900E0520020F7B550F81F
:10F70800044C0546002C55D000F1A40104F1240056
:10F7180065F05DFC2E1F05F15807002200233846CE
:10F7280022F004FE024658BB6B6D2BB101466FF008
:10F7380067033046FFF7A6FF002345F8043C05F1B0
:10F748005003D3E8EF1F21F00101C3E8E21F002AAC
:10F75800F7D1636A73BB04F10C060022002330461C
:10F7680022F0E4FD78B9666886B921461248266019
:10F7780069F0C7FD286803B0BDE8F04002F0DEBEBE
:10F78800F6F7FAFBC9E7F6F7F7FBE6E7A26833688E
:10F798009642636008BFA36077683FB1B3696FF0B2
:10F7A80067010093002320681A46B8473046FFF7E0
:10F7B80053FFD8E703B0F0BD601D002010B5044624
:10F7C8000430FFF79BFF1321606865F068F8034673
:10F7D80030B1BDE810400121024A034862F0C0BCC4
:10F7E80010BD00BF33620A00B05C0900F0B589B0F3
:10F7F800044654F8783D00AF38461968FEF728FAF1
:10F808006E4688B06A460B4BCDE905374FF4007356
:10F81800ADF81C30084B42F8103F00234FF4E2517A
:10F828000648F4F7B9FC2046B546FFF7C7FF24376A
:10F83800BD46F0BD51620A0003000001B05C09003A
:10F8480070B550F8043C0446061F002B3BD039B174
:10F85800436D002B37D01B7CDA0734D505231CE019
:10F868000568284602F0B2FD6B7A012B2BD0646D37
:10F878004CB3237CDB0726D5E368002BEED030465B
:10F888006269617CFEF7B0FF054668B9637C0121B7
:10F898000D4A0E4862F064FC0E2300223046BDE893
:10F8A80070401146FFF7EEBEE368D4E905129847A9
:10F8B80018B12846F6F760FBEEE729463046FEF712
:10F8C800B5FE0028F5D170BD7D620A00B05C090064
:10F8D80038B5836D044623B3164A934221D0CB68CA
:10F8E800DD78F5B1052D406815D00F2D1AD1437A72
:10F8F800012B17D8022165F065F808B1103011D135
:10F9080004F1780069F0ABFFA26D137C43F00103AA
:10F918001374002038BD437A032B03D8064AD15C00
:10F92800E9E70E2500222B4611462046FFF7AAFEDE
:10F93800EFE700BFE052002063BB0A0010B50C4699
:10F9480008B301B3FFF734FDE8B1436A3BB153F89C
:10F95800A82902B1A83A996D8C4206D062B9043040
:10F96800214665F034FB204602E02046064A9A65A7
:10F97800BDE81040FFF770BED2F8A81001B1A83951
:10F9880013460A46E7E710BDE0520020F8B51D46C9
:10F998000F461646F6F750FA1823044C03FB0040AE
:10F9A8000123C0E90376C3800575F8BD9452002091
:10F9B80008B584F06CFC38B101210346034A0448B9
:10F9C80065F05EFE6FF0040008BD00BFA4620A0087
:10F9D800085D090010B51846144607491022A047CB
:10F9E800041E07DA01212346044A054865F048FE4B
:10F9F800204610BD0024FBE7E0300020BA620A0070
:10FA0800085D090070B50D4C064623780D46834203
:10FA180004D12846611C65F089FE58B9237CB3429D
:10FA28000AD12846064965F081FE10B1012004EB91
:10FA3800001070BD0020FAE70020FAE714530020F8
:10FA48002553002070B50D4C064623780D46834299
:10FA580004D12846611C65F069FE58B9237BB3427E
:10FA68000AD12846064965F061FE0028054808BF06
:10FA7800002070BD2046FCE70020FAE7883000200F
:10FA8800953000209430002070B50E4C0546237840
:10FA98000E46834203D1601C65F048FE68B9237B9B
:10FAA800AB420CD13146084865F040FE20B1012038
:10FAB800404200F00C00204470BD0020F8E7002010
:10FAC800FAE700BFBEA50020CBA5002038B50C463C
:10FAD80019466BB103F114055B698AB9E268A36042
:10FAE800954200D1E36000230D681A464B61A84790
:10FAF800A3685BB9601C0649BDE8384065F043BEA1
:10FB08001360E3689D4208BFE260ECE738BD00BFC0
:10FB18008ABA0A0070B5204B144682689A420FD1FF
:10FB2800A568C66875B922793046216865F006FE71
:10FB3800024628B11949013065F025FE1570158176
:10FB4800012070BDE0680028FBD02B888B420AD0CA
:10FB5800F6D2E068A36801380433E060003818BFC3
:10FB68000120A360EDE7256822792946304665F033
:10FB7800E5FD024660B93046084965F0DFFD0246FA
:10FB88000028E6D02946013065F0FDFD2379137081
:10FB9800A3685B881381DCE7710001008ABA0A0058
:10FBA800102110B50648F9F799FB034630B1BDE8B6
:10FBB80010400121034A044865F062BD10BD00BF32
:10FBC800D0300020DB620A00085D090038B5054620
:10FBD80048B1154B1A4613F8011C5C1E64F053FF1C
:10FBE80058B1204606E011490F4865F09FFD78B1ED
:10FBF8000D4B581E38BD0020FCE72846217C04F137
:10FC0800110264F040FF0028F5D004F11000F1E77C
:10FC1800054B064903F1100065F088FD0028EAD07D
:10FC2800014B03F10F00E5E7155300208ABA0A00DB
:10FC380010B54A1C0C4628B1097864F024FF30B18D
:10FC4800204610BD1046034965F070FDF7E7002017
:10FC5800F7E700BF8ABA0A0038B5054648B1154B20
:10FC68001A4613F8011C5C1E64F00DFF58B12046BB
:10FC780006E011490F4865F059FD78B10D4B581E43
:10FC880038BD0020FCE72846217C04F1110264F00D
:10FC9800FAFE0028F5D004F11000F1E7054B0649FB
:10FCA80003F1100065F042FD0028EAD0014B03F192
:10FCB8000F00E5E7495300208ABA0A002DE9F04110
:10FCC80006468846174664F00EFA60B34146304649
:10FCD800FFF7B8FE0546B0B9144865F0CEFC0446F7
:10FCE800F8B1134865F0C9FC68B90124114D6342A5
:10FCF800114A03F00C030133D018414665F043FD67
:10FD08000C235C431655012105F10800B94065F044
:10FD180024FDBDE8F04147F612220023074822F0EF
:10FD280011BE054DE3E7BDE8F08100BF903000202B
:10FD38009C3000209430002088300020A030002023
:10FD48000246014610B5042311F8010B0832F9F7F1
:10FD580083FA034630B1BDE810400121024A034846
:10FD680065F08EBC10BD00BF01630A00085D090084
:10FD7800022110B5094865F0F0FC084007D1084990
:10FD8800084A0B88084CA24202D300B10B8010BD70
:10FD98005068083203449BB20120F4E73453002032
:10FDA800D6A50020985C0900A85C090008B50121C7
:10FDB800024A034865F03AFD002008BD1D630A00A9
:10FDC800085D090038B514460E4B82680D469A4204
:10FDD80015D122792168C06865F0B0FC78B1D4F8F3
:10FDE800C8302F2B03D9FFF7E1FF002038BD04EB03
:10FDF80083021581018901335181C4F8C83001207B
:10FE0800F4E700BF7100010008B50121034A044866
:10FE180065F00CFD6FF0150008BD00BF71630A00A6
:10FE2800085D090038B51546084B82689A420AD120
:10FE3800C46829680134204665F078FC18B120466A
:10FE4800696865F0A0FC012038BD00BF71000100A1
:10FE580008B513468168074A914209D11A79196889
:10FE6800C06865F06BFC18B1002303604360038130
:10FE7800012008BD7100010040F239120023014839
:10FE880022F060BD6831002008B50421084865F0FB
:10FE980064FC6FF00201064865F06AFC044865F0EE
:10FEA800ECFBC30701D5FFF7E7FF002008BD00BF43
:10FEB80098310020024608B50749013065F063FC17
:10FEC80000230C3202F8043CD2E8EF1FC2E8E03FFE
:10FED8000028F9D108BD00BF8ABA0A002DE9F0430D
:10FEE80085B00E4690469946044600AF58B90121A0
:10FEF800344A354865F09AFC6FF0150528461437E2
:10FF0800BD46BDE8F08307F1080163F06DFF0546C3
:10FF1800A0B16D4688B06A462C4BCDE905344FF444
:10FF28000073ADF81C302A4B42F8103F00234FF401
:10FF3800E2512548F4F730F9AD46DDE72046391D92
:10FF480062F029FB786858B10A2229465CF022FD44
:10FF5800034628B101211F4A1B4865F091FBCBE7F6
:10FF6800002007F10801FFF78FFD044620BB002E93
:10FF7800C4D01949FFF788FD044638B90121174A4A
:10FF8800114865F053FC6FF00B05B7E7002307F144
:10FF9800080100F8013B65F0F6FB04F108010422B2
:10FFA8004846C047041EA9DA012123460C4A0648E0
:10FFB80065F066FB2546A1E7002EEED10660466097
:10FFC80086609BE7064A0A00085D09007D630A000F
:10FFD8000300000199630A008ABA0A00B4630A00A0
:10FFE800BA620A002DE9F04706460D461D48002171
:08FFF80090461F469DF820A071
:020000021000EC
:10000000DDF82490FFF700FB044688B1456080F8D6
:1000100011A0C0F81490C760C0F818804A46514635
:100020003046FFF7BFFA054638B92046FFF718FB00
:100030006FF00B052846BDE8F0870022012311462A
:10004000FFF7A8FC2846A56042464946B847054642
:1000500018B12046FFF704FBECE72146304665F077
:1000600088FA05460028E5D0F3E700BF1C4E0E00D5
:100070002DE9F0471F46BDF8203006468846D1F8E6
:100080000C90002B4ED17B1E012B4ED8012F4946E0
:100090000CBF15781588FFF7CFFD0446B8B915B920
:1000A0003846BDE8F0874946FFF7C6FD044638B933
:1000B0001F4802211F4A65F0BDFB6FF01000F0E7FA
:1000C00006F17001013065F062FB337A2370D9F8D4
:1000D0001030DBB9B4F808A02581B9F80A30AB427A
:1000E00003D04946404665F0A7FBAA4505D000224B
:1000F000307A06F17001FFF7E5FD002DD0D10E49F1
:10010000601C65F044FB25702581C9E72A464146FD
:10011000304698470028C4DB01380128DAD96FF04F
:100120000D00BEE76FF00600BBE76FF00C00B8E70C
:10013000085D0900D6630A008ABA0A002DE9F04179
:1001400080460F4616461D46FFF7A2FC044680B9BE
:100150001749FFF79DFC044630B9BDE8F041012185
:10016000144A154865F066BB394600F8018B65F006
:100170000EFB238973B9628972B926816581214694
:1001800011F8010B63F0B3FF80B12046BDE8F041E8
:10019000FFF7DABD9E4204D36289AA4206D29E428C
:1001A000ECD263892681AB42E9D2E7E7BDE8F08172
:1001B0008ABA0A00F0630A00085D090010B5FFF76B
:1001C00067FC044678B1014611F8010BF9F756F8BF
:1001D000034620B10121044A044865F055FA002382
:1001E00023606360A36010BD0F640A00085D09000E
:1001F0002DE9F041214B1546826807469A4202D10B
:10020000C4686389E3B90120BDE8F08105F1700895
:100210004146287A63F06BFF68B9194B9C4202D1C2
:10022000284665F019FD3046164965F0B0FA0023FE
:100230002370238119E04146304665F0A8FA14E0A6
:10024000238993B1264616F8011B2846324664F0EE
:100250001EFC0028DAD131462078FDF759FC20B188
:10026000457BFCF7E1FF072DCDD00021E3686181DC
:10027000002BC8D038469847C5E700BF7100010081
:10028000380900208ABA0A0073B50C4605460821D1
:1002900004F11000164665F064FA12230422314678
:1002A000CDE9003228462246024BFFF79FFE02B0FE
:1002B00070BD00BFA55C070038B505460C460F4869
:1002C000012165F04EFA10F0010F0D4B0AD11D838C
:1002D0005C830A4865F0D5F9830709D4BDE8384046
:1002E000FFF7CEBD198B5A8BA94202D89442EFD8A2
:1002F00038BD94421D83ECD9EAE700BF9831002055
:10030000483100202DE9F0419846BDF818300646E6
:10031000012B174636D84344012B454635DCFFF701
:1003200059FC044668B9FFF755FC044648B9022158
:10033000194A1A4865F07EFA6FF010052846BDE8A4
:10034000F081B8F1000F11D00023217A21FA03F2D5
:10035000D00703D53A78DA40D20719D50133032BF9
:10036000F4D13B7803F007031943217206F17001C1
:10037000601C65F00CFA337A01212046237065F089
:10038000B6FCDBE76FF00605D8E76FF00C05D5E7A4
:100390006FF01205D2E700BF2C640A00085D090067
:1003A00010B56FF0020104460E4865F0E5F90D48FE
:1003B00065F067F9C20704D5002200230A4822F03D
:1003C000C5FA204665F00BF958B12046FFF702FC4C
:1003D00038B1037ADB0704D5BDE81040012165F090
:1003E00086BC10BD983100206831002070B56FF0D8
:1003F0000801184865F0C0F940F239120023164888
:10040000F8F7D0FD0026154C651C2846144965F008
:1004100091F9B0B9237ADB0713D52946FDF778FBAC
:10042000054620B165F0DDF82846FCF7FDFE6FF0CB
:10043000020104F10C0065F09FF90021204665F0EF
:1004400056FC731C022B4FF0010604F11004DBD1A3
:1004500070BD00BF98310020F03000201453002000
:100460008ABA0A002DE9F04385B0894616469846B7
:10047000044600AF58B90121414A424865F0DAF913
:100480006FF0150528461437BD46BDE8F08307F127
:10049000080163F0ADFC0546A0B16D4688B06A4620
:1004A000394BCDE905344FF40073ADF81C30374BB0
:1004B00042F8103F00234FF4E2513248F3F770FE48
:1004C000AD46DDE72046391D62F069F8786858B11D
:1004D0000A2229465CF062FA034628B101212C4A1F
:1004E000284865F0D1F8CBE7002007F10801FFF7B5
:1004F0008DFA044690B9FFF76DFB044638B9012127
:10050000244A204865F096F96FF00B05BAE70023FE
:1005100007F1080100F8013B65F039F9B9F1000F66
:100520002AD0022239464046B047061E07DA01218A
:100530003346194A134865F0A7F83546A2E73B78D9
:10054000022E237209D00221144A0E4865F072F976
:100550000021204665F0CBFB94E77B78012B05D981
:100560000F4A3146074865F08FF8F1E7204603F05F
:10057000010165F0ACFB85E72046FFF79FFC81E7B2
:10058000064A0A00085D09007D630A0003000001B5
:1005900099630A0058640A00BA620A007A640A0081
:1005A000CE640A0037B504460D46FFF72FFA02461F
:1005B000D0B1037A0C308DF8043065F062F810F099
:1005C000010318BF01238DF80530022301AA294633
:1005D0002046F8F75BFE034620B10121034A044898
:1005E00065F052F803B030BD0346F0E71F650A001E
:1005F000085D0900104908B5104865F09BF80146F0
:1006000040B90E4B581E65F062FB0C4911F8010C05
:10061000FFF7C8FF08490A4865F08CF8014650B951
:10062000084865F054FB084B187C03F11101BDE844
:100630000840FFF7B7BF08BD8ABA0A00155300206B
:1006400025530020245300201453002008B5012115
:10065000114865F086F8C3071CD4FFF78DFB0F49DE
:100660000F4869F0F2F8002340F239120C48F8F70D
:1006700093FC0C490C4869F0E8F802210B4865F03E
:1006800070F80B480B4969F0E0F8BDE808400A48EB
:10069000FDF7F2BC08BD00BF34530020215E070007
:1006A000F03000206D1201006831002098310020E8
:1006B000A0300020B15E07001009002003462DE99C
:1006C000F04148B1008A38B901244FF0140C1149A7
:1006D000DFF844E0714501D3BDE8F081D1E900764F
:1006E000BB4204D30CFB0672143A93420ED9344435
:1006F000A2B214460831EDE70CFB0578434507D05C
:1007000001356219AE4292B2F6D1F2E70025F8E760
:100710001046E1E7985C0900A85C09002DE9F74F55
:1007200099464FF6FF73BDF830400746002C08BFCE
:100730001C46444B90461B880091834252D2424B48
:100740001D68002D43D04FF0140B083DAE682EB14C
:1007500056F8083C1B8ABB4203D900266B689E42B0
:1007600043D3AD68002D32D0083DEFE773682B44CA
:10077000BB4234D29DB20836344B9E42F6D3DEE7FC
:100780004046D15863F05AFBA0B101350AF1010A85
:10079000ADB273685345EED9009B9D4217D8BD4258
:1007A000F3D3142303FB0AF3326802EB030BB8F113
:1007B000000FE5D1B9F1000F0CD1013CA4B22946DC
:1007C00058460E9A0D9B98470CB10028DDD103B016
:1007D000BDE8F08FDBF80C309945D6D1EDE74FF04E
:1007E000000AD6E701251A4EC6E70BFB06F2296878
:1007F000009801EB020ABAF810309842E7D39F4202
:1008000018D8B8F1000F0DD1B9F1000F14D1013C87
:100810001946A4B250460E9A0D9B9847002CD6D08C
:1008200040B9D4E740468958019363F007FB019B28
:100830000028E9D0013691E7DAF80C209145F9D18A
:10084000E5E700BFD6A5002038530020A85C0900CA
:10085000985C090010B59EB010220021684684F013
:10086000E9FC142200210DEB020084F0E3FC4FF4BC
:100870001053ADF8103080231022ADF812304FF431
:100880008063284C6946CDE906340DEB02001CABB1
:1008900083F090FB034630B1234A0121234864F0E2
:1008A000F3FE1EB010BD014648220AA884F0C2FC27
:1008B00022461C990AA883F0EBFC034660B1012193
:1008C0001B4A1A4864F0E0FE1C9883F0A9FA03461C
:1008D0000028E6D0174AE0E74FF6FF710120164ADC
:1008E0000AAB65F092FA1022144904AB0AA883F00F
:1008F000EDFC04461C9883F093FA14B1104A234689
:10090000CBE708220D4B03F11001187811F8014DC7
:10091000013A03F8014B0870F7D10821094864F047
:1009200020FFBEE70002C00348650A00085D090019
:1009300071650A008F650A008D560700D0300020CF
:10094000A5650A00983100202DE9F04118490446B8
:10095000A1F1300015461E46BDF8187068F09AFFE8
:10096000144864F08EFE010705D4FFF773FFFFF70C
:1009700041FEFFF719F92046FFF72CF968B1037A19
:10098000DA070AD500F10C04204664F07AFEC307AA
:1009900003D40221204664F0E4FE10233A46069375
:1009A00031462846BDE8F041034B65F092B800BFE0
:1009B0002031002098310020D030002010B51B4895
:1009C00064F05FFEC0F3C00080F0010408B9FFF7D7
:1009D00041FF164864F055FE0346144864F051FE8A
:1009E000DA0622D5830606D5FCB1FFF703FEBDE883
:1009F0001040FFF7D9B820210C4864F0B2FE102255
:100A00000B49881884F01EFC48B90A4868F02BFF8F
:100A1000BDE810406FF00101044864F0ADBE4FF630
:100A2000FF710120FFF748FCDFE710BD983100207F
:100A3000D03000206831002008B51021034864F050
:100A400090FEFFF7BBFF002008BD00BF98310020DB
:100A50002DE9F3470446624864F013FEC10713D43E
:100A6000FFF78AF92368002518684FF4C0536946D8
:100A70008DF80050ADF8023063F0E0F960B96FF026
:100A8000770002B0BDE8F087564864F0FAFD4207EF
:100A9000E6D46FF01500F4E7236801A9186841F661
:100AA00001038DF80450ADF8063063F0C7F9002853
:100AB000E5D04D4D22F0F6FA2B6826689BB9002E42
:100AC00065D1002204F10803A2606A68002A68D197
:100AD000C5E90033424864F0D4FDC30771D422F065
:100AE000F5FA0020CDE76B68002B77D053E902328E
:100AF000142101FB023333F8047C002E4FD1002F68
:100B0000DFD023681E8ABE42DBD829680029E1D0E5
:100B10000022A1F108031868008AB0424AD904F102
:100B20000803002A40D09168A1600029CDD09360CD
:100B3000D0E7F37C318A23F08003F37489B9791C00
:100B4000DBB289B243F080033182F3740F4609F1BE
:100B5000FF3914361FFA89F9B9F1000FE9D1474678
:100B6000CDE78F42F2D301AB0846204ACDF804A06E
:100B700065F04BF9019B43B1338A01211C4A1D48A2
:100B800064F082FD22F0A2FA83E73946DEE7984658
:100B9000194A17884FF0000AB4F80490DCE7B84609
:100BA000F8E713606B6095E76A68A1602B60002A24
:100BB00090D1F7E7986800288CD01A46A0F1080376
:100BC000A9E71421D4E9002301FB0323108A33F899
:100BD000041CFFF771FBFFF709FC80E71B68FFDED1
:100BE000345300209831002038530020235607004A
:100BF000BB650A00085D0900D6A500202DE9F04F6D
:100C0000B9B000AF0C46904638493A46D7F80801CB
:100C1000994661F0A0FC40B9FFF7FAF86FF01505AE
:100C20002846E437BD46BDE8F08F3E68391D3046A2
:100C300061F0B5FC3EB901212D4A2E4864F0FAFD61
:100C40006FF015043FE0786800BB4FF0000B07F130
:100C5000080A5146304687F814B063F0C9F80546D3
:100C600008B36C4688B06A46234BCDE905364FF48D
:100C70000073ADF81C30214B42F8103F4FF4E251A5
:100C80005B461C48F3F78CFAA546D9E70A220021F7
:100C90005BF084FE03460028D7D00121184A15488E
:100CA00064F0F2FCCCE7C7F810A0E4B1C0224846DB
:100CB00007F12001C047041E07DA01212346114A2B
:100CC0000C4864F0E1FC2546AAE7A40807F12003DC
:100CD000C7E906344FF6FF7101200B4A07F11003F4
:100CE00065F093F89CE72346F2E700BFDC650A0055
:100CF000064A0A00085D09007D630A00030000013E
:100D000099630A00BA620A001DFB0000002330B597
:100D1000B5B001918DF808003393044601AB0D4640
:100D200001204FF6FF710B4A65F06FF8339B73B1EA
:100D30009B0003AA29462046F8F7BEFA034620B1D5
:100D40000121054A054864F09FFC35B030BD1A46C4
:100D5000F0E700BFCDFD0000E3650A00085D090073
:100D60002DE9F34100F17008CDE9001204460F4669
:100D7000007A4146154663F0BAF906466B464FF6CF
:100D8000FF710120214A65F040F81EB14146207AEA
:100D9000FFF7BCFF3946207AFEF738FE40B12946FE
:100DA000013064F0F4FC1EB14146207AFFF7FAFBF3
:100DB00094F8088039464046FEF76AFE0446C8B1FA
:100DC00029464046FEF764FEC8B1844217D0228906
:100DD000638952EA030106D00589418995420CD8FE
:100DE000994200D24381002323606360A3600EB167
:100DF000FEF7AAFF02B0BDE8F0810281F0E7601CB7
:100E0000294664F0C4FC2046F1E700BF2DFE000037
:100E10002DE9F74F1421054603681A8A00924268AB
:100E200001FB023333F804BC22F03CF9384805F1E9
:100E3000080164F0F6FE814600285ED122F046F9F2
:100E40006FF0010003B0BDE8F08F14222B6802FBA5
:100E50000434304AA368934219D094F91330002B1C
:100E600005DA236923F000431B0C1B0423610AF1FC
:100E7000010A6B681FFA8AF4A342E6D8264864F098
:100E800000FCC3073CD422F021F90020DAE700235C
:100E9000E668224906F101084046738164F04AFC85
:100EA00007460028D9D141463078FCF731FE034689
:100EB00048B94146307863F01AF9A0B1414630781C
:100EC000FFF724FF0FE0427B072A14D100F17001E5
:100ED0003A46007A0193FEF7F5FE019B1846FCF7AF
:100EE000A3F9002FE5D140460C4964F050FC0023E3
:100EF00033703381B1E74F46F0E74FF0000AB8E7AF
:100F000059460098FFF7D8F9FFF770FABBE700BF22
:100F10003853002071000100345300208ABA0A00BF
:100F2000002307B50193FFF7C9FB411C89B20846AE
:100F3000034A01AB64F069FF019803B05DF804FB5C
:100F4000E75B07002DE9F04387B0437B8046072B22
:100F50000C46154602AF40F0A68000233B7342F6D4
:100F60000303206807F10C01FB8162F067FF06466E
:100F7000002834D1D4F80490B9F1000F05D1012133
:100F80004B4A4C4864F056FC8DE00123214600900A
:100F900007F10802C847031E11DA6D4688B002AA9D
:100FA000D36104234449C2E9051442F8103F4FF4C9
:100FB000015133463F48F3F7F3F8AD4673E0012B98
:100FC00005D001213D4A3B4864F05EFB6BE03B7A73
:100FD00013F0300F67D02046FFF7A2FF044600232E
:100FE00020683B7342F6021307F10C01FB8162F0AB
:100FF00025FF18B12046FFF793FF0446002642F66E
:101000000219206839463E70A7F8029062F016FF78
:1010100018BB002320683B7342F6021307F10C0152
:10102000FB8162F00BFF064600283CD1D4F8049007
:10103000B9F1000FA3D0022300902146404607F1EA
:101040000C02C847031EA8DB022BBAD1BB8905EAF4
:101050000300003818BF012026E042F60303206891
:10106000391D3E71FB8062F0E9FE0028D1D04FF4BB
:101070002053206807F108013E727B8162F0DEFE9A
:101080000028C6D042F60103206807F10C013E7328
:10109000FB8162F0D3FE0028BBD02046FFF740FF63
:1010A00004460028ADD100201437BD46BDE8F083CA
:1010B00001660A00085D090015660A003B660A0021
:1010C0002DE9F8431546894694226968064664F07E
:1010D0002AFF8046002841D1022230466968FFF786
:1010E00031FF00283DD000211F48AF8AFEF78CFA5F
:1010F0000237044680B11D211C4B47613A464174BA
:10110000C0F80C80436085613046FEF74BFA074615
:1011100038B92046FEF7A4FA6FF00B052846BDE863
:10112000F883012342464146FEF734FCA98A07F1C1
:101130000C00023161F030FC20F8029BAA8A296978
:1011400084F052F821463046A76064F012FA054652
:101150000028E3D02046FEF783FADFE74FF0FF35A3
:10116000DCE76FF01505D9E71C4E0E002956070085
:1011700070B505468AB03A4864F083FA42070C46D7
:1011800067D515B16B7B072B66D16668304605962F
:10119000FFF794FA2268ADF81800002A2FD005A9AD
:1011A0000291304900230191012100914FF6FF7116
:1011B0000593FFF7B3FA059E1EB96FF001000AB060
:1011C00070BD6660002330688DF8103042F603036E
:1011D00004A9ADF8123062F031FE40B90598C36839
:1011E0009B799B0608D564F0C9FDADF818000598F9
:1011F00064F06EFE606028B96FF01500DFE700282C
:10120000E0D1DAE7BDF818003DB1012301462246DE
:101210002846A375FFF754FFD1E76FF07F030793CC
:101220000223ADF8203042F60213ADF8123005ABC0
:10123000A57502930C4B4FF6FF710193012304AA8D
:1012400000932B4609948DF81050FFF767FA079822
:10125000B5E76FF00A00B2E76FF07F00AFE700BFBD
:101260000802002057560700D114010073B5044648
:1012700050F8083C00F130056FF00101A0F12006A4
:101280002846019364F078FA0D4B002044F81C3C8A
:101290000C4B314644F8183C01AB44F8103C042395
:1012A00024F8080C24F8060C24F80C3CFFF760FF27
:1012B00018B90221284664F054FA02B070BD00BF8C
:1012C00004680900A10301002DE9F84316463A4BD2
:1012D000826805469A4200AF24D1D0F80C80346869
:1012E000B8F80830F3B14246204612F8011B63F00B
:1012F000CEFBB8B14FF495722946204664F013FE38
:1013000028B3032812D16C4688B06A462B4BCDE92E
:10131000053542F8100F00234FF4C4512848F2F766
:101320003FFFA5460120BD46BDE8F88305282046BD
:101330000CBF4FF003094FF0020963F078FB8145C1
:1013400005D933794B45EDD286F80490EAE741465A
:10135000284664F071FA1B4B9845E3D1207A04F1DA
:101360007001FEF795FB05460028DBD0038913B911
:101370004389002BD6D02046FCF7DAF82A89124B95
:10138000124923F820206A8903EB80035A8018222F
:1013900002FB00110B6104230D4A20464A600D4AEE
:1013A0008B828A60FFF7E4FE0028BBD001210A4A45
:1013B000034864F03FFAB5E77100010054660A0083
:1013C000085D090038090020BAA50020FC52002061
:1013D000046809000B5D070068660A0070B50446E2
:1013E0008AB0384864F04DF942070D4663D514B110
:1013F000637B072B62D16E6830460596FFF75EF976
:101400002A68ADF81800002A2FD005A902912E49AC
:1014100000230191012100914FF6FF710593FFF721
:101420007DF9059E1EB96FF001000AB070BD6E60B7
:10143000002330688DF8103042F6030304A9ADF89C
:10144000123062F0FBFC40B90598C3689B79DB065B
:1014500008D564F093FCADF81800059864F038FDE9
:10146000686028B96FF01500DFE70028E0D1DAE7FF
:10147000BDF818002CB101462A46204664F08EFDC6
:10148000D3E76FF07F0342F6021207930123ADF812
:10149000122005AA02920D4AADF82030CDE90032A3
:1014A0004FF6FF71234604AA09958DF81040FFF707
:1014B00035F90798B9E76FF00A00B6E76FF07F00DB
:1014C000B3E700BF0802002057560700D1140100FF
:1014D0002DE9F0413D4B1546826807469A4203D0FC
:1014E00001273846BDE8F081D0F80C80384B98458C
:1014F00012D0B8F80820AB899A42F1D1414611F8D0
:10150000010BFCF705FB06460028E9D0437B072BBF
:1015100024D0FBF789FEE3E700262E4C20462E4917
:1015200064F008F978B90722214614F8010CFCF799
:1015300071FB80B92B6921461A6914F8010C538894
:101540001288FEF7FBFD731C022B4FF0010604F11D
:101550000C04E3D1CDE7FBF767FEF4E7D8F81430CD
:1015600023B13946984708B93046D2E73946942224
:10157000304664F0D8FC07460028F5D1AB89022B31
:1015800015D1B8F808309A071ED530462A69A988BF
:10159000FFF796FD044618B92A69937D01339375C8
:1015A0003046FBF741FE002CAC609ADB98E7012B3C
:1015B0000AD1B8F80830DB0706D530462A69A98871
:1015C00064F0ECFC0446EBE73C46E9E771000100FF
:1015D00038090020BFA500208ABA0A0073B5437BF2
:1015E0000446072B0D461AD1061D4FF480313046B4
:1015F00064F0B7F8C30315D402232046CDE90033C5
:101600002A460A4B0A49FEF7F1FC044620B16FF462
:101610008031304664F0B0F8204602B070BD6FF003
:101620007F04F9E76FF07704F6E700BF6958070019
:101630005F56070070B5437B0546072B0C4686B006
:1016400040F0A1800B7C062B10D8DFE803F00404E7
:101650005A5A629528000B68CBB11B784BB1022B0C
:1016600013D00121494A4A4864F00EF86FF0150082
:1016700009E0082301930623224600934549464B7F
:101680002846FEF7B3FC06B070BD1623F2E7102320
:1016900004212246CDE90031404B4149F0E708687A
:1016A0000028E3D00678002EE0D14FF4245302A99D
:1016B0008DF80860ADF80A3062F0C0FB08B342F65E
:1016C0000213206803A98DF80C60ADF80E3062F0AB
:1016D000B5FBB0B142F60313206804A98DF8106081
:1016E000ADF8123062F0AAFB58B142F6041320683C
:1016F00005A98DF81460ADF8163062F09FFB002844
:10170000B4D1082304222749CDE900322246264BD2
:10171000B6E7086880B300264FF4205302A98DF87D
:101720000860ADF80A3062F089FB00289ED042F6CE
:101730000103206803A98DF80C60ADF80E3062F04B
:101740007DFB002892D042F60203206804A98DF8A0
:101750001060ADF8123062F071FB002886D042F6BE
:101760000303206805A98DF81460ADF8163062F007
:1017700065FB00283FF47AAF04232246CDE900330D
:101780000A490B4B7CE76FF07F007CE785660A0017
:10179000085D0900476007009B5B0700FD580700D4
:1017A000B5170100D91801002D590700511C01007F
:1017B000955807002DE9F0478EB0064617461C469F
:1017C000169D31B12A4600216B680EB0BDE8F04786
:1017D000184763B902213D4A3D4864F02BF82A4678
:1017E000002130466B6898470EB0BDE8F08713784B
:1017F000062B08D0142B05D00121364A344863F05B
:1018000043FFECE702214FF00008C146013C8DF890
:101810001010A4B207F1010A9C420CD2002CDED1B8
:10182000B8F1000FDBD02A46414630460EB0BDE885
:10183000F04764F0EABB1422002109A883F0FAFC07
:10184000BAF8002093B2002BC9D0BAF802101FFAE0
:1018500081F8B8F1000FC2D04345C0D89DF81030D0
:1018600013B3022B25D02B7CADF80C10002B42F6C5
:10187000010308BF4FF42053ADF8063004AB0293C8
:1018800001AB099302ABADF834200C932A463046E5
:101890006B688DF8049009A998470028A4D03B787C
:1018A000E41AA4B29A44B7E7BAF80430ADF812309B
:1018B000D9E70AF104030DF111000AF1140C53F8F1
:1018C00004EB634540F804EBF9D1CCE79A660A00D3
:1018D000085D0900A4660A002DE9F04F93B0174691
:1018E00080461C460A461C9D31B12A4600216B6881
:1018F00013B0BDE8F04F1847297C022940F08380DF
:101900004BB99B4A9B4863F095FF2A46002140460D
:101910006B6898475BE03B78062B08D0082B05D016
:101920000121954A934863F0AFFEEEE71146002689
:1019300042F6020A013C8DF82010A4B207F1010B17
:101940009C420BD2002CE0D1002EDED02A4631463C
:10195000404613B0BDE8F04F64F057BBBBF80090B1
:101960001FFA89F6002ED0D0BBF802009DF8202087
:10197000ADF81C00BBF80410ADF81E1062B1022ACD
:1019800015D0296831B308A862F058FA10B33B7833
:10199000E41AA4B29B44D3E708AA06929BF8062057
:1019A0009BF8071042EA0122ADF82220E9E70A235A
:1019B0006881A981A5F808904046019200932A46C3
:1019C0006E4B6F49FEF712FB86B2002EBED113B0EC
:1019D000BDE8F08F4FF00003102200210EA88DF813
:1019E0001430ADF816A083F025FC05AA0D9206AAC6
:1019F000109240462A466B68ADF844900DA998476E
:101A00000028C4D1E3E7032966D113B90221584A5B
:101A100078E73B78072B02D0152B81D102220026D4
:101A2000013C8DF82020A4B207F101090DF1200A34
:101A30009C4287D3B9F800B01FFA8BF6002E3FF412
:101A400064AF9DF8203063B1022B13D02968F1B147
:101A5000504662F0F3F9D0B13B78E41AA4B299444D
:101A6000E6E799F8053099F8062043EA0223ADF835
:101A70002230EBE709F105030DF1210209F115010F
:101A800053F8040B8B4242F8040BF9D1DEE799F8C6
:101A90000230B9F803208DF81E304FF000038DF8A6
:101AA000143042F603030021ADF81C200EA81022CA
:101AB000ADF81630CDF818A083F0BCFB05AB0D9344
:101AC00006AB10932A4640466B68ADF844B00DA9AA
:101AD00098470028C0D17AE72A68167876B92BB9DA
:101AE000234A0221234863F0A5FE07E03B78012B3F
:101AF00009D80221204A1F4863F0C6FD2A4600216A
:101B000040466B68F4E6B2F802A0013CA4B207F1CB
:101B10000109AAF5245A9C4204D2002CEED1002ED1
:101B2000ECD013E7012C01D8164ADAE7B9F800B077
:101B30001FFA8BF6002EE1D0BAF1040FDED801A314
:101B400053F82AF0591B0100FD1A0100611B010026
:101B5000691B0100D11B0100032C1BD80A4AC0E7F6
:101B6000032C17D8094ABCE7032C13D8084AB8E756
:101B70009A660A00085D0900A4660A0081580700F9
:101B8000191C0100B8660A00C6660A00D4660A007D
:101B9000E2660A00B9F80230ADF820302B68102256
:101BA00000210EA8039383F045FB039B2A460D9367
:101BB00008AB109340466B68ADF844B00DA9984748
:101BC00000283FF404AF3B78E41AA4B29944A2E79A
:101BD000082C01D80F4A84E799F802308DF820309C
:101BE00099F803308DF8213099F8052099F80430E0
:101BF00043EA0223ADF8223099F806308DF82430FC
:101C000099F8073099F8082043EA0223ADF8263006
:101C1000C4E700BFF0660A0070B5102B05461146F8
:101C2000049C0BD00121084A084863F02DFD224690
:101C3000284663680021BDE8704018472246BDE889
:101C4000704064F04CBA00BFA4660A00085D090049
:101C50002DE9F04F8FB00746189D184629B953B9A2
:101C60000221544A544863F0E5FD2A4600213846D3
:101C70006B6898479BE01378012B07D0022B20D08C
:101C800001214E4A4C4863F0FFFCEEE70B464FF053
:101C90000409013880B248458DF81030E5D34FF083
:101CA0000008B0FBF9FBC246541CCDF8008004AE1E
:101CB000BBF1000F08D12A463846009964F0A5F917
:101CC00075E04FF01209E4E723880193BDF8043072
:101CD0000093B8F1000F53D19DF81030002B37D08E
:101CE000022B3CD02968002945D12B7C042B4DD1F7
:101CF0004FF42053304602A98DF808A0ADF80A3001
:101D000062F09CF800283BD042F60103304603A95C
:101D10008DF80CA0ADF80E3062F090F880B342F66A
:101D20000203304609A98DF824A0ADF8263062F0F0
:101D300085F828B342F60303304609A98DF824A09C
:101D4000ADF8263062F07AF800BB4FF0010819E0D8
:101D5000A378E27843EA0223ADF81230C2E7A31C6D
:101D60000DF1110204F1120153F8040B8B4242F8F9
:101D7000040BF9D1B6E7304662F060F80028B4D021
:101D80004FF000080BF1FF3B4C4491E7102200217B
:101D90000AA883F04FFABDF804302A46ADF8343073
:101DA00038466B68099609A998470028EAD10FB010
:101DB000BDE8F08F9A660A00085D0900FE660A0019
:101DC00007B5437B0A46072B2CD14B683BB9082348
:101DD0004FF0040ECDE9003E144B154909E0012BEC
:101DE00011D0097B5B00019341B12023114900937D
:101DF000114BFEF7FBF803B05DF804FB0E230F490F
:101E000000930F4BF5E74B8933B10C234FF0040CD3
:101E1000CDE9003C0B4BE0E70A230221CDE900317C
:101E2000094BDAE76FF07F00E5E700BFED5B0700E5
:101E30004D1E0100515A070091590700115A070021
:101E400069590700C1580700AD5807002DE9F04F48
:101E500085B002AF804691469A460E463C6B41B92A
:101E60006BB92568002322460093F1B24046A8478B
:101E700030E0B1F5807F28BF0E262568F2E7636861
:101E8000002B71D123890AF1FF35B4F80AB07B60C9
:101E9000ADB202F1010A002D4DD099F80030AB42ED
:101EA00028BF2B46012B0AD802213E4A3E4863F048
:101EB000EBFB00230093224604212568D6E7BAF8FD
:101EC0000020023B91B29BB241B90121374A36480A
:101ED00063F0B0FC0C37BD46BDE8F08F78688842EF
:101EE00001D88B4518D26D468AB002AA304BC2E9A0
:101EF00005317B68C2E9073B052342F8103F002308
:101F00004FF422512848F2F74BF9AD4600230093D5
:101F1000256822460E21A9E722810093224600214E
:101F2000404626680AF10203B0470028D2D099F84B
:101F30000030AB4206D921464046FFF741FF00285A
:101F4000C8DAE3E7238962899A4205D10023009326
:101F500025682246194689E70133238199F8003024
:101F6000ED1AADB29A4496E7CDF800A01346256865
:101F70002246A8470028ADD0238A013B9A4503DAC0
:101F8000009633462568E4E7638921460AEB03059A
:101F900040466581FFF714FF00289BDA0096334620
:101FA0002568B6E710670A00085D090048670A005F
:101FB00057670A0073B5437B0546072B0C4603D0D1
:101FC0006FF07F0002B070BDCB88B3B1284663F0DC
:101FD0004AFA0028F4D0A289431F9BB2934228BF3B
:101FE000134604339BB201931623224600930A49F9
:101FF0000A4B2846FDF7FAFFE4E78E8963F033FACF
